:100000000C9414290C948B4E0C94604E0C94354E29
:100010000C940A4E0C94DF4D0C94B44D0C94894D05
:100020000C945E4D0C9445290C9445290C9445295B
:100030000C9445290C9413EF0C9445290C944529F4
:100040000C9445290C9402DE0C9445290C94452906
:100050000C9445290C9445290C9410D00C947250A2
:100060000C9445290C94AD730C944A740C94452956
:100070000C9445290C9445290C9445290C94452948
:100080000C9445290C9445290C9445290C94452938
:100090000C9445290C9445290C9445290C94452928
:1000A0000C9445290C9445290C9445290C94452918
:1000B0000C9445290C9445290C9445290C94452908
:1000C0000C9445290C9445290C9445290C944529F8
:1000D0000C9445290C9445290C9445290C944529E8
:1000E0000C94452998459B458A458E459445D245B3
:1000F0009F45A345A945AD45B145B745BB45BF455E
:10010000D245C545C945CD45364F3B4F404F4A4F77
:10011000544FCD4F5E4F664F6E4F784F824F8C4F8E
:100120009B4FA54FCD4FAF4FB94FC34F965F965FD3
:100130009D5F9D5F9D5FA45FA45FA45FB15FAB5FA8
:10014000AB5FAB5FE373E973FA7305740D742274EC
:10015000117422741574197422741F74B0D0B4D041
:10016000DDD0E1D0C3D0CED09DD0084AD73B3BCE26
:10017000016E84BCBFFDC12F3D6C74319ABD5683A6
:100180003DDA3D00C77F11BED9E4BB4C3E916BAA5E
:10019000AABE000000803F05A84CCDB2D44EB938AD
:1001A00036A9020C50B9918688083CA6AAAA2ABE94
:1001B000000000803F004E414E494E495459494E7F
:1001C00046CDCCCC3D0AD7233C17B7D13877CC2BC2
:1001D000329595E6241FB14F0A000020410000C867
:1001E0004200401C4620BCBE4CCA1B0E5AAEC59DE8
:1001F00074434F4D4D554E49434154494F4E004471
:10020000525952554E004552524F525300494E4694
:100210004F004543484F0020746F6F206C6F6E672E
:1002200020657874727573696F6E2070726576657B
:100230006E7465640A0020636F6C64206578747264
:100240007573696F6E2070726576656E7465640A89
:1002500000536C6565702E2E2E004C756C7A426FC3
:10026000742054415A20352072656164792E005201
:100270006573756D696E67207072696E7400436C8A
:1002800069636B20746F20726573756D652E2E2EF9
:10029000004E6F206D6F76652E004D313235004671
:1002A000696C652064656C657465643A0044656CCE
:1002B0006574696F6E206661696C65642C2046699F
:1002C0006C653A20006F70656E206661696C6564CC
:1002D0002C2046696C653A20002569730025696DFC
:1002E00020256973002569682025696D20256973BB
:1002F00000256964202569682025696D20256973BA
:100300000025697920256964202569682025696DA3
:1003100020256973005072696E742074696D653AA6
:100320002000000125301D0CFF24311C0BFF232F62
:100330001B0AFFFF040306080202222B1A41422176
:100340002A193F40033809FF3607FF372829452778
:10035000444350726F7465637465642050696E0A1B
:100360000012020D020602FF01F1016F66660044F1
:10037000454255473A006F6B00436F6F6C696E677B
:1003800020646F6E652E0048656174696E67206435
:100390006F6E652E0020573A00457874727564655B
:1003A00072202569202573004C756C7A426F742089
:1003B00054415A20352072656164792E004265648B
:1003C00020646F6E652E0020573A004265642068F5
:1003D000656174696E672E0042656420636F6F6C9F
:1003E000696E672E004C756C7A426F742054415AC6
:1003F0002035204F66662E002F2F20007A5F6D6912
:100400006E3A2000795F6D696E3A2000785F6D6901
:100410006E3A20005265706F7274696E6720656E67
:100420006473746F70207374617475730A0053651C
:100430007474696E672054726176656C20416363E1
:10044000656C65726174696F6E3A200053657474EF
:10045000696E6720526574726163742041636365DD
:100460006C65726174696F6E3A20005365747469CB
:100470006E67205072696E7420416363656C6572AB
:100480006174696F6E3A200053657474696E6720F9
:100490005072696E7420616E642054726176656C6E
:1004A00020416363656C65726174696F6E3A200008
:1004B000205A00205900580020204D61783A200031
:1004C000205A00205900580020204D696E3A200023
:1004D0004F6E20004F666600536F667420656E6431
:1004E00073746F70733A2000486F74656E64206F88
:1004F0006666736574733A0020643A0020693A00B6
:1005000020703A0020643A0020693A0020703A00D6
:1005100043290A0061626C656420286D696E20744D
:10052000656D702000436F6C64206578747275642B
:1005300065732061726520004B642000236465664A
:10054000696E65202044454641554C545F004B6917
:10055000200023646566696E652020444546415548
:100560004C545F004B70200023646566696E652003
:100570002044454641554C545F0050494420417544
:10058000746F74756E652066696E69736865642141
:100590002050757420746865206C617374204B70F2
:1005A0002C204B6920616E64204B6420636F6E7356
:1005B00074616E74732066726F6D2062656C6F7704
:1005C00020696E746F20436F6E666967757261741F
:1005D000696F6E2E680A00504944204175746F742B
:1005E000756E65206661696C6564212074696D654E
:1005F0006F75740A00504944204175746F74756EAC
:1006000065206661696C6564212054656D70657252
:10061000617475726520746F6F20686967680A007D
:10062000204B643A2000204B693A2000204B703A5E
:1006300020000A20436C6173736963205049442091
:100640000A002054753A2000204B753A2000206D96
:1006500061783A2000206D696E3A200020643A20CB
:100660000020626961733A20004F66667365747397
:10067000206170706C696564004572723A20546F35
:100680006F206661722100546F6F20666172206670
:10069000726F6D207265666572656E636520706F3E
:1006A000696E740A00556E6B6E6F776E20636F6DA6
:1006B0006D616E643A2022000000200023002600B5
:1006C00029002C002F003200000100000301060168
:1006D00009014E6F204C696E65204E756D62657222
:1006E000207769746820636865636B73756D2C206F
:1006F0004C617374204C696E653A200053544F501E
:100700005045442E20005072696E746572207374D7
:100710006F707065642064756520746F20657272F7
:100720006F72732E20466978207468652065727236
:100730006F7220616E6420757365204D39393920E0
:10074000746F20726573746172742E202854656D05
:100750007065726174757265206973207265736566
:10076000742E20536574206974206166746572204C
:1007700072657374617274696E67290A004E6F2026
:10078000436865636B73756D2077697468206C6965
:100790006E65206E756D6265722C204C61737420DD
:1007A0004C696E653A2000636865636B73756D20F4
:1007B0006D69736D617463682C204C617374204C97
:1007C000696E653A20004C696E65204E756D6265F4
:1007D00072206973206E6F74204C617374204C69B1
:1007E0006E65204E756D6265722B312C204C6173E5
:1007F00074204C696E653A20004D313130004D3324
:1008000031004D383420582059205A204500534497
:100810002072656164206572726F720A00446F6EA7
:1008200065207072696E74696E672066696C650A0E
:100830000025753A2530327500253032753A25305D
:1008400032750025756420253032753A25303275B1
:100850000000060900FE000000000001090008FE7B
:10086000000005080806000040F0C8888898781045
:10087000050808060000C0F88888888888F80505FB
:10088000050600012030F830200508080600002089
:1008900070F820202020E00509090600FF2070A83C
:1008A000A8B8888870200509090600FFE080C0B05C
:1008B000A8283028280509090600FFF8A888888894
:1008C0008888A8F8050A0A0600FE20505050508873
:1008D000A8A8887003030306000340A0400006098F
:1008E00000FE070192032120FFFF08FF07FF000021
:1008F000000600000107070602008080808080005B
:1009000080030202060105A0A005070706000050AB
:1009100050F850F850500507070600002078A070E6
:1009200028F020050707060000C0C81020409818CE
:100930000507070600006090A040A8906802030326
:10094000060104C0408003070706010020408080A4
:1009500080402003070706010080402020204080BF
:1009600005050506000120A870A82005050506005C
:10097000012020F820200203030602FFC04080056A
:100980000101060003F8020202060200C0C00505CC
:1009900005060001081020408005070706000070CA
:1009A00088888888887003070706010040C0404097
:1009B0004040E0050707060000708808708080F856
:1009C000050707060000F81020100808F0050707C3
:1009D00006000010305090F81010050707060000C0
:1009E000F880F0080888700507070600007080800E
:1009F000F0888870050707060000F80810202020FE
:100A00002005070706000070888870888870050731
:100A1000070600007088887808087002050506023D
:100A200000C0C000C0C00206060602FFC0C000C071
:100A30004080040707060000102040804020100579
:100A40000303060002F800F80407070601008040CF
:100A5000201020408005070706000070880810203D
:100A6000002005070706000070880868A8A8700520
:100A70000707060000708888F88888880507070639
:100A80000000F08888F08888F005070706000070ED
:100A9000888080808870050707060000F0888888B5
:100AA0008888F0050707060000F88080F08080F84D
:100AB000050707060000F88080F0808080050707A2
:100AC000060000708880B888887005070706000057
:100AD000888888F888888801070706020080808057
:100AE00080808080050707060000381010101090E5
:100AF000600507070600008890A0C0A09088050741
:100B000007060000808080808080F80507070600C7
:100B10000088D8A888888888050707060000888884
:100B2000C8A8988888050707060000708888888804
:100B30008870050707060000F08888F0808080052F
:100B4000070706000070888888A8906805070706D0
:100B50000000F08888F0A09088050707060000785C
:100B60008080700808F0050707060000F8202020A4
:100B7000202020050707060000888888888888705C
:100B80000507070600008888888888502005070721
:100B90000600008888888888A85005070706000096
:100BA00088885020508888050707060000888888B4
:100BB00050202020050707060000F808102040807C
:100BC000F8030707060100E08080808080E00505CB
:100BD000050600018040201008030707060100E019
:100BE0002020202020E00503030600042050880573
:100BF0000101060000F80202020602058040050518
:100C00000506000070087888780507070600008050
:100C100080B0C88888F005050506000070808088CF
:100C20007005070706000008086898888878050599
:100C3000050600007088F880700507070600003080
:100C400048E0404040400506060600FF708888786E
:100C500008700507070600008080B0C888888801F2
:100C60000707060200800080808080800308080655
:100C700001FF200020202020A040040707060000DC
:100C8000808090A0C0A090030707060100C04040EC
:100C9000404040E0050505060000D0A8A8A8A8052A
:100CA0000505060000B0C88888880505050600000F
:100CB00070888888700506060600FFF08888F08036
:100CC000800506060600FF7888887808080505056F
:100CD000060000B0C8808080050505060000708011
:100CE0007008F00407070600004040E04040403034
:100CF0000505050600008888889868050505060032
:100D00000088888850200505050600008888A8A866
:100D10005005050506000088502050880506060687
:100D200000FF888888780870050505060000F8101F
:100D30002040F80307070601002040408040402083
:100D400001070706020080808080808080030707FB
:100D5000060100804040204040800502020600025B
:100D6000689000000006000000000006000000007F
:100D70000006000000000006000000000006000061
:100D80000000000600000000000600000000000651
:100D90000000000000060000000000060000000047
:100DA0000006000000000006000000000006000031
:100DB0000000000600000000000600000000000621
:100DC0000000000000060000000000060000000017
:100DD0000006000000000006000000000006000001
:100DE00000000006000000000006000000000006F1
:100DF00000000000000600000000000600000000E7
:100E000000060000000000060000000000060000D0
:100E100000000006000000000006000000000006C0
:100E200000000000000600000000000600000107AE
:100E3000070602008000808080808005070706008A
:100E4000002070A8A0A87020050707060000304009
:100E500040E04050A80505050600008870507088E5
:100E6000050707060000885020F820F82001070732
:100E7000060200808080008080800508080600004F
:100E80003048205050209060030101060107A00562
:100E90000707060000F888B8B8B888F805070706FD
:100EA0000001700878887800F8050505060001281B
:100EB00050A05028050303060001F80808020202AA
:100EC0000602064080050707060000F888A88898F3
:100ED000A8F8050101060006F804040406000360F2
:100EE0009090600507070600002020F8202000F8F9
:100EF00004050506000360902040F0030505060088
:100F000003E020E020E0020202060206408005081D
:100F1000080600FF8888888898E88080050707060B
:100F2000000078989878181818020202060202C089
:100F3000C00202020602FF408003050506000340CE
:100F4000C04040E0050707060001708888887000EF
:100F5000F8050505060001A0502850A00507070662
:100F600000008890A858B808080507070600008800
:100F700090B848982038050808060000C040C048CE
:100F8000D8380808050707060000200020408088A0
:100F9000700508080600004020007088F888880561
:100FA00008080600001020007088F88888050808E6
:100FB0000600002050007088F888880508080600A0
:100FC000006890007088F8888805080806000050BE
:100FD00000708888F88888050808060000205020DE
:100FE0007088F888880507070600003860A0B8E018
:100FF000A0B80508080600FF70888080887020600F
:10100000050808060000402000F880F080F8050878
:1010100008060000081000F880F080F805080806AF
:101020000000205000F880F080F805070706000057
:101030005000F880F080F8030808060100804000A6
:10104000E0404040E0030808060100204000E04086
:101050004040E003080806010040A000E040404096
:10106000E0030707060100A000E0404040E005075C
:1010700007060000704848E8484870050808060060
:101080000068900088C8A8988805080806000040F5
:101090002070888888887005080806000010207075
:1010A000888888887005080806000020500070882D
:1010B0008888700508080600006890007088888895
:1010C0007005080806000050007088888888700540
:1010D000050506000188502050880508080600FF15
:1010E0001070A8A8A8A870400508080600004020B5
:1010F000888888888870050808060000102088887D
:1011000088888870050808060000205000888888B4
:101110008870050808060000500088888888887054
:10112000050808060000102088502020202005090E
:10113000090600FFC040704848704040E0040808BD
:101140000601FF609090A09090E0800508080600DE
:101150000040200070087888780508080600001014
:1011600020007008788878050808060000205000E4
:1011700070087888780508080600006890007008F4
:10118000788878050707060000500070087888788E
:1011900005080806000020502070087888780506A9
:1011A00006060000D02878A0A8500506060600FF15
:1011B00070808870206005080806000040200070DC
:1011C00088F880700508080600001020007088F874
:1011D00080700508080600002050007088F88070B4
:1011E00005070706000050007088F88070030808A3
:1011F00006010080400040C04040E00308080601AE
:101200000020400040C04040E003080806010040C4
:10121000A00040C04040E0030707060100A00040D6
:10122000C04040E0050707060000A040A0107888F5
:1012300070050808060000689000B0C88888880516
:10124000080806000040200070888888700508089B
:1012500006000010200070888888700508080600C5
:101260000020500070888888700508080600006813
:10127000900070888888700507070600005000708D
:10128000888888700505050600012000F800200503
:1012900007070600FF1070A8A8A8704005080806F8
:1012A000000040200088888898680508080600002B
:1012B00010200088888898680508080600002050DB
:1012C000008888889868050707060000500088880D
:1012D0008898680509090600FF102000888888F8AA
:1012E00008700407070601FFC04060506040E00539
:1012F00008080600FF50008888887808705A00594E
:10130000005800092000000000000000000000005C
:1013100000007FFFE000000000000000000000006F
:10132000007000E00000000000000000000000006D
:1013300061F86000000000000000000000000041B3
:10134000F82000000000000000000000000040F055
:1013500020000000000000000000000000406020AD
:101360000000000000000000000000005801A07F05
:1013700080003FC0000000004104005C63A0FBC08F
:101380000079E0000000002082005EF7A0F3C000BA
:1013900076E0000000002082005EF7A0EBC0007E37
:1013A000E0000000004104005C63A07B80003DC0C1
:1013B000000000008208005801A07B80003BC000B4
:1013C000000001041000406020FBC00077E0000036
:1013D000000104100040F020FBC00070E00000009D
:1013E0000082080041F820FFC0007FE000000000FC
:1013F00041040061F8603F00001F80000000000011
:1014000000007000E01E00000F0000000001FFFF60
:10141000807FFFE00C0000060000000001FFFF805D
:101420000000000000000000000000000000007F3D
:10143000FFE000000000000000000000000070005D
:10144000E0000000000000000000000000630C60ED
:10145000000000000000000000000000470E200017
:1014600000000000000000000000004F0F200000FE
:10147000000000000000000000005F0FA00000005E
:101480000000000000000000005E07A07F80003F19
:10149000C000000000410400406020FBC00079E073
:1014A0000000000020820040F020F3C00076E00041
:1014B00000000020820040F020EBC0007EE0000031
:1014C00000004104004060207B80003DC00000001F
:1014D000008208005E07A07B80003BC00000000186
:1014E0000410005F0FA0FBC00077E00000000104C3
:1014F00010004F0F20FBC00070E0000000008208C9
:1015000000470E20FFC0007FE00000000041040003
:10151000630C603F00001F800000000000000070AE
:1015200000E01E00000F0000000001FFFF807FFFB1
:10153000E00C0000060000000001FFFF800000003A
:1015400000000A0B02090C0D0E080703040100003D
:10155000000000000000000000000000000000008B
:101560000000000000000000000000001211100048
:10157000000000000000000000000000000000006B
:10158000000000000000486F6D652025732573255D
:1015900073206669727374002066697273740A003E
:1015A0005A0059005800486F6D652000534420636D
:1015B000617264206F6B0A006F70656E526F6F749A
:1015C000206661696C65640A00766F6C756D652EC6
:1015D000696E6974206661696C65640A0053442011
:1015E000696E6974206661696C0A006175746F25A3
:1015F000692E67004D3234004D3233202573005779
:10160000726974696E6720746F2066696C653A2030
:10161000006F70656E206661696C65642C20466998
:101620006C653A20006F70656E206661696C656458
:101630002C2046696C653A200046696C652073650C
:101640006C65637465640A002053697A653A20000A
:1016500046696C65206F70656E65643A20006F7036
:10166000656E206661696C65642C2046696C653A1C
:1016700020002066696C653A20004E6F77200022BA
:1016800020706F73002220706172656E743A2200C0
:10169000535542524F5554494E452043414C4C20DE
:1016A0007461726765743A22004B494C4C45442E74
:1016B0002000747279696E6720746F2063616C6CAE
:1016C000207375622D67636F64652066696C65734E
:1016D000207769746820746F6F206D616E79206C5B
:1016E0006576656C732E204D4158206C6576656C6F
:1016F0002069733A004572726F723A001FFFFFFF54
:10170000FFFFFF600000000001FF4000000000003C
:10171000FF8000000000007F83CF00000C303F8777
:10172000FF80000C301F867980000C000F8C30C7C2
:10173000838C30E78C30CFC7CC31F38C30DCECECD1
:1017400033B98C30D86C6C33198C30D06C0C3319A5
:101750008C30D86C0C33198C30DC6C0E3B198C300F
:10176000CF7C079F198C30C77C038F194000000085
:10177000000002600000000000061FFFFFFFFFFFE7
:10178000F82020506C616E6E6572427566666572F7
:1017900042797465733A20002046726565204D6574
:1017A0006D6F72793A2000436F6D70696C65643AB1
:1017B000204A616E20313120323031380A00207CDD
:1017C00020417574686F723A2028416C65706820FA
:1017D0004F626A6563747320496E632E2C204C75CA
:1017E0006C7A426F7420476974205265706F736918
:1017F000746F7279290A004A616E203131203230CB
:10180000313830383A33383A343200204C6173740E
:1018100020557064617465643A2000312E312E3594
:101820000A004D61726C696E0020536F66747761B7
:1018300072652052657365740A002057617463688D
:10184000646F672052657365740A002042726F7777
:101850006E206F75742052657365740A0020457898
:101860007465726E616C2052657365740A00506F06
:1018700077657255700A0073746172740A0065723C
:10188000726F722077726974696E6720746F206658
:10189000696C650A00456E6473746F70732025630C
:1018A00020256320256320256300205A3A00205913
:1018B0003A0020583A00656E6473746F7073206844
:1018C00069743A2000446F6E6520736176696E67B3
:1018D0002066696C652E0A004D32390020496E760B
:1018E000616C6964206578747275646572200000AB
:1018F0000000C0000000000000000000008F430056
:10190000008A4300007A4347322F473320626164E4
:1019100020706172616D65746572730A005A20707F
:10192000726F6265206F75742E206265640A005ABA
:101930002070726F6265206F75742E20626564007E
:10194000486F6D652058592066697273740A0048A3
:101950006F6D6520585920666972737400456E6416
:101960002066696C65206C6973740A00426567695A
:101970006E2066696C65206C6973740A005344209C
:101980007072696E74696E67206279746520004EAA
:101990006F74205344207072696E74696E670A0018
:1019A0004D36303020486F74656E6420746F6F2040
:1019B000636F6C6420746F206368616E6765206676
:1019C000696C616D656E740A004B494C4C45442E40
:1019D000200045787472756465206D6F72650052E1
:1019E0006573756D65207072696E7400524553554C
:1019F0004D45204F5054494F4E533A0020204E6FD2
:101A00007A7A6C653A20006368616E6765006F667C
:101A1000207468652066696C616D656E740057613D
:101A2000697420666F722073746172740050524939
:101A30004E54205041555345440020204E6F7A7A31
:101A40006C653A2000200066696C616D656E7420DB
:101A5000756E6C6F6164005761697420666F720007
:101A60005052494E54205041555345440020204E79
:101A70006F7A7A6C653A20002000506C656173655E
:101A800020776169742E2E2E0048656174696E6737
:101A9000206E6F7A7A6C65005052494E5420504146
:101AA000555345440020204E6F7A7A6C653A2000E9
:101AB000200068656174206E6F7A7A6C652E005024
:101AC0007265737320627574746F6E20746F00504A
:101AD00052494E54205041555345440020204E6FEA
:101AE0007A7A6C653A2000746F20636F6E74696E49
:101AF00075652E2E2E00616E6420707265737320E2
:101B0000627574746F6E00496E73657274206669D5
:101B10006C616D656E74005052494E5420504155B1
:101B20005345440020204E6F7A7A6C653A2000209D
:101B30000066696C616D656E74206C6F616400573E
:101B400061697420666F72005052494E54205041B2
:101B5000555345440020204E6F7A7A6C653A200038
:101B6000200066696C616D656E74206578747275AD
:101B70006465005761697420666F72005052494E67
:101B8000542050415553454400746F20726573755D
:101B90006D65005761697420666F72207072696E9E
:101BA00074005052494E542050415553454400450D
:101BB00078747275646572202569202573004C75F0
:101BC0006C7A426F742054415A20352072656164EA
:101BD000792E00202F002040002042403A00204073
:101BE0003A004D31343520533C696E6465783E20AF
:101BF0006F7574206F662072616E67652028302DC6
:101C000031290A00205A3A0020593A0020436F75C2
:101C10006E7420583A0020453A00205A3A00205964
:101C20003A00583A004361703A454D455247454E97
:101C300043595F5041525345523A310A0043617053
:101C40003A434153455F4C494748545F42524947E4
:101C500048544E4553533A300A004361703A544F4A
:101C600047474C455F4C49474854533A300A004374
:101C700061703A534F4654574152455F504F574554
:101C8000523A300A004361703A4C4556454C494E31
:101C9000475F444154413A300A004361703A5A5F09
:101CA00050524F42453A300A004361703A41555410
:101CB0004F4C4556454C3A300A004361703A5052F9
:101CC000494E545F4A4F423A310A004361703A50DC
:101CD000524F47524553533A300A004361703A41DC
:101CE00055544F5245504F52545F54454D503A3120
:101CF0000A004361703A454550524F4D3A310A004F
:101D00004649524D574152455F4E414D453A4D610E
:101D1000726C696E20204649524D574152455F56BC
:101D2000455253494F4E3A312E312E352E37302001
:101D300045585452554445525F545950453A466CA3
:101D40006578794475616C6C7920763220534F55F3
:101D50005243455F434F44455F55524C3A68747453
:101D600070733A2F2F636F64652E616C6570686FB6
:101D7000626A656374732E636F6D2F64696666753E
:101D800073696F6E2F4D41524C494E2050524F5443
:101D90004F434F4C5F56455253494F4E3A312E30C8
:101DA000204D414348494E455F545950453A4C7582
:101DB0006C7A426F742054415A2035204558545251
:101DC000554445525F434F554E543A32205555497C
:101DD000443A63333235356339362D343039372D53
:101DE000343838342D386564302D64656432666665
:101DF0003962616536310A004E6F20636173652078
:101E00006C696768740A007C3C3E5E2B3D3F2F5B2B
:101E10005D3B2C2A225C004D6F76652061786973EA
:101E20000044697361626C652073746570706572DB
:101E300073004D3834004175746F20686F6D650014
:101E4000473238004D61696E004D3530320A4D35EC
:101E50003030004C6F61642073657474696E677311
:101E600000526573746F7265206661696C73616698
:101E7000650053746F72652073657474696E67735F
:101E800000416476616E6365642053657474696EA5
:101E90006773004D61696E004D363030204230204E
:101EA0005431004D36303020423020543000466CE2
:101EB0006F77203200466C6F77203200466C6F7768
:101EC000203100466C6F7720310046616E207370C0
:101ED00065656420310046616E207370656564201D
:101EE000310042656400426564004E6F7A7A6C6529
:101EF0002032004E6F7A7A6C652032004E6F7A7A0B
:101F00006C652031004E6F7A7A6C65203100537019
:101F1000656564005370656564004D61696E004DD0
:101F20006F76652058004D6F76652059004D6F76AD
:101F300065205A0045787472756465723200457880
:101F400074727564657231004D6F766520302E3184
:101F50006D6D004D6F766520316D6D004D6F76654E
:101F60002031306D6D004D6F7665206178697300AA
:101F70004578747275646572004D6F7665205A00FD
:101F80004D6F76652059004D6F7665205800457875
:101F90007472756465723200457874727564657226
:101FA000004D6F7665205A004D6F76652059004DC3
:101FB0006F76652058004D6F76656D656E740043D1
:101FC0006F6F6C646F776E0046616E20737065652D
:101FD0006420310046616E207370656564203100B5
:101FE00042656400426564004E6F7A7A6C65203207
:101FF000004E6F7A7A6C652032004E6F7A7A6C658B
:102000002031004E6F7A7A6C652031004D61696E27
:10201000005654726176206D696E00565472617676
:10202000206D696E005654726176206D696E00569F
:102030006D696E00566D696E00566D696E00566D65
:10204000617820453200566D617820453200566D2A
:10205000617820453200566D617820453100566D1B
:10206000617820453100566D617820453100566D0C
:102070006178205A00566D6178205A00566D61785B
:10208000205A00566D6178205900566D61782059AC
:1020900000566D6178205900566D617820580056C1
:1020A0006D6178205800566D61782058004D6F742E
:1020B000696F6E00416D617820453200416D617835
:1020C00020453200416D617820453100416D6178D5
:1020D00020453100416D6178205A00416D617820C2
:1020E0005A00416D6178205900416D617820590096
:1020F000416D6178205800416D6178205800412D74
:1021000074726176656C00412D74726176656C0045
:10211000412D7265747261637400412D7265747231
:1021200061637400416363656C00416363656C00C7
:102130004D6F74696F6E0020746F6F206C6F6E67E7
:1021400020657874727573696F6E2070726576653C
:102150006E7465640A0020636F6C64206578747225
:102160007573696F6E2070726576656E7465640A4A
:102170000056652D6A65726B0056652D6A65726B37
:102180000056652D6A65726B00567A2D6A65726B12
:1021900000567A2D6A65726B0056792D6A65726BEE
:1021A0000056792D6A65726B0056792D6A65726BDF
:1021B0000056782D6A65726B0056782D6A65726BD1
:1021C0000056782D6A65726B004D6F74696F6E00F2
:1021D000453273746570732F6D6D0045327374658D
:1021E00070732F6D6D00453173746570732F6D6D55
:1021F00000453173746570732F6D6D005A7374658B
:1022000070732F6D6D005A73746570732F6D6D0050
:102210005973746570732F6D6D00597374657073A5
:102220002F6D6D005873746570732F6D6D0058734A
:10223000746570732F6D6D004D6F74696F6E004F14
:102240006666004F6E2000456E6473746F70206187
:10225000626F72740053746570732F6D6D004A6500
:10226000726B00416363656C65726174696F6E00C7
:1022700056656C6F6369747900416476616E63655D
:10228000642053657474696E67730043616E6E6F8A
:102290007420656E746572207375626469723A2089
:1022A00000022E2E004D61696E0020204E6F7A7A5A
:1022B0006C653A200020004261636B004D696E69D5
:1022C0006D756D2054656D70206973203132302E2C
:1022D0000048656174696E67206661696C656400B9
:1022E00043616E6E6F74206F70656E2073756264EB
:1022F000697220006563686F3A00544845524D4149
:102300004C2052554E415741592042454400546893
:1023100065726D616C2052756E6177617900544809
:1023200045524D414C2052554E415741592045315F
:1023300000544845524D414C2052554E4157415949
:102340002045300000002200250028002B002E0030
:102350003100340002010000050108010B010000FA
:102360002100240027002A002D0030003300010145
:102370000000040107010A01050505050705080815
:102380000808020202020A0A0808040404040101FF
:102390000101010101010303030303030303040714
:1023A00007070C0C0C0C0C0C0C0C020202020606AB
:1023B0000606060606060B0B0B0B0B0B0B0B01029E
:1023C0001020200808102040102040800201020147
:1023D00008040201010204081020408080402010FF
:1023E0000804020180040201804020100804020158
:1023F00008040201010204081020408001020408C0
:1024000010204080436172642072656D6F76656450
:10241000004361726420696E7365727465640000C4
:10242000060900FE06018902FE20FFFE07FE06FEE9
:10243000000000060007010606060200808080807A
:102440000080030303060103A0A0A0050707060000
:10245000FF5050F850F850500509090600FE207052
:10246000A8A07028A870200608080600FF40A84809
:1024700010204854080507070600FF6090906098F8
:1024800090680103030602038080800207070602AA
:10249000FF408080808080400207070602FF804066
:1024A00040404040800505050600008850F85088EF
:1024B0000505050600002020F8202002040406027D
:1024C000FEC0404080050101060002F8020202063B
:1024D0000200C0C0040606060100101020408080E3
:1024E00004060606010060909090906003060606C0
:1024F000010040C0404040E0040606060100609034
:10250000102040F0040606060100F020601010E0E4
:1025100005060606000010305090F8100406060666
:102520000100F080E01010E0040606060100608063
:10253000E0909060040606060100F0101020404074
:10254000040606060100609060909060040606068E
:102550000100609090701060020505060200C0C086
:1025600000C0C00207070602FEC0C000C040408095
:1025700005050506000018608060180503030600C5
:1025800001F800F8050505060000C0300830C00459
:10259000070706010060901060400040050606062F
:1025A00000007090A8B0807005060606000020505C
:1025B00088F88888050606060000F088F08888F00C
:1025C00004060606010060908080906004060606FE
:1025D0000100E090909090E0040606060100F08073
:1025E000E08080F0040606060100F080E080808034
:1025F000040606060100609080B09060040606069E
:1026000001009090F0909090030606060100E040D3
:10261000404040E0050606060000381010109060AB
:1026200004060606010090A0C0A0909004060606CD
:1026300001008080808080F005060606000088D8B2
:10264000A8A8888804060606010090D0B090909053
:10265000050606060000708888888870040606064D
:102660000100E09090E080800407070601FF609081
:1026700090D0B06010040606060100E09090E09053
:102680009004060606010060904020906005060652
:10269000060000F8202020202004060606010090F5
:1026A0009090909060040606060100909090F06073
:1026B000600506060600008888A8A8D888050606D2
:1026C0000600008850202050880506060600008875
:1026D0008850202020040606060100F010204080CB
:1026E000F0030606060100E080808080E004060614
:1026F000060100808040201010030606060100E05D
:1027000020202020E0050303060003205088050157
:10271000010600FEF80202020602048040040404DE
:10272000060100709090700406060601008080E0AB
:102730009090E00404040601007080807004060696
:1027400006010010107090907004040406010060EF
:10275000B0C070040606060100205040E04040046E
:1027600006060601FE6090907010600406060601E1
:10277000008080E09090900306060601004000C0B3
:102780004040E00308080601FE200060202020A051
:10279000400406060601008080A0C0A09003060643
:1027A000060100C040404040E0050404060000D09F
:1027B000A8A888040404060100E090909004040492
:1027C000060100609090600406060601FEE090900D
:1027D000E080800406060601FE70909070101004E0
:1027E0000404060100A0D0808004040406010070E7
:1027F000C030E00406060601004040E040502004DE
:1028000004040601009090907004040406010090F6
:1028100090606005040406000088A8A85004040421
:10282000060100906060900406060601FE909090FC
:10283000709060040404060100F02040F0030707D4
:10284000060100204040804040200107070602FFAB
:1028500080808080808080030707060100804040E0
:102860002040408004020206010350A0FFFFFFFF4A
:10287000FFFFFFFFFFFFFFFFFFFFFFFFFFFFFFFF68
:10288000FFFFFFFFFFFFFFFFFFFFFFFFFF00000055
:102890000600070106060602008000808080800492
:1028A00006060601FF2070A0A0702005070706009D
:1028B000FF304840F04040F8050505060000A850EC
:1028C0008850A80506060600008850F820F8200168
:1028D00007070602FF8080800080808004070706CB
:1028E00001FF708060906010E0030101060105A007
:1028F000060707060000788494A4948478030505ED
:1029000006010160A06000E00505050600002850F2
:10291000A05028040303060100F010100401010672
:102920000102F00607070600007884B4A4A48478A6
:10293000040101060105F004030306010260906032
:102940000507070600FF2020F8202000F8030505F2
:1029500006010140A02040E0030505060101C0205A
:102960004020C00202020602044080040505060160
:10297000FF9090B0D08005060606000078E8E86871
:102980002828010101060202800202020602FE401E
:102990008003050506010140C04040E0030505062F
:1029A000010140A04000E0050505060000A05028F8
:1029B00050A00508080600FF40C040507030781055
:1029C0000508080600FF40C0405068081038050898
:1029D000080600FFC0204030F030781004070706DA
:1029E000010020002060809060050707060000407D
:1029F000202050708888050707060000102020500E
:102A000070888805070706000020502050708888CD
:102A10000507070600002850205070888805070722
:102A20000600005000205070888805070706000047
:102A30002050205070888805060606000078A0F017
:102A4000A0A0B80408080601FE6090808090602075
:102A5000400407070601004020F080E080F00407F2
:102A6000070601002040F080E080F004070706011F
:102A7000002050F080E080F00407070601005000BD
:102A8000F080E080F00307070601008040E040404E
:102A900040E00307070601002040E0404040E0031B
:102AA000070706010040A0E0404040E0030707069A
:102AB0000100A000E0404040E0050606060000706E
:102AC00048E848487004070706010050A090D0B0BD
:102AD00090900407070601004020609090906004E9
:102AE00007070601002040609090906004070706E9
:102AF000010020506090909060040707060100508C
:102B0000A06090909060040707060100500060905C
:102B10009090600505050600008850205088040844
:102B2000080601FF1070B0B0D0D0E080040707069F
:102B3000010040209090909060040707060100205B
:102B400040909090906004070706010020509090FC
:102B500090906004070706010050009090909060EC
:102B600005070706000010208850202020040606D4
:102B700006010080E09090E08004060606010060F7
:102B800090A0A090A00407070601004020007090CC
:102B900090700407070601002040007090907004B8
:102BA0000707060100205000709090700407070688
:102BB000010050A0007090907004060606010050BD
:102BC000007090907004070706010020502070905C
:102BD000907005040406000070A8B078040606068C
:102BE00001FE70808070204004070706010040202D
:102BF0000060B0C07004070706010020400060B00C
:102C0000C07004070706010020500060B0C07004C7
:102C10000606060100500060B0C0700307070601F9
:102C200000804000C04040E003070706010020404C
:102C300000C04040E003070706010040A000C0407C
:102C400040E0030606060100A000C04040E0040783
:102C500007060100306010709090600407070601BD
:102C60000050A000E090909004070706010040206B
:102C7000006090906004070706010020400060900B
:102C800090600407070601002050006090906004E7
:102C9000070706010050A000609090600406060639
:102CA00001005000609090600505050600002000BE
:102CB000F8002004040406010070B0D0E004070707
:102CC0000601004020009090907004070706010064
:102CD00020400090909070040707060100205000EB
:102CE000909090700406060601005000909090703D
:102CF0000409090601FE2040009090907090600445
:102D000008080601FE8080E09090E08080040808BA
:102D10000601FE50009090907090601000C9021063
:102D2000012C014001220170011801B0010E01F0D7
:102D30000104015002FA00B002F0003003E600D0B6
:102D400003DC009004D2007005C800A006BE00009D
:102D500008B400B009AA00D00BA000600E96006075
:102D6000118C000015820020197800C01D6E00A093
:102D7000226400B0275A00902C500000314600E039
:102D8000343C0010383200903A2800603C1E00A00D
:102D90003D1400803E0A00203F00006265640A0086
:102DA0002C2073797374656D2073746F7070656413
:102DB00021204865617465725F49443A2000486586
:102DC0006174696E67206661696C65642042454480
:102DD0000048656174696E67206661696C656400AE
:102DE00048656174696E67206661696C6564004856
:102DF000656174696E67206661696C656420453140
:102E00000048656174696E67206661696C6564205D
:102E10004530001000AD0330016A0150022B0170F3
:102E2000030A019004F500B005E500D006D800F0D3
:102E300007CE001009C500300ABE00500BB7007065
:102E40000CB100900DAB00B00EA600D00FA200F0A8
:102E5000109D0010129900301395005014920070CC
:102E6000158E0090168B00B0178700D0188400F0E4
:102E7000198100101B7E00301C7B00501D790070F2
:102E80001E7600901F7300B0207000D0216E00F0FD
:102E9000226B001024690030256600502663007004
:102EA00027610090285E00B0295C00D02A5900F00C
:102EB0002B5600102D5400302E5100502F4E007014
:102EC000304B0090314800B0324500D0334200F022
:102ED000343E0010363B0030373700503833007036
:102EE000392E00903A2900B03B2300D03C1B00F063
:102EF0003D1100103F0100F03F00004572723A2082
:102F00004D494E54454D5020424544004D494E5484
:102F1000454D50207472696767657265640045723B
:102F2000723A204D494E54454D502045310045726E
:102F3000723A204D494E54454D502045300045725F
:102F4000723A204D415854454D5020424544004D61
:102F5000415854454D5020747269676765726564C5
:102F6000004572723A204D415854454D502045312C
:102F7000004572723A204D415854454D502045301D
:102F8000004572726F722077726974696E6720747F
:102F90006F20454550524F4D210A00290A002062FA
:102FA000797465733B2063726320005365747469A0
:102FB0006E67732053746F72656420280020286345
:102FC000616C63756C6174656429210A0020213D80
:102FD0002000454550524F4D20435243206D6973A8
:102FE0006D61746368202D202873746F7265642985
:102FF0002000290A002062797465733B20637263A4
:1030000020002073746F7265642073657474696E38
:103010006773207265747269657665642028002084
:103020004D61726C696E3D563430290A0028454561
:1030300050524F4D3D00454550524F4D20766572E0
:1030400073696F6E206D69736D617463682000240D
:10305000F4D43050C38E20C2A24017828B7011125C
:103060007A910D816CD90AA861E108C75866076199
:103070005143061E4B5D05C145A7041A41110409C1
:103080003D9803713931034036DB0265339102D438
:10309000305402802E1D02632CEE01752AC501B04A
:1030A00028A001102781018F2564012B244B01E00A
:1030B000223401AC211F018D200D01801FFC0084F2
:1030C0001EED00971DDF00B81CD200E61BC60020D5
:1030D0001BBC00641AB200B219A8000A19A0006A49
:1030E000189900D117910040178B00B51684003154
:1030F000167E00B31579003A157300C7146F005897
:10310000146A00EE1366008813630025135E00C77F
:10311000125B006C12570015125400C1115100705F
:10312000114F0021114B00D61049008D1047004669
:1031300010440002104200C00F4000800F3E0042C9
:103140000F3C00060F3B00CB0E3800930E37005C9F
:103150000E3500270E3400F30D3200C10D31009002
:103160000D3000600D2E00320D2D00050D2C00D904
:103170000C2B00AE0C2900850C29005C0C270035B7
:103180000C27000E0C2600E80B2400C40B2400A022
:103190000B23007D0B23005A0B2100390B21001853
:1031A0000B2000F80A1F00D90A1E00BB0A1E009D52
:1031B0000A1D00800A1D00630A1C00470A1B002C20
:1031C0000A1B00110A1A00F7091A00DD091900C4C8
:1031D000091900AB091900920917007B091800634F
:1031E0000917004C09160036091600200916000AB6
:1031F000091500F5081500E0081400CC081400B803
:10320000081400A4081400900813007D0812006B35
:103210000813005808120046081200340811002351
:103220000811001208110001081100F0071000E059
:10323000071000D0071000C0071000B0070F00A152
:1032400007100091070E0083070F0074070F006539
:10325000070E0057070E0049070E003B070D002E12
:10326000070E0020070D0013070D0006070D00F9DB
:10327000060C00ED060D00E0060C00D4060C00C89C
:10328000060C00BC060C00B0060C00A4060B00994E
:10329000060C008D060B0082060B0077060B006CF7
:1032A000060B0061060A0057060B004C060A004296
:1032B000060A0038060A002E060A0024060A001A2A
:1032C000060A001006090007060A00FD050900F4B9
:1032D000050900EB050900E2050900D9050900D040
:1032E000050900C7050900BE050900B5050800ADC0
:1032F000050800A50509009C050800940508008C38
:10330000050800840508007C050800740508006CA9
:10331000050700650508005D050700560508004E15
:10332000050700470507004005080038050700317C
:103330000507002A050700230507001C05060016DF
:103340000507000F0507000805060002050700FB3A
:10335000040600F5040700EE040600E8040600E297
:10336000040700DB040600D5040600CF040600C9EC
:10337000040600C3040600BD040600B7040600B13D
:10338000040500AC040600A6040600A00405009B8A
:1033900004060095040500900406008A04050085D3
:1033A000040500800406007A040500750405007019
:1033B0000405006B04050066040500610405005C5B
:1033C00004050057040500520405004D040500489B
:1033D000040500430405003E0404003A04050035DA
:1033E000040500300404002C040500270404002315
:1033F0000405001E0404001A04040016040500114C
:103400000404000D04040009040500040404000081
:10341000040400FC030400F8030400F4030400F0B7
:10342000030400EC030400E8030400E4030400E0E8
:10343000030400DC030400D8030400D4030400D018
:10344000030400CC030400C8030300C503030024E5
:10345000F404D9201BC40C5C0E9804C4095F0265F7
:10346000077101F405F900FB04B30048048700C1AB
:103470000369005803550003034500BE023A008467
:1034800002310053022A002902250004022000E430
:10349000011C00C8011900AF011700980114008435
:1034A000011300710110006101100051010E004371
:1034B000010D0036010B002B010B0020010B001544
:1034C0000109000C01090003010800FB000800F3DA
:1034D000000800EB000700E4000600DE000600D84C
:1034E000000600D2000600CC000500C7000500C29F
:1034F000000500BD000400B9000400B5000400B1DF
:10350000000400AD000400A9000400A5000300A20F
:103510000003009F0004009B000300980003009537
:1035200000020093000300900003008D0002008B56
:10353000000300880002008600020084000300816E
:103540000002007F0002007D0002007B0002007983
:103550000002007700010076000200740002007291
:10356000000100710002006F0002006D0001006C9C
:103570000002006A000100690002006700010066A5
:1035800000010065000100640002006200010061AA
:10359000000100600001005F0002005D0001005CAE
:1035A0000001005B0001005A0001005900010058B1
:1035B00000010057000100560001005500010054B1
:1035C00000010053000000530001005200010051AF
:1035D000000100500001004F0001004E0000004EAD
:1035E0000001004D0001004C0001004B0000004BA9
:1035F0000001004A000100490001004800000048A5
:10360000000100470001004600000046000100459F
:103610000000004500010044000100430000004399
:103620000001004200000042000100410000004192
:10363000000100400001003F0000003F0001003E8B
:103640000000003E0001003D0000003D0001003C84
:103650000000003C0000003C0001003B0000003B7B
:103660000001003A0000003A000100390000003972
:103670000001003800000038000000380001003769
:103680000000003700010036000000360000003660
:103690000001003500000035000000350001003455
:1036A000000000340000003400010033000000334B
:1036B0000000003300010032000000320000003240
:1036C0000001003100000031000000310001003035
:1036D00000000030000000300001002F0000002F2B
:1036E0000000002F0000002F0001002E0000002E1F
:1036F0000000002E0001002D0000002D0000002D14
:103700000000002D0001002C0000002C0000002C07
:103710000000002C0001002B0000002B0000002BFB
:103720000000002B0001002A0000002A0000002AEF
:103730000000002A000100290000002900000029E3
:1037400000000029000000290001002800000028D6
:1037500000000028000000280000002800010027C9
:1037600000000027000000270000002700000027BD
:1037700000010026000000260000002600000026B0
:1037800000000026000100250000002500000025A3
:103790000000002500000025000000250001002495
:1037A0000000002400000024000000240000002489
:1037B000000100230000002300000023000000237C
:1037C000000000230000002300000023000100226D
:1037D0000000002200000022000000220000002261
:1037E0000000002200010021000000210000002153
:1037F0000000002100000021000000210000002145
:103800000001002000000020000000200000002037
:103810000000002000000020000000200000002028
:103820000001001F0000001F0000001F0000001F1B
:103830000000001F0000001F0000001F0001001E0C
:103840000000001E0000001E0000001E0000004DD1
:10385000383420582059205A204500526573656E2F
:10386000643A20002042002050006F6B004B494C0E
:103870004C45442E20004B494C4C206361757365C8
:1038800064206279204B494C4C20627574746F6ED1
:103890002F70696E0A004B494C4C45442E20004B5A
:1038A000494C4C2063617573656420627920746FA4
:1038B0006F206D75636820696E6163746976652039
:1038C00074696D65202D2063757272656E74206356
:1038D0006F6D6D616E643A2000506C656173652098
:1038E0007265736574005052494E544552204841E8
:1038F0004C544544005072696E7465722068616C66
:103900007465642E206B696C6C28292063616C6C73
:103910006564210A00656E7175657565696E67205D
:103920002200000000C000000000000000000000B5
:10393000484200004842000040400000000057613B
:10394000726E696E673A20486F6D696E67204275C6
:103950006D702044697669736F72203C20310A00D3
:103960000202040000A0400000A04000000040004F
:1039700000904300008A4300007A43FFFFFF416349
:10398000746976652045787472756465723A2000B2
:103990000201050800FF060121023520FFFF07FF95
:1039A00006FF090050221656808080800080153363
:1039B00053A0A0A00257575050F850F8505002574B
:1039C000572070A07028702013355580A040A0208B
:1039D00002475740A0A040A0A050251353808080EC
:1039E00012265640808080804012265680404040FB
:1039F00040800245559060F060900255552020F8B7
:103A00002020113353604080044151F01133534062
:103A1000E04002465610102040808012365640A0EA
:103A2000A0A0A04012365640C0404040E00246569A
:103A30006090106080F0024656F0206010906002A6
:103A400046562060A0F02020024656F080E01090FC
:103A5000600246566080E0909060024656F010206A
:103A6000204040024656609060909060024656604A
:103A70009090701060122555C0C000C0C01136561D
:103A800060600060408012365620408080402003F5
:103A90004353F000F012365680402020408012360A
:103AA0005640A020400040015858304898A8A8909F
:103AB0004030024656609090F09090024656E0905A
:103AC000E09090E0024656609080809060024656FA
:103AD000E090909090E0024656F080E08080F00206
:103AE0004656F080E0808080024656609080B0901C
:103AF000600246569090F0909090123656E040400A
:103B00004040E002465670202020A04002465690D9
:103B1000A0C0A0A0900246568080808080F002461F
:103B20005690F0F090909002465690D0F0B0B09041
:103B3000024656609090909060024656E09090E069
:103B40008080014757609090D0B06010024656E0E8
:103B50009090E0909002465660904020906012361F
:103B600056E0404040404002465690909090906011
:103B7000024656909090906060024656909090F069
:103B8000F090024656909060609090025656888859
:103B900050202020024656F010204080F012365669
:103BA000E080808080E00246568080402010101225
:103BB0003656E020202020E016325240A00141512C
:103BC000F016225280400244547090907002465683
:103BD0008080E09090E0123454608080600246560D
:103BE00010107090907002445460B0C0600246564D
:103BF000205040E040400145556090701060024602
:103C0000568080E09090901236564000C04040E0D0
:103C10001137572000202020A04002465680809077
:103C2000E09090123656C040404040E0025454D0DC
:103C3000A8A8A8024454E090909002445460909048
:103C400060014555E090E08080014555709070100E
:103C500010024454A0D0808012345460C020C002AE
:103C600046564040E04050200244549090907012DC
:103C70003454A0A0A04002545488A8A85002445430
:103C8000906060900145559090709060024454F0AF
:103C90002040F0024757304020C0204030221656C6
:103CA000808080808080024757C02040304020C004
:103CB00006425250A0FFFFFFFFFFFFFFFFFFFFFF85
:103CC000FFFFFFFFFFFFFFFFFFFFFFFFFFFFFFFF04
:103CD000FFFFFFFFFFFF0900502216568000808083
:103CE00080800146562070A0A070200246562050C9
:103CF000E04050A002555588705070880256568892
:103D000050F820F8202217578080800080808002A1
:103D100047577080E0907010E0173151A00256565E
:103D200070A8C8C8A87014355560A06000E00343AF
:103D30005350A050123353E02020143151E002566A
:103D40005670E8D8E8D870173151E015335340A0C9
:103D50004012355540E04000E014355540A0204069
:103D6000E0143555C020C020C016225240800145C5
:103D700055909090E08002565678E8E8682828240C
:103D8000115180112252408014355540C04040E00E
:103D900014355540A04000E0034353A050A0024713
:103DA00057808080A060F0200247578080A0D0100C
:103DB000207002475780408060A0F02012365640A5
:103DC000004080A04002475740206090F090900251
:103DD000475720406090F090900247576090609065
:103DE000F0909002475750A06090F0909002475793
:103DF00090006090F0909002475760906090F09033
:103E00009002465670A0A0F0A0B001475760908085
:103E1000809060400247574020F080E080F00247E9
:103E2000572040F080E080F00247576090F080E03B
:103E300080F00247579000F080E080F01237578002
:103E400040E0404040E01237572040E0404040E032
:103E500012375740A0E0404040E0123757A000E042
:103E6000404040E00256567048E8484870024757C4
:103E700050A090D0B0909002475740206090909012
:103E800060024757204060909090600247576090D2
:103E9000609090906002475750A0609090906002B0
:103EA000475790006090909060123353A040A0025A
:103EB000465670B0B0D0D0E0024757402090909066
:103EC0009060024757204090909090600247576062
:103ED00090909090906002475790009090909060E2
:103EE0000257571020885020202002465680E0902C
:103EF00090E0800246566090A0A090A002475740F4
:103F00002000709090700247572040007090907091
:103F10000247572050007090907002475750A00001
:103F20007090907002465650007090907002475703
:103F300060906070909070025454F068B0781135C1
:103F400055608080604002475740200060B0C060EC
:103F500002475720400060B0C060024757609000A1
:103F600060B0C060024656500060B0C06012375763
:103F7000804000C04040E0123757204000C0404021
:103F8000E012375740A000C04040E0123656A00073
:103F9000C04040E0024757A040A010709060024728
:103FA0005750A000E090909002475740200060904A
:103FB0009060024757204000609090600247576031
:103FC00090006090906002475750A0006090906011
:103FD0000246569000609090601235554000E00017
:103FE0004002445470B0D0E0024757402000909007
:103FF00090700247572040009090907002475760A1
:1040000090009090907002465690009090907001B1
:10401000485820400090907090600147578080E0A1
:1040200090E080800147579000909070906001056B
:104030000700FE0500FB01F220FFFE05FE05FE0263
:1040400000400215258080800080053242A0A00239
:10405000556550F850F8500146562070C030E020A9
:104060000255659010204048025565608068906850
:10407000051222808002253540808080400225354F
:104080008040404080043343A040A003334340E0DD
:10409000400122324080043141E00211218002556A
:1040A0006508102040800245556090909060022580
:1040B00035C040404040024555E0106080F0024568
:1040C00055E0106010E00245552060A0F020024548
:1040D00055F080E010E00245556080E090600245B8
:1040E00055F01020404002455560906090600245B8
:1040F00055609070106003132380008002142480A8
:104100000080800235452040804020033343E0009A
:10411000E00235458040204080024555E0106000B7
:10412000400255657088B8A870024555609090F0BF
:1041300090024555E090E090E00235456080808037
:1041400060024555E0909090E0023545E080E080C7
:10415000E0023545E080E080800245557080B090F7
:10416000700245559090F09090023545E0404040F7
:10417000E0024555301010906002455590A0C0A057
:104180009002354580808080E002556588D8A888F7
:104190008802455590D0B09090024555609090901F
:1041A00060024555E09090E0800146566090909006
:1041B0006010024555E09090E09002455570806097
:1041C00010E0023545E04040404002455590909057
:1041D00090600245559090A0A04002556588A8A81F
:1041E000A85002455590906090900245559090706F
:1041F0001060023545E0204080E0022535C0808017
:1042000080C00255658040201008022535C040401E
:1042100040C005324240A0024151F00522328040A8
:104220000244547090907002455580E09090E002F6
:104230003444608080600245551070909070024454
:104240005460B0C0600235452040E0404000465612
:1042500070909070106002455580E090909002152B
:10426000258000808080002737400040404040800B
:104270000245558090A0E0900215258080808080C6
:10428000025464F0A8A8A8024454E090909002441C
:104290005460909060004656E09090E08080004628
:1042A00056709090701010023444A0C08080024478
:1042B0005470C030E002354540E040402002445494
:1042C000909090700244549090A040025464A8A82A
:1042D0005050023444A04040A00046569090907048
:1042E0001060024454F02040F002354560408040A8
:1042F000600215258080808080023545C0402040C6
:10430000C005425250A0FFFFFFFFFFFFFFFFFFFF6E
:10431000FFFFFFFFFFFFFFFFFFFFFFFFFFFFFFFFAD
:10432000FFFFFFFFFFFFFF020040FFFFFFFFFFFF58
:10433000FFFFFFFFFFFFFFFFFFFFFFFFFFFFFFFF8D
:10434000FFFFFFFFFFFFFFFFFFFFFFFFFFFFFFFF7D
:10435000FFFFFFFFFFFFFFFFFFFFFFFFFFFFFFFF6D
:10436000FFFFFFFFFFFFFFFFFFFFFFFFFFFFFFFF5D
:10437000FFFFFFFFFFFFFFFFFFFFFFFFFFFFFFFF4D
:10438000FFFFFFFFFFFFFFFFFF01060D00FE09011A
:104390006602D620FFFE0BFE0AFE0D0060221969A0
:1043A000808080808080800080183363A0A0A0037C
:1043B00057675050F850F850500259692078A0A023
:1043C000702828F02002596948A85010204050A8B1
:1043D0009002586840A0A040A0989068281363807D
:1043E0008080113B6B204040808080808040402056
:1043F000113B6B804040202020202040408006550B
:104400006520A870A8200455652020F820201133CD
:1044100063604080065161F811336340E040025907
:104420006908081010204040808002596920508897
:104430008888888850200259692060A02020202088
:1044400020F80259697088880810204080F80259C5
:1044500069F8081020700808887002596910103037
:10446000505090F81010025969F88080B0C80808C0
:10447000887002596970888080F088888870025935
:1044800069F808101020204040400259697088885F
:1044900088708888887002596970888888780808C8
:1044A000887011386840E040000040E040113868F2
:1044B00040E04000006040800259690810204080C0
:1044C00040201008045464F80000F8025969804044
:1044D0002010081020408002596970888808102038
:1044E00020002002596970888898A8A8B0807802B6
:1044F00059692050888888F8888888025969F04866
:10450000484870484848F002596970888080808027
:10451000808870025969F048484848484848F00285
:104520005969F8808080F0808080F8025969F880AD
:104530008080F080808080025969708880808098B7
:1045400088887002596988888888F88888888812DD
:104550003969E040404040404040E002596938102D
:1045600010101010109060025969888890A0C0A0A7
:104570009088880259698080808080808080F802DD
:1045800059698888D8A8A88888888802596988C8FD
:10459000C8A8A898988888025969708888888888E7
:1045A000888870025969F0888888F080808080014E
:1045B0005A6A70888888888888A87008025969F0C3
:1045C000888888F0A09088880259697088808070F7
:1045D00008088870025969F8202020202020202017
:1045E000025969888888888888888870025969880B
:1045F000888888505050202002596988888888A867
:10460000A8A8A8500259698888505020505088881E
:10461000025969888850502020202020025969F8CA
:1046200008101020404080F8113B6BE080808080B3
:104630008080808080E00259698080404020101096
:104640000808113B6BE0202020202020202020E0C3
:10465000085363205088015161F82A226280400289
:104660005666700878889868025969808080F0885A
:10467000888888F002566670888080887002596940
:104680000808087888888888780256667088F880D4
:10469000887002596930484040F04040404000581E
:1046A000687088888878088870025969808080B02E
:1046B000C8888888881238684000C040404040E080
:1046C000004A6A1000301010101090906002596972
:1046D00080808090A0C0A09088123969C04040407E
:1046E00040404040E0025666D0A8A8A8A8880256DC
:1046F00066B0C888888888025666708888888870FE
:10470000005868F0888888F0808080005868788831
:10471000888878080808025666B0C88080808002C1
:1047200056667088601088700258684040F04040BB
:10473000404830025666888888889868025666889D
:1047400088885050200256668888A8A8A85002562B
:1047500066885020205088005868888888986808A3
:104760008870025666F810204080F8015B6B1820B4
:10477000202020C0202020201822196980808080DD
:104780008080808080015B6BC0202020201820204A
:104790002020C008536348A890FFFFFFFFFFFFFFE2
:1047A000FFFFFFFFFFFFFFFFFFFFFFFFFFFFFFFF19
:1047B000FFFFFFFFFFFFFFFFFFFF0D0060221969F2
:1047C0008000808080808080800358682070A8A04E
:1047D000A0A8702002596930484040E0404048B0ED
:1047E0000356668870505070880259698888505006
:1047F000F820F82020221969808080800080808045
:1048000080124A6A609080609090601090601A32C6
:1048100062A0A00359697088A8D8C8D8A888700475
:104820005767700878887800F80356662850A0A06B
:104830005028045363F80808163161E00359697081
:1048400088E8D8D8E8D888700A5161F817446460BD
:104850009090600357672020F8202000F807356506
:1048600040A02040E007356540A04020C02A2262D9
:1048700040800058688888888898E8808002596954
:1048800078E8E8E8E868282828262161C020226224
:10489000408007356540C04040E004576770888815
:1048A000887000F8035666A050282850A0025A6A63
:1048B00040C04040E00818283808025A6A40C0400A
:1048C00040E01028081038025A6A40A04020A04852
:1048D00018283808025969200020204080888870F4
:1048E000025A6A40200020508888F88888025A6A54
:1048F00010200020508888F88888025A6A304800C2
:1049000020508888F88888025A6A285000205088E9
:1049100088F88888025A6A50500020508888F888A1
:1049200088025A6A20502020508888F888880259C6
:104930006958A0A0A0B0E0A0A0B8005B6B70888010
:104940008080808088702040025A6A402000F88071
:1049500080F08080F8025A6A102000F88080F08091
:1049600080F8025A6A304800F88080F08080F802AF
:104970005A6A505000F88080F08080F8123A6A80BD
:104980004000E04040404040E0123A6A204000E0F1
:104990004040404040E0124A6A609000E0404040A1
:1049A0004040E0123A6AA0A000E04040404040E0B1
:1049B000025969F0484848E8484848F0025A6A28CD
:1049C00050008888C8A8988888025A6A40200070D9
:1049D000888888888870025A6A10200070888888C1
:1049E000888870025A6A3048007088888888887081
:1049F000025A6A28500070888888888870025A6A2B
:104A000050500070888888888870035565885020C9
:104A10005088015B6B08709898A8A8A8C8C87080D7
:104A2000025A6A40200088888888888870025A6AFA
:104A300010200088888888888870025A6A30480068
:104A400088888888888870025A6A505000888888C8
:104A500088888870025A6A10200088885020202098
:104A60002002596980F0888888F080808002596926
:104A7000609090A0A0908888B00259694020007092
:104A8000087888986802596910200070087888981A
:104A90006802596930480070087888986802596936
:104AA0002850007008788898680259695050007042
:104AB0000878889868025A6A304830007008788808
:104AC0009868025666702870A0A8500058687088D0
:104AD0008080887020400259694020007088F880EA
:104AE00088700259691020007088F8808870025917
:104AF000693048007088F880887002596950500009
:104B00007088F8808870123969804000C040404049
:104B100040E0123969204000C040404040E0124966
:104B200069609000C040404040E0123969A0A00098
:104B3000C040404040E0025A6A50206010708888AF
:104B4000888870025969285000B0C888888888020F
:104B5000596940200070888888887002596910203F
:104B60000070888888887002596930480070888889
:104B70008888700259692850007088888888700277
:104B800059695050007088888888700357672020C2
:104B900000F8002020015868087098A8A8C8708004
:104BA00002596940200088888888986802596910ED
:104BB0002000888888889868025969304800888869
:104BC0008888986802596950500088888888986851
:104BD000005B6B1020008888889868088870005AED
:104BE0006A8080B0C88888C8B08080005B6B5050F5
:104BF000008888889868088870000000000000001D
:104C000000000000000000000000000000000000A4
:104C10000000000000000000000000000C00000088
:104C2000000000000C000000000000001200000066
:104C30000000000023000000000000002100000030
:104C4000000000004C800000000000005E800000BA
:104C5000000000009240000000000000A1400000A1
:104C60000000000121200000000000027F900000F1
:104C7000000000020010000000000007FFF8000024
:104C8000000000040008000000000008000400000C
:104C900000000008000600000000001000020000F4
:104CA000000000301E010000000000207F81000095
:104CB00000000041FFE0800000000043FCF08000A5
:104CC000000000873B7840000000018EDBFC6000A4
:104CD0000000010FEBCC20000000021FEDB6100019
:104CE0000000021FDEB6100000000439CD7F08006E
:104CF00000000436E0FF08000000087EC0BB84000E
:104D00000000187F005D86000000107FC0ED82006B
:104D10000000203CC07301000000203B337F0100F5
:104D20000000701BE77E03800000C81DEEDE04C09B
:104D30000000880FDEDC04400001240FDF3C092066
:104D400000012607DBF8192000027203E7F0139038
:104D500000025101FFE02290000489007F80244876
:104D6000000904801E004824000BFE400000DFF410
:104D70000010004000008002001FFFFFFFFFFFFE49
:104D80000000000000000000000000000000000023
:104D90000000000000000000001022103C3C0E1F2C
:104DA0000010221004221104001022100822110405
:104DB00000102210083C11040010221010221104CF
:104DC0000010221020221104001E1C1E3C3C0E0468
:104DD00000000000000000000000000000000000D3
:104DE00000000000000000000000000000000000C3
:104DF00000000000000000000000000000000000B3
:104E000000000000000000000000000000000000A2
:104E10000000000000000000000000000000000092
:104E20000000000000000000000000000000000082
:104E30000000000000000048617264636F646564F4
:104E40002044656661756C742053657474696E677F
:104E500073204C6F616465640A00282300002823D6
:104E600000006400000010270000000096430000CE
:104E70009643000040400000C8410000C9420000C5
:104E8000C9420000C84400804F4400804F44204481
:104E90000020490020204D333034205000204400B1
:104EA00020490020204D3330312050002044002084
:104EB000490020500020204D33303120450050491A
:104EC000442073657474696E67733A0A0020460063
:104ED00020420020480020204D3134352053004D21
:104EE0006174657269616C206865617475702070A9
:104EF0006172616D65746572733A0A002059002011
:104F0000580020204D323138205400486F74656EAF
:104F100064206F6666736574733A0A00205A002035
:104F2000590020204D323036205800486F6D6520E2
:104F30006F66667365743A0A00204500205A0020A7
:104F4000590020580020420020540020204D3230CB
:104F500035205300416476616E6365643A20533CAA
:104F60006D696E5F66656564726174653E20543C70
:104F70006D696E5F74726176656C5F66656564729B
:104F80006174653E20423C6D696E5F7365676D6557
:104F90006E745F74696D655F6D733E20583C6D6122
:104FA000785F78795F6A65726B3E205A3C6D6178F4
:104FB0005F7A5F6A65726B3E20453C6D61785F6524
:104FC0005F6A65726B3E0A00205400205200202068
:104FD0004D323034205000416363656C65726174FA
:104FE000696F6E2028756E6974732F7332293A20A9
:104FF000503C7072696E745F616363656C3E2052F1
:105000003C726574726163745F616363656C3E20BA
:10501000543C74726176656C5F616363656C3E0AD3
:105020000020450020204D323031205400205A000D
:1050300020590020204D3230312058004D617869D0
:105040006D756D20416363656C65726174696F6E27
:105050002028756E6974732F7332293A0A0020452F
:105060000020204D323033205400205A00205900B7
:1050700020204D3230332058004D6178696D756DB8
:10508000206665656472617465732028756E697445
:10509000732F73293A0A0020450020204D39322011
:1050A0005400205A0020590020204D393220580049
:1050B00053746570732070657220756E69743A0A56
:1050C0000020204D3230302044300A0020204D3264
:1050D000303020543120440020204D3230302044E4
:1050E000002044697361626C65640A0046696C6102
:1050F0006D656E742073657474696E67733A002011
:10510000204D3134392043203B20556E6974732083
:10511000696E2043656C736975730A0020204732FD
:1051200031202020203B20556E69747320696E2049
:105130006D6D0A0045313A200045303A20005A3A58
:105140002000593A2000583A20004D53312C4D533D
:10515000322050696E730A005072696E742070615B
:1051600075736564004D31323500004D32340050A6
:1051700072696E742061626F72746564004E6F2094
:1051800053442063617264005072696E74206672C9
:105190006F6D2053440053746F70207072696E7489
:1051A00000526573756D65207072696E7400506190
:1051B000757365207072696E74004368616E67650F
:1051C0002066696C616D656E742045320041626FC6
:1051D0007574204669726D77617265004368616E0F
:1051E00067652066696C616D656E742045310043AA
:1051F0006F6E66696775726174696F6E0054656D74
:105200007065726174757265004D6F76656D656E5F
:10521000740054756E6500496E666F207363726525
:10522000656E0000A6BA3FE811241FBECFEFD1E2A1
:10523000DEBFCDBF00E00CBF14E0A0E0B2E0E2E6CC
:10524000F1E102E00BBF02C007900D92AE30B10752
:10525000D9F725E1AEE0B4E001C01D92A136B20756
:10526000E1F719E2C3E1D9E200E006C021970109A4
:10527000802FFE010F942D08C231D10780E008076E
:10528000A9F70E9484600D94A0080C9400002F924E
:105290003F924F925F926F927F928F929F92AF92C6
:1052A000BF92CF92DF92EF92FF920F931F93CF9313
:1052B000DF93CDB7DEB7C259D1090FB6F894DEBF80
:1052C0000FBECDBF0091180920E6029F8001112476
:1052D0000856184F8091070A80FF1AC0E4EFF2E2E7
:1052E00084917F013FEFE31AF30A811102C0780134
:1052F00004C00E944B72F701F3CFD7018D917D015D
:10530000882319F00E944B72F8CF8AE00E944B72FA
:1053100010922D0410922C048FE38093420410927B
:105320004104109240041092280410922904109213
:105330002A0410922B04F80180810F5F1F4F8032E6
:10534000D1F38E34B1F4818190ED980F9A3020F032
:105350008D3211F08B3269F43296DF0131962C9147
:1053600020532A30D0F3CD01FC0101962081203258
:10537000D9F3F093E113E093E0137F01BFEFEB1A51
:10538000FB0A10816AE270E0C7010F947108009770
:1053900031F0FC01319780818032E1F311821D34BC
:1053A00029F0143519F0173409F0C9C0F7018081CC
:1053B0002FEFE21AF20A8032C9F380538A3008F0E4
:1053C000BEC01093420420914004309141044AE051
:1053D0003196429FC001439F900D1124DF01119728
:1053E0002C9130E020533109280F391F80818053E0
:1053F0008A3070F33093410420934004DF013196EA
:105400008C918032D9F31D34D1F42E31310591F0D5
:105410003CF42731310571F02C31310581F40AC09B
:105420002537310564F02737310524F0203A43E071
:10543000340729F4B0932D04A0932C0480C010925B
:105440002D0410922C040091E01361E070E0FD0146
:1054500031968C91882309F472C08132A1F41D34F5
:1054600091F42032310579F4F0932D04E0932C046B
:1054700063E270E0CF010F947108009709F45FC0F8
:10548000DC011C925CC09FEBD92ED80E49E1C42EE2
:10549000CD14C0F1AF01FA0190814F5F5F4F9032A0
:1054A000D1F340ED490F4A3040F043ED490F42300F
:1054B00020F09B3211F00C94133FAF01AD2CB12CB6
:1054C0007501A3E0F594E794AA95E1F7C701885D1B
:1054D0009B4F7C018D2D8770DB0102C0AA0FBB1F83
:1054E0008A95E2F7CD01D7019C91892B8C934115C8
:1054F000510511F0401B01C040E0D501A25FBB4F38
:105500004C930AC080912C0490912D04892B21F496
:10551000B0932D04A0932C04808181548A3110F41F
:10552000DF0195CFDF0131969C9190539A30D0F3F3
:10553000CD01FC01019640814032D9F3F1CF809139
:1055400042048D3409F409C2843511F40C94CD3E23
:10555000873411F00C94F63E2091400430914104C0
:105560002A31310509F45EC18CF42430310544F44C
:10557000223031050CF006C137FF28C00C94103FD3
:105580002430310509F407C10C94103F2A35310548
:1055900009F4DAC174F42B31310509F44AC12C3114
:1055A000310511F00C94103F80E00E94FD690C94CD
:1055B000103F2B35310509F4CBC12C35310511F0E5
:1055C0000C94103F0E94F2670C94103F8091780277
:1055D000882311F40C94103F0E94316885E299E011
:1055E0000E9464EB0E9468508091070A83FD79C095
:1055F000C0903109D0903209E0903309F09034091D
:1056000020912D0530912E0540912F0550913005A8
:10561000C701B6010F940901882309F462C0809183
:1056200046050E94F849882301F1C0922D05D092C9
:105630002E05E0922F05F0923005E4EFF2E284911E
:105640008F010F5F1F4F882321F00E944B72F801DA
:10565000F6CFE6E3F2E084918F010F5F1F4F8823BE
:1056600021F00E944B72F801F6CFC0903109D09022
:105670003209E0903309F090340920912D053091E2
:105680002E0540912F0550913005C701B6010F94AA
:10569000410520E030E048E453E40F946807181611
:1056A00004F5C0922D05D0922E05E0922F05F092C0
:1056B0003005E4EFF2E284918F010F5F1F4F8823E2
:1056C00021F00E944B72F801F6CFE7E1F2E08491FD
:1056D0008F010F5F1F4F882321F00E944B72F8014A
:1056E000F6CF209125093091260940912709509144
:1056F00028096091210570912205809123059091E0
:1057000024050F94090181111DC0209129093091B0
:105710002A0940912B0950912C096091250570911F
:10572000260580912705909128050F940901811184
:1057300009C06091870270918802809189029091DE
:105740008A021AC06091240270912502072E000C73
:10575000880B990B0F940F012091870230918802DA
:105760004091890250918A020F946E012AE037ED30
:1057700043E25CE30F946E010E9496710E949D6C5F
:105780000C94103F81E02230310509F080E00E9446
:10579000A76C0C94103F80E50E94E649882329F00D
:1057A0000E9444496B017C0103C0C12CD12C7601BD
:1057B00083E50E94E649882361F00E94844920E045
:1057C00030E04AE754E40F946E010F948B066B01AE
:1057D0007C010E9444F880913302811105C060E091
:1057E00081E592E00E94E1C50E9468508091E21339
:1057F0009091E313A091E413B091E513C80ED91E64
:10580000EA1EFB1E0E941050DC01CB018C199D0981
:10581000AE09BF09B7FD02C00C94103F80E00E94A2
:10582000D5E8F0CF81E08093780210924A050C947D
:10583000103F0E948D5E81110C94103F80E50E9404
:10584000E649882321F00E945449262F01C020E018
:105850006091290570912A0580912B0590912C0566
:10586000C12CD12CE12C31E4F32EC982DA82EB82F7
:10587000FC82C12CD12C45E8E42E43E4F42ECD82E9
:10588000DE82EF82F886C12CD12C50EAE52E51E45D
:10589000F52EC986DA86EB86FC86C12CD12CE0EC8D
:1058A000EE2EEFE7FE2ECD86DE86EF86F88A2130DB
:1058B00071F1223021F518A219A21AA21BA220E030
:1058C00030E040EA51E40F9442056B017C0120E096
:1058D00030E04AE753E40F946807181634F4C12CFB
:1058E000D12C2AE7E22E23E4F22ECBAEDCAEEDAED5
:1058F000FEAEBE01605E7F4FCE01CB9611C020E0B0
:1059000030E040EA51E40F94090187FF0BC018A270
:1059100019A21AA21BA2BE01605E7F4FCE0109969A
:105920000E94EC6918A219A21AA21BA29E01205E75
:105930003F4F49E255E0BE016B5F7F4FCE010196BC
:105940000E940C690C94103F10923F040C94103F7D
:1059500081E080933F040C94103F8091400490912B
:1059600041048737910511F40C9401350CF0CCC03B
:105970008C34910509F4DDC40CF06BC088319105BD
:1059800009F45CC2B4F58231910509F40AC7C4F484
:1059900097FF02C00C94103F823091050CF4C0C1F7
:1059A000419711F00C94103F60E081E992E00E9471
:1059B000E1C5179816981598149813980C94103FF1
:1059C0008531910509F430C244F4449711F00C94E8
:1059D000103F0E94B6660C94103F8631910509F481
:1059E00027C2479711F00C94103F0E94A2660C94B6
:1059F000103F8E31910509F456C2C4F48A319105E5
:105A000009F449C20CF439C28B31910509F447C23B
:105A10004C9711F00C94103F40E060E080912C0412
:105A200090912D040E948E590C94103F8032910564
:105A300009F449C30CF491C38A32910509F433C4C3
:105A40008B34910511F00C94103F0E94535E0C941E
:105A5000103F8936910509F42AC53CF58335910537
:105A600009F49AC67CF48135910509F476C60CF0E8
:105A70008FC68D34910511F00C94103F0E9487BDA4
:105A80000C94103F8535910509F4BEC60CF489C607
:105A90008C35910509F4D3C68836910511F00C9424
:105AA000103F0E9437870C94103F8F36910509F400
:105AB00057C484F48B36910509F498C50CF471C56C
:105AC0008D36910509F438C58E36910509F435C433
:105AD0000C94103F8337910509F44FC75CF482376B
:105AE000910511F00C94103F0E9444F80E94138518
:105AF0000C94103F8537910509F443C7863791050B
:105B000009F448C70C94103F8C32B1E09B0711F4A4
:105B10000C9454380CF074C0893C910511F40C9429
:105B2000D9354CF58C38910509F4A3C464F4893750
:105B3000910509F4D1C70CF4C8C78D37910509F454
:105B40006DC50C94103F8B39910509F4CAC44CF40F
:105B50008139910511F00C94103F0E94D2850C946C
:105B6000103F8E3B910509F405C5883C910509F469
:105B7000B9C70C94103F833D910511F40C9447373D
:105B800034F58C3C910511F40C9437363CF48B3C85
:105B9000910511F40C940C360C94103F8D3C91053A
:105BA00011F40C94A3368E3C910511F00C94103F27
:105BB0003EE4A32E33E0B32E41E2C42E45E0D42EC2
:105BC00056E6E52E57E0F52E10E00C9410378C3D8C
:105BD000910511F40C94EC373CF48A3D910511F4D5
:105BE0000C94DF370C94103F8D3D910511F40C940B
:105BF000F937823E910511F40C9412380C94103F41
:105C0000843FF1E09F0711F40C949F3E0CF04DC0CF
:105C10008E3531E0930711F40C94C73EB4F48E3204
:105C200051E0950711F40C94983914F40C947D38D4
:105C30008F32B1E09B0711F40C94EC398033914022
:105C400011F40C941B390C94103F8336F1E09F073C
:105C500011F40C94CA3E4CF48F35914011F00C9421
:105C6000103F0E9400820C94103F803941E094075D
:105C700011F40C94C13D8C3A914011F00C94103FFA
:105C800056E6C52E57E0D52E61E2E62E65E0F62EEB
:105C900078EE272E74E0372E00E010E0E22DE0953C
:105CA0002896EFAF28970C94C43D8835A2E09A0758
:105CB00011F40C94C13EB4F4863FE1E09E0711F468
:105CC0000C94A53E14F40C94A23E873F21E0920769
:105CD00011F40C94A83E8C31924011F40C94B63E11
:105CE0000C94103F8C3843E0940711F40C94C43E9C
:105CF0004CF48B38934011F00C94103F0E94AA8210
:105D00000C94103F803AB3E09B0709F419C2873E18
:105D1000934011F00C94103F0E94D4810C94103FDA
:105D2000A0902C04B0902D0480E50E94E6498823C1
:105D300059F00E9444496B017C0111E0672B682BEC
:105D4000692B31F410E004C010E0C12CD12C760195
:105D500083E50E94E6498823F1F00E94844920E00F
:105D600030E04AE754E40F946E010F948B066B0108
:105D70007C01111112C0672B682B692B71F4A114DF
:105D8000B10459F0D5018C91882339F061E0C50147
:105D90000E94FFC507C0112391F360E08EE792E0F7
:105DA0000E94E1C581E08093F10D0E9444F80E94B9
:105DB0006850C114D104E104F104F1F08091E213C0
:105DC0009091E313A091E413B091E513C80ED91E8E
:105DD000EA1EFB1E0E941050DC01CB018C199D09AC
:105DE000AE09BF09B7FF1CC08091F10D8823C1F037
:105DF00080E00E94D5E8EECF8091F10D882321F05C
:105E000080E00E94D5E8F8CF80911F0B60E08823E6
:105E100019F08FE692E002C08AE592E00E94E1C5A7
:105E20001092F10D0C94103F0E94BD5C0C94103F39
:105E300010921F0B1092200B0C94103F19821A82A3
:105E40001B821C8218A219A21AA21BA280914609C9
:105E5000882341F040E0BE016F5F7F4FCE01809606
:105E60000E9402768091200B882319F081E08093B4
:105E70001F0B0E94535E0C94103F10921F0B0E9448
:105E80006F5F8AE992E090935707809356070E94CC
:105E900057460C94103F0E9488660C94103F0E9455
:105EA0004B660C94103F8091200B882311F40C94C6
:105EB000103F81E19DE00E94BF8981E19DE00E9449
:105EC000F18910921E0B10921D0BE0902C04F090A3
:105ED0002D048091200B882311F40C94103F0E9414
:105EE0007CBD1D8218861C821B8284E993E09A8304
:105EF000898383E79BE09093930B8093920BF70148
:105F000080818F3209F068C06FE270E0C7010F94A2
:105F100071088C010F5F1F4F9E012F5F3F4F49019A
:105F20000115110509F45EC06FE270E0C8010F941D
:105F300071086C01009709F456C00817190708F09A
:105F400052C05C01A01AB10AA501B801CE01809629
:105F50000F949108E0E2F0E0EC0FFD1FEA0DFB1D4D
:105F600010828E01005E1F4FD8018D918D01882314
:105F700019F00E944B72F8CF8AE00E944B72609138
:105F8000920B7091930B6115710511F06C5F7F4F4F
:105F900021E0AE01405E5F4FCE0105960E94F58F75
:105FA000811112C0BE01605E7F4F85EC92E00E94BD
:105FB00063C18EE20E944B728AE00E944B72C40160
:105FC0000E945CE80C94103F9092930B8092920B8D
:105FD00086010F5F1F4FA4CF84E99BE09093930B42
:105FE0008093920B87016091920B7091930B6115D6
:105FF000710511F06C5F7F4F18A21BA222E0A8016F
:10600000CE0180960E94F58F811102C0F12C14C040
:10601000CE0180960E94EABC8823C1F361E0CE01E4
:1060200080960E94A389009789F325EEFC012083C6
:106030001BA20E940FB0F82ECE0180960E94F2495A
:10604000FF2011F19FE9E92E92E0F92EF7018491EA
:10605000882331F0FFEFEF1AFF0A0E944B72F6CF50
:10606000D8018D918D01882319F00E944B72F8CFD1
:106070008AE00E944B721092C20D1092C30D1092D2
:10608000C40D1092C50D19C08DEAE82E82E0F82EDD
:10609000F7018491882331F0FFEFEF1AFF0A0E9485
:1060A0004B72F6CFD8018D918D01882319F00E9493
:1060B0004B72F8CF8EE20E944B72CE0101960E9485
:1060C0005CE80C94103F80911F0B81110E9444F8F2
:1060D000E0902C04F0902D0480E50E94B749182F21
:1060E000882319F00E947549182F8091200B88236E
:1060F00011F40C94103F412F61E0C7010E948E59AA
:1061000083E50E94E649882381F00E945449AB014F
:10611000BC014093C20D5093C30D6093C40D7093A6
:10612000C50D81E19DE00E94BA888091200B8823F3
:1061300019F081E080931F0B11110C94103F99CE40
:1061400080912C0490912D0421E020931E0B40E0BF
:1061500060E00E948E590C94103F0E94F4BE1CE334
:10616000C12ED12CE12CF12CA70196010F94E4044F
:10617000762E672ECA01B901A70196010F94E40497
:106180006B017C01CA01B90128E130E040E050E038
:106190000F94E4044B015C01C9016DE671E00F94BA
:1061A00006088E010F5F1F4F6115710599F06F9200
:1061B0007F92DF92CF929F928F929F938F937F9344
:1061C0006F9381E093E09F938F931F930F930F94AE
:1061D000A20012C00097B1F06F927F92DF92CF922F
:1061E0009F928F929F938F9381EF92E09F938F93D3
:1061F0001F930F930F94A2000FB6F894DEBF0FBE4B
:10620000CDBF36C081149104A104B10479F06F921E
:106210007F92DF92CF929F928F9285EE92E09F9332
:106220008F931F930F930F94A200E6CFC114D10454
:10623000E104F10469F06F927F92DF92CF928DEDCD
:1062400092E09F938F931F930F930F94A200D4CF4C
:106250006F927F9289ED92E09F938F931F930F939C
:106260000F94A2000F900F900F900F900F900F902F
:1062700060E0C8010E94FFC5E4EFF2E284917F0173
:106280009FEFE91AF90A882321F00E944B72F70167
:10629000F5CFB80185E193E00E9463C18AE00E94D6
:1062A0004B720C94103F83E50E94E649882311F459
:1062B0000C94103F0E946449E82E80E50E94E64954
:1062C000882311F40C94103F80E50E94E64988234E
:1062D00039F00E9454498B0177FF04C00C94103FA1
:1062E0000DE010E0902FE2E2F3E080E38E0F2491C6
:1062F000921729F031968E13FACF0C94243FE5EFD4
:10630000F6E184918F010F5F1F4F882321F00E94D7
:106310004B72F801F6CFE2E5F3E084918F010F5F55
:106320001F4F882311F40C94103F0E944B72F80108
:10633000F4CF0E946F5F0C94103F8EE40E94E649F8
:10634000882311F40C94103F0E9454496093C513A4
:106350007093C6138093C7139093C8130C94103F87
:1063600083E50E94E649882319F00E94644901C030
:1063700080E08093070AE4EFF2E284918F010F5FDF
:106380001F4F882321F00E944B72F801F6CFEFE6F1
:10639000F3E084918F010F5F1F4F882321F00E944B
:1063A0004B72F801F6CF8091070A8823A1F1B1E67C
:1063B000CB2EB3E0DB2EE12CF12C20E08091070AFC
:1063C00090E00E2C02C0959587950A94E2F780FF25
:1063D00017C0BB24B394B20E222319F08CE20E94A2
:1063E0004B72F60125913491F901849189010F5F77
:1063F0001F4F882321F00E944B729801F5CF2B2D5F
:10640000FFEFEF1AFF0A32E0C30ED11C45E0E4169D
:10641000F104A1F629C0EBE6F3E084918F010F5F50
:106420001F4F882309F10E944B72F801F6CF0DE24D
:1064300015E180E20E944B72D8016D917D918D91A2
:106440009D918D0142E00E9424738CE20E944B7268
:10645000F801648175818681978142E00E942473EE
:10646000F5E105331F0729F78AE00E944B720C946F
:10647000103F8091070A83FF02C00C94103F83E510
:106480000E94E649882311F40C94103F0E9484492D
:106490000F9486066739710514F066E970E0709311
:1064A000160A6093150A0E94CBCD0C94103F89E622
:1064B00090E00E94067281110C949644E6E7F3E0A6
:1064C00084918F010F5F1F4F882321F00E944B7230
:1064D000F801F6CF0E9449868AE00E944B720C9424
:1064E000964483E50E94E649882311F40C94103FFA
:1064F0000E9464498093CD138D3318F08CE3809310
:10650000CD130E9410506B017C012091CD1330E01F
:10651000A8EEB3E00F943205DC01CB018C0D9D1D7C
:10652000AE1DBF1D8093C9139093CA13A093CB13C4
:10653000B093CC130C94103F8DE690E00E9406724D
:1065400081110C94103F8091070A83FF02C00C94C4
:10655000103F83E50E94E64928968FAF2897811166
:106560000C94403F82E50E94E64981110C94403F23
:106570000C94103F8091070A83FF02C00C94103FD7
:1065800083E50E94E6492E968FAF2E9781110C94D9
:10659000044182E50E94E64981110C9404410C9467
:1065A000103F83E50E94E649882339F00E94544950
:1065B0008B016F3F710519F010F00FEF10E080E5CF
:1065C0000E94E649882339F00E946449823010F025
:1065D0000C94103F01C080E0E82FF0E0EE0FFF1FA9
:1065E000EF5EF54F118300830C94103F80E50E940D
:1065F000E649882341F00E9454496230710510F049
:106600000C94103F02C060E070E0660F771FFB0142
:10661000EF5EF54F118210820C94103F8CE40E94C3
:10662000B749882319F00E94844904C060E070E0F3
:1066300080E090EC27966CAF7DAF8EAF9FAF279731
:106640008AE50E94E649882319F00E94844903C024
:1066500060E070E0CB0120E030E040E251E40F94D4
:10666000420523966CAF7DAF8EAF9FAF239788E531
:106670000E94E649882319F00E94844903C060E023
:1066800070E0CB0120E030E040E251E40F9442059D
:10669000E0914605EE2359F0A4E0EA9FF0011124B1
:1066A000E35DFA4E208131814281538103C020E0B5
:1066B00030E0A9010F9442056BAF7CAF8DAF9EAF68
:1066C00089E50E94E649882319F00E94844903C0A5
:1066D00060E070E0CB0120E030E04AE853E40F9442
:1066E000420520E030E040E251E40F944105E091A2
:1066F0004605EE2359F0B4E0EB9FF0011124EB5C6A
:10670000FA4E208131814281538103C020E030E084
:10671000A9010F94420568A379A38AA39BA31982B8
:106720001A821B821C828091460981110C94103FB1
:10673000C12CE12C8E010F5F1F4F9E01205E3F4F49
:10674000AE01455C5F4FBE01615C7F4FCE018D5B4A
:106750009F4F0E947D740C94103F0E946ECE0E9449
:1067600044F80E9467E81092120A1092110A1092DF
:10677000140A1092130A68EE73E080E090E00E9421
:1067800048C460E085EE93E00E94E1C50C94103FA0
:1067900010923E040C94103F81E080933E040C94D0
:1067A000103F83E50E94E6498823A1F00E948449B6
:1067B00020E030E04AE754E40F946E010F948B061A
:1067C0006093830270938402809385029093860283
:1067D0000C94103F88E50E94B74981110C948B42BC
:1067E00089E50E94B74981110C948B428AE50E9489
:1067F000B74981110C948B4285E40E94B7498111FD
:106800000C948B420C94AA4283E50E94B7498823DA
:1068100011F40C94103F0E94844920E030E04AE7D4
:1068200054E40F946E010F948B066093E6137093FB
:10683000E7138093E8139093E9130C94103F8CE5D1
:1068400090E00E94067281110C94103FEEE4F3E098
:106850002996FFAFEEAF2997A1E3CA2EA5E0DA2E65
:10686000F12C2996AEADBFAD29978D912996BFAF7A
:10687000AEAF29970E94B749882309F473C0B3E0EB
:10688000FB1269C00E9484492B013C0120E030E0EA
:1068900040EA51E40F940901E0902E0487FF50C0B4
:1068A0000E2D10E00D5F1F4F000F111F000F111F65
:1068B000F801EF5CFA4FA30192016081718182813E
:1068C00093810F941E064B015C019B01AC0160910A
:1068D000740A7091750A8091760A9091770A0F94E4
:1068E0006E016093740A7093750A8093760A909390
:1068F000770AF801EC5DF54F1F01A5019401608155
:106900007181828193810F946E01D1016D937D938A
:106910008D939C9313970356114FF80160817181F9
:10692000828193810F940D01A50194010F946E0152
:106930000F948B06D8016D937D938D939C93139741
:10694000B4E0EB9EF0011124E35CFA4F40825182E7
:106950006282738207C00E948449F601608371835A
:1069600082839383F394F4E0CF0ED11C24E0F212DF
:1069700078CF0E9407E60C94103F0E948A840C9402
:10698000103F60E080912C0490912D040E94FFC57F
:106990000C94103F85E40E94B749882381F00E943F
:1069A0007549882361F0E4EFF2E284918F010F5F73
:1069B0001F4F882321F00E944B72F801F6CF81E42B
:1069C0000E94B749882381F00E947549882361F0AD
:1069D000E8EFF3E084918F010F5F1F4F882321F0D0
:1069E0000E944B72F801F6CF00912C0410912D04F7
:1069F000D8018D918D01882309F436CD0E944B7208
:106A0000F7CFE4E1F4E084918F010F5F1F4F8823FB
:106A100021F00E944B72F801F6CFECE0F4E0849193
:106A20008F010F5F1F4F882321F00E944B72F801E6
:106A3000F6CF1E9B03C00AEE12E002C00FEE12E07A
:106A4000F80181918F01882319F00E944B72F8CFD1
:106A50008AE00E944B72E4E0F4E084918F010F5FC2
:106A60001F4F882321F00E944B72F801F6CF1D9B27
:106A700003C00AEE12E002C00FEE12E0D8018D91C1
:106A80008D01882319F00E944B72F8CF8AE00E9492
:106A90004B72ECEFF3E084918F010F5F1F4F88235F
:106AA00021F00E944B72F801F6CF1C9B03C00AEE46
:106AB00012E002C00FEE12E0F80181918F018823ED
:106AC00009F4D2CC0E944B72F7CF81E08093650726
:106AD000809364070C94103F10926507109264072E
:106AE0000C94103F88EC90E00E94067281110C9487
:106AF000103F84E40E94B749882309F456C00E94DD
:106B0000844911E020E030E0A9010F9409018111CE
:106B100001C010E010935115112309F446C00091F3
:106B20002E0410E00E948449000F111F000F111F56
:106B3000F801E75BFA4E608371838283938320E0E0
:106B400030E0A9016091491570914A1580914B156B
:106B500090914C150F94090181110CC080E090E0D8
:106B6000A0E4B0E48093491590934A15A0934B1587
:106B7000B0934C1520E030E0A90160914D15709163
:106B80004E1580914F15909150150F940901811168
:106B90000CC080E090E0A0E4B0E480934D159093A9
:106BA0004E15A0934F15B09350150E94E3EA0C9434
:106BB000103F89EC90E00E94067281110C94103F06
:106BC0007EE4C72E73E0D72E00E0D6018D916D01D3
:106BD0000E94B7498823C9F0033019F410912E049C
:106BE00001C010E00E948449100FB4E01B9F900187
:106BF0001124F901E75CF54F7F010F948B06D70153
:106C00006D937D938D939C9313970F5F0430E9F6FA
:106C10000E94B7E40C94103F8BEC90E00E94067247
:106C200081110C94103F6EE4E62E63E0F62E00E036
:106C3000F70181917F010E94B749882399F00330C1
:106C400019F410912E0401C010E00E948449100F25
:106C500024E0129FF0011124EC5DF54F60837183F5
:106C6000828393830F5F043019F70C94103F83E500
:106C70000E94B7498823D9F00E948449AB01BC0126
:106C80004093550A5093560A6093570A7093580AD6
:106C900040934D0A50934E0A60934F0A7093500AE6
:106CA00088E894E00E9406C18AE00E944B7280E569
:106CB0000E94B749882399F00E948449AB01BC0126
:106CC0004093550A5093560A6093570A7093580A96
:106CD0008BE694E00E9406C18AE00E944B7282E536
:106CE0000E94B749882399F00E948449AB01BC01F6
:106CF0004093510A5093520A6093530A7093540A76
:106D00008CE494E00E9406C18AE00E944B7284E504
:106D10000E94B749882311F40C94103F0E948449C3
:106D2000AB01BC0140934D0A50934E0A60934F0A49
:106D30007093500A8EE294E00E9406C18AE00E949D
:106D40004B720C94103F83E50E94B749882351F0A1
:106D50000E9484496093200A7093210A8093220A3A
:106D60009093230A84E50E94B749882351F00E943A
:106D7000844960931C0A70931D0A80931E0A9093A5
:106D80001F0A82E40E94B749882351F00E944449B7
:106D90006093451570934615809347159093481559
:106DA00088E50E94B749882351F00E948449609386
:106DB000680A7093690A80936A0A90936B0A89E55E
:106DC0000E94B749882351F00E94844960936C0A5D
:106DD00070936D0A80936E0A90936F0A8AE50E9401
:106DE000B749882351F00E9484496093700A7093D8
:106DF000710A8093720A9093730A85E40E94B749DE
:106E0000882311F40C94103F0E9484496093740A03
:106E10007093750A8093760A9093770A0C94103FCA
:106E2000D5018D915D010E94B749882311F10E941F
:106E300084492B013C01F70120813181428153813A
:106E40000F9441059B01AC01D6016D917D918D910F
:106E50009C910F944205F601608371838283938332
:106E6000D7014D925D926D927C921397812F0E9473
:106E7000AF711F5FB4E0CB0ED11CE4E0EE0EF11C4D
:106E8000133071F60E943A490E941385C9C7E4EF96
:106E9000F2E284918F010F5F1F4F882321F00E943F
:106EA0004B72F801F6CF83E50E94B749882321F0A1
:106EB0000E94754980933202E8EDF4E084918F01DD
:106EC0000F5F1F4F882321F00E944B72F801F6CF0D
:106ED00080913202811103C0E4EDF4E002C0E0EDE4
:106EE000F4E084918F010F5F1F4F882321F00E94EF
:106EF0004B72F801F6CFE8ECF4E084918F010F5F5C
:106F00001F4F882321F00E944B72F801F6CF409169
:106F10002F0450913004609131047091320486EC5A
:106F200094E00E9406C14091330450913404609172
:106F300035047091360483EC94E00E9406C14091C0
:106F40003704509138046091390470913A0480EC10
:106F500094E00E9406C1E8EBF4E084918F010F5F9A
:106F60001F4F882321F00E944B72F801F6CF409109
:106F7000260250912702609128027091290286EB27
:106F800094E00E9406C140912A0250912B02609128
:106F90002C0270912D0283EB94E00E9406C1409177
:106FA0002E0250912F02609130027091310280EBDD
:106FB00094E00E9406C18AE00E944B7231C78AEDBC
:106FC00090E00E94067281112BC710912E041123AC
:106FD00009F426C70C94AF4283E50E94E649882352
:106FE00009F41EC70E94544970932502609324023D
:106FF00017C78DED90E00E940672811111C783E5DD
:107000000E94E649882309F40BC700912E0410E082
:107010000E945449000F111FF801E05EFD4F71837B
:107020006083FEC680E50E94B749882309F4F8C64C
:107030000E945449F62E062F172F83E50E94E64939
:10704000882321F00E9454496B0103C0CC24CA94C8
:10705000DC2CC6010196039708F0E2C617FDE0C6D6
:107060000E9444F82FEFC216D20631F0CA94CD2800
:1070700071F401E010E00DC08F2D0E94B64E31E09A
:1070800020E0892B09F030E0032F122F02C000E02E
:1070900010E08F2D0E94B64E8017910709F4C0C6EC
:1070A00080E00E94D5E8F5CF83E50E94E649882379
:1070B00019F00E94544902C064E071E079A368A30A
:1070C00080E50E94E649882339F00E9454496938D6
:1070D00043E1740730F402C068EE73E07A83698399
:1070E00004C088E893E19A838983BE01605E7F4F84
:1070F000CE0101960E94045E93C685E40E94E64993
:10710000811110C080E50E94B749882391F00E9448
:10711000844960931D1570931E1580931F159093DD
:10712000201507C00E946449823060F3E5EFF6E164
:1071300071C089E40E94B749882381F00E94844984
:107140002CEA35EC47E25EE30F946E01609319156B
:1071500070931A1580931B1590931C1584E40E945C
:10716000B749882381F00E9484492CEA35EC47E234
:107170005EE30F941E0660931515709316158093A9
:10718000171590931815E4EFF2E284918F010F5FC9
:107190001F4F882321F00E944B72F801F6CF4091D7
:1071A0001D1550911E1560911F157091201580E0DE
:1071B00095E00E9406C12CEA35EC47E25EE360915F
:1071C000191570911A1580911B1590911C150F942B
:1071D0001E06AB01BC018CEF94E00E940F662CEA06
:1071E00035EC47E25EE360911515709116158091BC
:1071F0001715909118150F946E01AB01BC0188EF23
:1072000094E00E940F668AE00E944B7209C60E94B9
:107210004B72F80184918F010F5F1F4F8111F7CFDF
:1072200001E013E0D8018D918D01882309F41CC978
:107230000E944B72F7CF80E50E94B749882351F036
:107240000E94844960931115709312158093131551
:107250009093141589E40E94B749882381F00E9415
:1072600084492CEA35EC47E25EE30F946E016093AB
:107270000D1570930E1580930F159093101584E4DF
:107280000E94B749882381F00E9484492CEA35EC9A
:1072900047E25EE30F941E066093091570930A158A
:1072A00080930B1590930C15E4EFF2E284918F011B
:1072B0000F5F1F4F882321F00E944B72F801F6CF19
:1072C000409111155091121560911315709114157C
:1072D0008CE095E00E9406C12CEA35EC47E25EE3C3
:1072E00060910D1570910E1580910F1590911015EC
:1072F0000F941E06AB01BC0188E095E00E940F666A
:107300002CEA35EC47E25EE36091091570910A15AD
:1073100080910B1590910C150F946E01AB01BC017F
:1073200084E095E00E940F668AE00E944B7278C567
:1073300083E50E94B749182F882371F00E94844981
:107340000F94860670931F0260931E0221E0672B44
:1073500009F020E02093060A80E50E94B7498823BF
:1073600059F020911E0230911F02232B11F00E9430
:1073700075498093060A54C5111152C5E4EFF2E233
:1073800084918F010F5F1F4F882321F00E944B7261
:10739000F801F6CF8091060A811103C069EF72E00F
:1073A00002C06CEE72E085E295E00E9463C16091DC
:1073B0001E0270911F0284E195E00E944AC1E0E143
:1073C000F5E084918F010F5F1F4F882309F428C5D2
:1073D0000E944B72F801F5CF85E40E94E6498823AC
:1073E00021F00E9454491B0102C0212C312C83E45E
:1073F0000E94E649882339F00E945449E9967FAFFC
:107400006EAFE99706C0E5E0F0E0E996FFAFEEAFBA
:10741000E99785E50E94B749AE968FAFAE9788236E
:1074200029F00E947549AE968FAFAE9737FC07C022
:10743000C12CD12CB6E1EB2EB3E4FB2E06C0C12C3F
:10744000D12CACE8EA2EA2E4FA2E83E50E94E649AC
:10745000882321F00E9484496B017C01F2E02F1601
:10746000310410F420922E040E9410502B013C0194
:10747000C1010196039718F402E113E00CC005E284
:1074800013E0D8018D918D01882311F40C943432CE
:107490000E944B72F6CFF80181918F01882319F079
:1074A0000E944B72F8CF8AE00E944B720E946ECE0F
:1074B000FFEF2F163F0649F487E68093920EF7E61A
:1074C0008F2E912CA12CB12C0AC08FE7F101EB5625
:1074D000F14F8083EFE78E2E912CA12CB12CC701A8
:1074E000B6010F948606072E000C880B990B0F949B
:1074F0000F01A0966FAFA097A1967FAFA197A2961C
:107500008FAFA297A3969FAFA39781E080939A0233
:107510002FEF2216320629F48EEC90E0A0E0B0E0C6
:1075200004C08FEF90E0A0E0B0E09C01AD012351DA
:10753000310941095109C158DF4F288339834A83F2
:107540005B83CF57D0409C01AD01245131094109E3
:107550005109CD57DF4F288339834A835B83C35852
:10756000D0409C01AD015595479537952795C95752
:10757000DF4F288339834A835B83C758D0409C01FF
:10758000AD012150310941095109C557DF4F288309
:1075900039834A835B83CB58D04061968CAE9DAED5
:1075A000AEAEBFAE6197E3964CAE5DAE6EAE7FAE53
:1075B000E397ED964CAE5DAE6EAE7FAEED97A496C2
:1075C0001FAEA49730E4A5963FAFA5974CE1A696D1
:1075D0004FAFA69756E4A7965FAFA797A8961FAEA2
:1075E000A897A9961FAEA997AA961FAEAA97AB9681
:1075F0001FAEAB976F961CAE1DAE1EAE1FAE6F9743
:107600006B961CAE1DAE1EAE1FAE6B97C12CD12C5F
:107610007601E7961CAE1DAE1EAE1FAEE79781E069
:10762000AF968FAFAF9767961FAE1EAE679728963F
:107630001FAE28972A961FAE2A9700E010E0D101CE
:10764000AB56B14FEF96BFAFAEAFEF97C101880F0A
:10765000991F880F991FFC01E452FB4FAD96FFAFB5
:10766000EEAFAD9780919A02882309F483C20E94FD
:10767000105065966CAF7DAF8EAF9FAF65978091D0
:10768000820E882309F434C10E9454CFFFEF2F16D5
:107690003F0679F42091E40428962FAF2897309183
:1076A000E5042A963FAF2A970091E6041091E7047B
:1076B00019C0AD96AEADBFADAD97BC912896BFAF2A
:1076C0002897AD96EEADFFADAD97F1812A96FFAF4D
:1076D0002A97AD96AEADBFADAD9712960C911297AD
:1076E00013961C9128962FAD28972A963FAD2A977E
:1076F000A801A8966FADA897A9967FADA997AA965D
:107700008FADAA97AB969FADAB970F94090187FFFA
:1077100012C02896BFAD2897A896BFAFA8972A9603
:10772000EFAD2A97A996EFAFA997AA960FAFAA97A0
:10773000AB961FAFAB9728962FAD28972A963FADF3
:107740002A97A801A4966FADA497A5967FADA5979B
:10775000A6968FADA697A7969FADA7970F9468079B
:10776000181694F42896FFAD2897A496FFAFA49717
:107770002A962FAD2A97A5962FAFA597A6960FAF5D
:10778000A697A7961FAFA797AF963FADAF97A096C6
:107790002FADA097332309F47FC0A1963FADA197E9
:1077A000A2964FADA297A3965FADA39728966FAD13
:1077B00028972A967FAD2A97C8010F946807181654
:1077C0000CF096C065968CAD9DADAEADBFAD659726
:1077D00084199509A609B709C157DF4F8883998392
:1077E000AA83BB83CF58D04088589341A109B109DF
:1077F000B7FD7EC0D501C40161962CAD3DAD4EAD47
:107800005FAD6197821B930BA40BB50BB595A79544
:10781000979587953FEF2316330619F48093920EC0
:1078200005C0EF96EEADFFADEF978083C157DF4FF8
:10783000288139814A815B81CF58D040E7962CAFAF
:107840003DAF4EAF5FAFE797A0963FADA097A8962C
:107850003FAFA897A1964FADA197A9964FAFA99713
:10786000A2965FADA297AA965FAFAA97A3968FAD97
:10787000A397AB968FAFAB9765962CAD3DAD4EAD54
:107880005FAD6597E3962CAF3DAF4EAF5FAFE3972B
:10789000AF961FAEAF972CC0A1963FADA197A29611
:1078A0004FADA297A3965FADA39728966FAD28978B
:1078B0002A967FAD2A97C8010F94090187FF18C047
:1078C00065968CAD9DADAEADBFAD6597E3962CAD25
:1078D0003DAD4EAD5FADE397821B930BA40BB50B93
:1078E000AC01BD01485853416109710977FF73C666
:1078F00020E030E040EA51E4A0966FADA097A19659
:107900007FADA197A2968FADA297A3969FADA397A7
:107910000F9442059B01AC0128966FAD28972A96DB
:107920007FAD2A97C8010F94680718166CF4E5EF2D
:10793000F5E084918F010F5F1F4F882309F470C217
:107940000E944B72F801F5CF80E398EFAFEFBFEFE5
:10795000ED962CAD3DAD4EAD5FADED97821B930B1B
:10796000A40BB50B65962CAD3DAD4EAD5FAD6597E7
:10797000820F931FA41FB51FB7FD11C00E94498637
:107980008AE00E944B7265968CAD9DADAEADBFADE9
:107990006597ED968CAF9DAFAEAFBFAFED97659697
:1079A0008CAD9DADAEADBFAD6597880F991FAA1F79
:1079B000BB1FE3962CAD3DAD4EAD5FADE397821B93
:1079C000930BA40BB50B84199509A609B709813847
:1079D0009F44A241B10568F0E7EDF5E084918F0185
:1079E0000F5F1F4F882309F41BC20E944B72F801DE
:1079F000F5CF67964EAD5FAD6797E9968EAD9FADBB
:107A0000E997841795070CF0B2C0EAE7F5E0849196
:107A10008F010F5F1F4F882321F00E944B72F801E6
:107A2000F6CF9FEF2916390619F009EC13E002C0D2
:107A30000DEF12E0B80188E695E00E9463C1B7013E
:107A4000A60184E695E00E9406C18AE00E944B727E
:107A5000B80182E595E00E9463C16B964CAD5DADC7
:107A60006EAD7FAD6B978EE495E00E9406C18AE013
:107A70000E944B72B8018CE395E00E9463C16F963F
:107A80004CAD5DAD6EAD7FAD6F9788E395E00E9424
:107A900006C18AE00E944B72AE96AFADAE97AA23A4
:107AA00009F4BEC12320209489F5C0921115D0920B
:107AB0001215E0921315F09214152CEA35EC47E2FA
:107AC0005EE36B966CAD7DAD8EAD9FAD6B970F9405
:107AD0006E0160930D1570930E1580930F159093A2
:107AE00010152CEA35EC47E25EE36F966CAD7DAD88
:107AF0008EAD9FAD6F970F941E066093091570931E
:107B00000A1580930B1590930C158AC1C0921D1510
:107B1000D0921E15E0921F15F09220152CEA35EC3C
:107B200047E25EE36B966CAD7DAD8EAD9FAD6B971E
:107B30000F946E016093191570931A1580931B159D
:107B400090931C152CEA35EC47E25EE36F966CAD22
:107B50007DAD8EAD9FAD6F970F941E06609315158A
:107B600070931615809317159093181559C10E949C
:107B70000FC678CD80919A02811152C10E946ECEBB
:107B80004FC10E9444F84CC1D1018D911D01882341
:107B900009F4A3C0F7014080518062807380F8012E
:107BA000EA5DFD4F2081318142815381F801E15D21
:107BB000FB4F60817181828193810F94420520E0A7
:107BC00030E040E05FE30F946E019B01AC01C30124
:107BD000B2010F946807181644F4F801EE5DF64CF4
:107BE00085909590A590B49003C0812C912C540160
:107BF000F801E651FC4E2081318142815381C3015D
:107C0000B2010F9441059B01AC01C501B4010F9471
:107C100041054B015C0120E030E040EA51EC0F945B
:107C2000680787FD2BC020E030E040EA51E4C50141
:107C3000B4010F94090118160CF1D6012D913D9154
:107C40004D915C91C501B4010F9441059B01AC01BC
:107C5000C301B2010F944205F701608371838283EF
:107C60009383D6018D929D92AD92BC9213972896E4
:107C70008FAD2897820D0E94AF712FC0E5EFF6E11E
:107C800084918F010F5F1F4F882321F00E944B7258
:107C9000F801F6CFE7E8F6E084918F010F5F1F4F00
:107CA000882321F00E944B72F801F6CF61E089E74A
:107CB00096E00E94E1C50E94175688E290E09A8300
:107CC000898388EC90E099A388A3BE016F5F7F4F02
:107CD000CE0180960E94045EA3C0B4E0CB0ED11CFE
:107CE0000C5F1F4FE4E0EE0EF11C0C30110509F0A3
:107CF0004BCF0E943A490E94138560E089E696E0E6
:107D00000E94E1C583E992E099A388A304E610E00C
:107D10001A830983BE01605E7F4FCE0101960E94E7
:107D2000045E8AEB92E099A388A31A830983BE01BB
:107D3000605E7F4FCE0101960E94045E71C00E947A
:107D4000FCD86EC00E94DDD36BC00E94B8F468C03E
:107D500083E50E94B749882319F00E94754901C044
:107D600081E091E089270E94B2EF5AC083E50E942A
:107D7000B749882309F454C00E9475498093760757
:107D80004FC00E94DB824CC00E948D8249C00E947D
:107D9000558246C00E94E58143C000914004809115
:107DA0004605081751F083E50E94B749182F88232C
:107DB00029F00E947549182F01C011E086E40E9445
:107DC000E649882319F00E94844903C060E070E00E
:107DD000CB0120E030E040E752E40F941E06AB01F7
:107DE000BC01212F802F0E949F811AC0E4EFF2E294
:107DF00084918F010F5F1F4F882321F00E944B72E7
:107E0000F801F6CF6091E0137091E11385EA96E0F6
:107E10000E9463C182E20E944B728AE00E944B7210
:107E20000E94B9EB83C540912C0450912D04452B41
:107E300039F4AF014150510950932D0440932C0463
:107E400040E050E00C945E2A802F0E9484BB6E2D8F
:107E5000802F0E94DF4EF12CB701802F0E940F4F20
:107E60000630110529F4F092120AE092110AD8CFD7
:107E700008301105A9F6F092140AE092130AD0CF47
:107E80000E948449F0902E042F2D30E0220F331FE2
:107E90008901095E154F0F948606D8016D937C9376
:107EA0008F2D0E9416CE0E94844920E030E040E7EA
:107EB00052E40F940901181644F00E9487BD60E057
:107EC00088EA93E00E94E1C502C00E94535E0091DF
:107ED0002E0410E0F801EE0FFF1FE95EF54F608100
:107EE0007181072E000C880B990B0F940F01F8017C
:107EF000EE0FFF1FEE0FFF1FE452FB4F2081318179
:107F0000428153810F94680718160CF075C184EDF7
:107F100092E09F938F930F5F1F4F1F930F9389E9F9
:107F200093E09F938F931F920E94385E0FB6F89450
:107F3000DEBF0FBECDBF81E080939A022D961CAEAE
:107F40001DAE1EAE1FAE2D9765961CAE1DAE1EAEAD
:107F50001FAE6597312C66961FAE66979CE36896B8
:107F60009FAF6897ACE16C96AFAF6C97B6E4A09604
:107F7000BFAFA097C12CD12C50E8E52E6FEBF62EA9
:107F8000812C912C540100912E0410E0F801EE0F89
:107F9000FF1FE95EF54F60817181072E000C880B91
:107FA000990B0F940F01762E672E582E492E262FEF
:107FB000372F482F592FB601C7010F940901882385
:107FC000F9F0000F111F000F111FF801E452FB4FD1
:107FD0002081318142815381672D762D852D942D0D
:107FE0000F940901382E331C3324331C2896CFAC50
:107FF0002897CC2049F0332039F033243394EAC059
:108000007C2C6D2C5E2C4F2C0E9410506B017C013F
:10801000DC01CB0165962CAD3DAD4EAD5FAD6597F6
:10802000821B930BA40BB50BB7FD3CC0D701C60157
:1080300088519C4FAF4FBF4F65968CAF9DAFAEAF91
:10804000BFAF65970E944986E5E9F3E084918F010F
:108050000F5F1F4F882321F00E944B72F801F6CF6B
:1080600081149104A104B104B9F0D501C40188516F
:108070009C4FAF4FBF4FBC01CD016C197D098E09DC
:108080009F0928EE33E040E050E00F94E404CA0179
:10809000B9010E940A7303C08FE30E944B728AE009
:1080A0000E944B7280E00E94D5E80E946850E091E7
:1080B0002E0494E0E99FF0011124E452FB4F20804C
:1080C000A1812E96AFAF2E9702811381222D3A2FD8
:1080D000A801672D762D852D942D0F9441059F774E
:1080E00020E030E040E251E481149104A104B104A5
:1080F00029F40F94090187FF07C004C00F94680793
:10810000181614F446015701332009F449C02D967E
:108110002CAD3DAD4EAD5FAD2D972115310541051F
:10812000510541F0D701C601821B930BA40BB50B7F
:10813000B7FD36C0222D2E963FAD2E97A80166962C
:108140006FAD669768967FAD68976C968FAD6C97AC
:10815000A0969FADA0970F94410520E030E040EC41
:108160005FE30F94090187FD48CFD701C601805A0C
:108170009541AF4FBF4F2D968CAF9DAFAEAFBFAF08
:108180002D9766962FAE66972E969FAD2E97689682
:108190009FAF68976C960FAF6C97A0961FAFA09794
:1081A00080919A028823B1F081149104A104B10452
:1081B00029F4C72CD62CE52CF42CE5CEA8EECA1A4F
:1081C000A3E0DA0AE108F108C818D908EA08FB08B0
:1081D000F7FCEFCF80919A02882309F421CE60E06A
:1081E000332029F089E793E00E94E1C519CE87E8A2
:1081F00093E00E94E1C514CE2896CFAC2897C11019
:108200009ACE8FED92E085CE0E9484490F94860627
:108210006739710514F066E970E07093160A60938F
:10822000150A0E94CBCD0E94844920E030E040EA4C
:1082300050E40F946807181614F40E94535E60917E
:10824000150A7091160A072E000C880B990B0F94D3
:108250000F012091E4043091E5044091E60450912F
:10826000E7040F94090160E087FF03C088ED93E005
:1082700002C08BEC93E00E94E1C581E080939A02FA
:108280008091460580932E042D961CAE1DAE1EAE29
:108290001FAE2D9765961CAE1DAE1EAE1FAE659728
:1082A00028961FAE289766961FAE6697BCE3689621
:1082B000BFAF6897ECE16C96EFAF6C97F6E4A096D1
:1082C000FFAFA097C12CD12C90E8E92E2FEBF22E16
:1082D000812C912C54016091150A7091160A072E79
:1082E000000C880B990B0F940F01162F072F782E77
:1082F000692E262F372F482F592FB601C7010F940B
:108300000901882331F12091E4043091E504409182
:10831000E6045091E704612F702F872D962D0F945E
:108320000901881F8827881F28968FAF28972E96C7
:10833000CFAC2E97CC2089F0882379F080919A02D7
:10834000882309F46DCD60E08DEB93E00E94E1C5D8
:1083500067CD1C2D0D2D7E2C6F2C0E9410506B01B3
:108360007C01DC01CB0165962CAD3DAD4EAD5FAD22
:108370006597821B930BA40BB50BB7FD3DC0D701CE
:10838000C60188519C4FAF4FBF4F65968CAF9DAFD4
:10839000AEAFBFAF65970E944986E7ECF3E08491EA
:1083A0002F019FEF491A590A882321F00E944B722E
:1083B000F201F5CF81149104A104B104B9F0D50103
:1083C000C40188519C4FAF4FBF4FBC01CD016C1908
:1083D0007D098E099F0928EE33E040E050E00F94BC
:1083E000E404CA01B9010E940A7303C08FE30E942A
:1083F0004B728AE00E944B7280E00E94D5E80E9496
:1084000068502090E4043090E5044090E6045090D9
:10841000E7049101A201612F702F872D962D0F94F3
:1084200041059F7720E030E040EA50E48114910458
:10843000A104B10429F40F94090187FF07C004C007
:108440000F946807181614F4460157012896AFAD2B
:108450002897AA2309F443C02D962CAD3DAD4EAD0F
:108460005FAD2D97211531054105510541F0D7012B
:10847000C601821B930BA40BB50BB7FD30C0910155
:10848000A20166966FAD669768967FAD68976C9609
:108490008FAD6C97A0969FADA0970F94410520E0FB
:1084A00030E040EC5FE30F94090187FD47CFD7012F
:1084B000C601805A9541AF4FBF4F2D968CAF9DAFEF
:1084C000AEAFBFAF2D9766962FAE669768963FAE5C
:1084D00068976C964FAE6C97A0965FAEA097809110
:1084E0009A02882309F42ACF81149104A104B104CB
:1084F00029F4C12ED02EE72CF62CEDCE98EEC91A19
:1085000093E0D90AE108F108C818D908EA08FB087D
:10851000F7FE14CFEECF0E9444F888E528D78823D1
:1085200019F0179A1092470589E521D7882319F089
:10853000169A109248058AE51AD7882319F0159AD9
:108540001092490585E413D7882309F469CC0E9469
:1085500064E866CC0E9444F80E9467E861CC88E534
:1085600035D7882359F0D0D624E0129FF00111248A
:10857000E35DFA4E608371838283938389E526D716
:10858000882379F000912E0410E0BED6000F111F51
:10859000000F111FF801EB5CFA4E60837183828338
:1085A0009383E4EFF2E284918F010F5F1F4F8823E2
:1085B00021F00E944B72F801F6CFE8EEF4E08491CE
:1085C0008F010F5F1F4F882311F40C9417320E9404
:1085D0004B72F801F4CF67964EAD5FAD67971416F6
:1085E00015060CF042C1E7964CAC5DAC6EAC7FACAE
:1085F000E797480E591E6A1E7B1EE7962CAD3DADCF
:108600004EAD5FADE797281B390B4A0B5B0BCA01D8
:10861000B90161962CAD3DAD4EAD5FAD61970F9444
:10862000D504A30192010F940605820E931EA41E89
:10863000B51E34E183169104A104B1040CF466C1A3
:10864000C158DF4F88819981AA81BB81CF57D04023
:1086500088169906AA06BB060CF04FC1C957DF4F12
:10866000288139814A815B81C758D0402815390556
:108670004A055B059CF4C557DF4F88819981AA8123
:10868000BB81CB58D04088199909AA09BB096196CA
:108690008CAF9DAFAEAFBFAF619706C061968CAE99
:1086A0009DAEAEAEBFAE6197B501A40181E696E086
:1086B0000E9423C161964CAD5DAD6EAD7FAD6197FB
:1086C0008CE596E00E9423C1A4964FADA497A59691
:1086D0005FADA597A6966FADA697A7967FADA79716
:1086E00085E596E00E9406C1A8964FADA897A99689
:1086F0005FADA997AA966FADAA97AB967FADAB97E2
:108700008EE496E00E9406C16796AEADBFAD679756
:1087100013970CF4AAC061966CAD7DAD8EAD9FAD84
:1087200061970F940F0120E030E040E850E40F948F
:108730006E016B017C01A4962FADA497A5963FAD69
:10874000A597A6964FADA697A7965FADA797A896B3
:108750006FADA897A9967FADA997AA968FADAA9756
:10876000AB969FADAB970F9441052BED3FE049E4ED
:1087700050E40F946E0120E030E040E05FE30F949E
:108780006E019B01AC01C701B6010F941E066B017F
:108790007C01C301B2010F940F012FE632E143E8DF
:1087A0005AE30F946E012B013C01B701A60188E446
:1087B00096E00E9406C1B301A20182E496E00E9405
:1087C00006C12AE939E949E15FE3C701B6010F941F
:1087D0006E016B017C019B01AC010F944205A3016A
:1087E00092010F941E066B966CAF7DAF8EAF9FAF5C
:1087F0006B97A3019201C701B6010F946E0120E0AF
:1088000030E040E05EE30F946E016F966CAF7DAF99
:108810008EAF9FAF6F97E2E3F6E084913F01BFEF29
:108820006B1A7B0A882321F00E944B72F301F5CF6B
:10883000B701A6018CE296E00E9406C16B964CAD92
:108840005DAD6EAD7FAD6B9786E296E00E9406C18E
:108850006F964CAD5DAD6EAD7FAD6F9780E296E0EB
:108860000E9406C18AE00E944B7261968CAD9DAD5C
:10887000AEADBFAD6197880D991DAA1DBB1DB59505
:10888000A79597958795EFEF2E163E0619F48093DE
:10889000920E05C0EF96EEADFFADEF978083679621
:1088A0002EAD3FAD67972F5F3F4F67963FAF2EAF1F
:1088B0006797A0963FADA097A4963FAFA497A196C7
:1088C0004FADA197A5964FAFA597A2965FADA29782
:1088D000A6965FAFA697A3968FADA397A7968FAFE7
:1088E000A79765964CAC5DAC6EAC7FAC659791E09C
:1088F000AF969FAFAF970C94783CCD57DF4F8880F1
:108900009980AA80BB80C358D040B5CE84E1882E20
:10891000912CA12CB12C24E130E040E050E0619694
:108920002CAF3DAF4EAF5FAF6197BECECE56DF4F9F
:108930000FB6F894DEBF0FBECDBFDF91CF911F9170
:108940000F91FF90EF90DF90CF90BF90AF909F90EE
:108950008F907F906F905F904F903F902F900895F1
:1089600090915615E92FF0E0EE58F84F80839F5F05
:10897000943018F49093561502C0109256158091B9
:1089800019098F5F809319090895CF92DF92EF92B2
:10899000FF920F931F93CF93DF936C017A018B01AA
:1089A000C0E0D0E0CE15DF0589F0D8016D918D01D2
:1089B000D601ED91FC910190F081E02DC601199551
:1089C000892B11F47E0102C02196ECCFC701DF9103
:1089D000CF911F910F91FF90EF90DF90CF9008956E
:1089E000089580E090E0089580E008950B96FC01E2
:1089F000849108950A96FC0184910895FC01849164
:108A00000895FCDF882321F0823011F083E008957F
:108A100086E00895FC01E60FF11D849190E0982F07
:108A200088273196E4918E0F911D089568E0F2CF6A
:108A300066E0F0CF0895FC01A681B7818281481BD2
:108A40008581483018F0A80FB11D4770382F369532
:108A500036953695562F577080E890E002C0959570
:108A600087955A95E2F7439F402D112466956695A8
:108A70006695E62FF0E0E40FF11DEA0FFB1F308151
:108A8000222311F0832B02C08095832380830895D5
:108A9000FB014181DC0112962C911297421760F084
:108AA00013962C911397241738F0608115962C910A
:108AB000621710F42481BFCF0895FC018081928158
:108AC000980F92832181921760F494819F5F948321
:108AD0009381890F821710F08FEF820F838381E0DB
:108AE000089580E00895FC01128280818150838383
:108AF0001482089581E00895089590E0FC01319773
:108B0000E231F10508F04EC08827EE58FF4F8F4F35
:108B10000D942D08809180008F7703C08091800094
:108B20008F7D80938000089580918000877FF9CFAA
:108B300084B58F7702C084B58F7D84BD0895809100
:108B4000B0008F7703C08091B0008F7D8093B0001C
:108B50000895809190008F7707C0809190008F7D5D
:108B600003C080919000877F80939000089580914A
:108B7000A0008F7707C08091A0008F7D03C08091F7
:108B8000A000877F8093A0000895809120018F77B7
:108B900007C0809120018F7D03C080912001877FD5
:108BA0008093200108953FB7F894809148049091F4
:108BB0004904A0914A04B0914B0426B5A89B05C076
:108BC0002F3F19F00196A11DB11D3FBFBA2FA92F4C
:108BD000982F8827820F911DA11DB11DBC01CD01C9
:108BE00042E0660F771F881F991F4A95D1F70895B5
:108BF000EF92FF920F931F93CF93DF931F92CDB706
:108C0000DEB7082F162FE5EFF6E184917F012FEFF5
:108C1000E21AF20A882331F099830E944B72F7011D
:108C20009981F3CFE02FF92F84917F019FEFE91A0B
:108C3000F90A882321F00E944B72F701F5CF609169
:108C4000C5137091C6138091C7139091C8130E94E9
:108C50000A738AE00E944B7211110E9423EC109259
:108C6000B3041092B2040F90DF91CF911F910F9136
:108C7000FF90EF900895CF93FC0180818B33A1F09A
:108C800080911909843080F4C62FBF018091561558
:108C900020E6829FC00111248856984F0F947C08CB
:108CA0008C2F5EDE81E001C080E0CF910895DF92DD
:108CB000EF92FF920F931F93CF93DF93CDB7DEB761
:108CC0006E970FB6F894DEBF0FBECDBF609156070A
:108CD000709157076115710501F14DE150E0CE012A
:108CE00001967C010F9479001E8EF7018F010E19F9
:108CF0001F09D190DD2019F09AE0D912F7CFF701C2
:108D0000E00FF11F108260E0C701B5DF882329F072
:108D1000C7010E941EE8811109C081E02091560719
:108D200030915707232BA1F480E012C0DD2049F0D9
:108D30000F5F1F4F8091560790915707080F191F1B
:108D400002C000E010E01093570700935607E5CFEC
:108D50006E960FB6F894DEBF0FBECDBFDF91CF91F8
:108D60001F910F91FF90EF90DF9008952F923F9207
:108D70004F925F927F928F929F92AF92BF92CF92CB
:108D8000DF92EF92FF920F931F93CF93DF931F9287
:108D9000CDB7DEB78CDF81115AC2809119098430BA
:108DA00058F42FB7F8948091C8099091C9092FBF42
:108DB000891B8F7709F044C180911F0B882309F428
:108DC00046C280911909811102C01092B604EE24A6
:108DD000E3944091C20D5091C30D6091C40D709108
:108DE000C50D8091BE0D9091BF0DA091C00DB091A9
:108DF000C10D481759076A077B0708F4E12C00E00A
:108E000010E09924939480E6882E92E0C92E98E091
:108E1000D92E2EEFA22E27E0B22E3DE8732E8091A0
:108E20001909843008F013C2E11011C28091B60410
:108E300081110DC28091190D90911A0DA0911B0DF9
:108E4000B0911C0D8093C20D9093C30DA093C40DDF
:108E5000B093C50D41E050E0BE016F5F7F4F81E1EF
:108E60009DE00E94EA8C019719F4898190E002C08C
:108E70008FEF9FEFF82EEE24E3942090C20D3090F8
:108E8000C30D4090C40D5090C50D4091BE0D509142
:108E9000BF0D6091C00D7091C10D241635064606B8
:108EA0005706C8F4E12C8F3FFFEF9F0709F47AC003
:108EB0002AE0821709F495C08DE0F81609F491C0F4
:108EC00093E2F91619F0EAE3FE12A0C08091B5040E
:108ED00081119CC081C0EDE1F8E084912F012FEF5A
:108EE000421A520A882321F00E944B72F201F5CFF8
:108EF0000E9444F881E19DE00E94F18980912C0D4F
:108F0000882359F1815080932C0D789EC001112443
:108F100041E061E08F5C924F0E948E59E0912C0DF0
:108F200084E0E89FF0011124E35DF24F408151811C
:108F3000628173814093C20D5093C30D6093C40D41
:108F40007093C50D81E19DE00E94BA888091200B4D
:108F50008823C1F090921F0B15C010921F0BD09266
:108F60005707C0925607A3DE0E9487BD0E94F4BE39
:108F70006D3371058105910528F0B0925707A092D5
:108F8000560795DE1092CA0D8091200B882319F0A8
:108F90000E940C5C21C00E94BD5C8091200B81115D
:108FA000F7CF1AC0E5EFF6E184912F019FEF491A40
:108FB000590A882321F00E944B72F201F5CFEEE0AE
:108FC000F8E084912F012FEF421A520A882321F0F2
:108FD0000E944B72F201F5CF83E2F81202C0909228
:108FE000B6041092B5040115110509F418CF80914B
:108FF0005615889E000D111D1124F801E856F84FF2
:10900000108280E0ADDC00E010E009CF0F351105E3
:1090100008F005CF9BE3F91202C09092B50480914D
:10902000B5048111FCCE80915615F801889EE00DA3
:10903000F11D1124E856F84FF0820F5F1F4FEFCE5D
:109040000E9495732091B2043091B3048A3019F0D4
:109050008D3009F0CBC01092B4042115310509F40C
:109060009CCEF901EE5AFB4F10821092B30410927D
:10907000B20422E534E08901F90180812F5F3F4F7E
:109080008032C9F378018E3411F000E010E06AE21A
:1090900070E0C7010F9471086C010115110509F406
:1090A00074C069EF77E0C7010F948800BB24B394C4
:1090B000892B11F4B12C09C06EE470E0C70104964D
:1090C0000F947108009709F08C014AE050E060E0CD
:1090D00070E0C80101960E94FDFD60934E047093FC
:1090E0004F0480935004909351040091C513109144
:1090F000C6132091C7133091C8130F5F1F4F2F4F16
:109100003F4F601771078207930731F0B11004C019
:1091100061E086EC97E026C0C114D10401F180E043
:1091200010E0F701E80FF11D90819A3219F08F5F7E
:109130001927F7CF4AE050E060E070E0C6010196E1
:109140000E94FDFD012F10E020E030E06017710764
:109150008207930749F061E087EA97E003C061E086
:109160008DE797E045DD28CE80914E0490914F0425
:10917000A0915004B09151048093C5139093C613ED
:10918000A093C713B093C81306C0892B21F060E0E9
:1091900082ED96E0E7CF80917802811122C067E4EA
:1091A00070E0C7010F9471080097D9F04AE050E0D1
:1091B00060E070E001960E94FDFD6430710588F466
:1091C000E6E0F7E084918F010F5F1F4F882321F0C5
:1091D0000E944B72F801F6CF60E08CEF96E00E949F
:1091E000E1C561E082E594E046DDD7CD2F3531055C
:1091F0000CF0D3CD8C35B1F42FB7F8948091C80919
:109200009091C9092FBF891B8F7709F4C6CD0E94A1
:1092100095739091B4049111C0CD2091B204309116
:10922000B30409C08B3319F491E09093B404909186
:10923000B4049111B2CDA9014F5F5F4F5093B304B5
:109240004093B204F901EE5AFB4F8083A6CD0F90F4
:10925000DF91CF911F910F91FF90EF90DF90CF9012
:10926000BF90AF909F908F907F905F904F903F9076
:109270002F9008952DE235E049E255E065E275E072
:1092800081E295E00C943DE580914C0490914D0471
:10929000009731F04AE050E060E070E00C9425FF68
:1092A00060E070E0CB01089580914C0490914D04F2
:1092B000009731F04AE050E060E070E00C94FDFD72
:1092C00060E070E0CB010895EFDF97FD0AC0ECDFAE
:1092D0006F3F71058105910509F02CF4E5DF862FBC
:1092E000089580E008958FEF089580914C04909147
:1092F0004D04892B31F0E8DF91E0811103C090E04B
:1093000001C091E0892F08950F931F93CF9380910F
:109310004C0490914D040097F1F0FC018F01C19134
:109320002C2F2F7D89F0C53411F0C536B9F7F8011F
:10933000108260E070E00E9496FCF801C083562F16
:10934000472F382F292F0BC060E070E0CF911F917D
:109350000F910C9496FC50E040E030E020E0652F47
:10936000742F832F922FCF911F910F9108958154C5
:109370008A3150F5482F50E0FA0193E0F595E795D2
:109380009A95E1F7E85DFB4F208130E08770B901E5
:1093900002C0759567958A95E2F760FF15C0FA01DE
:1093A000E25FFB4F2081222339F08091E0139091FE
:1093B000E113820F911D02C080E090E090934D0474
:1093C00080934C0481E0089580E00895D0DF8823E5
:1093D00041F081E020914C0430914D04232B09F49D
:1093E00080E00895FC01238121110C94F1890895F6
:1093F000CF93DF939091060A91111CC094E0899F4E
:10940000E0011124C452DB4F60911E0270911F02D3
:10941000072E000C880B990B0F940F019B01AC01D8
:10942000688179818A819B810F940901881F88272F
:10943000881F01C080E0DF91CF9108958091F00AEC
:109440009091F10A891B8F700895CF92DF92FF925D
:109450000F931F93CF93DF931F921F92CDB7DEB769
:109460006901DB0112960D911C911397423309F4A7
:1094700070C0B8F4453109F477C0473109F487C0AA
:10948000443109F09DC0D80115962C911597169678
:10949000ED91FC911797CF01820F911D820F911DC5
:1094A0005CC0463409F483C0473409F484C04B33AC
:1094B00009F086C0F90181819381913029F09330C0
:1094C00031F4482F885004C048E0480F01C0482FAD
:1094D00021E0D80113963C91381708F420E031E0E0
:1094E000F8015281451708F430E051E0481708F0C0
:1094F00050E0822F852B382319F4252309F460C00E
:10950000D6011296FC90913051F030F0923049F033
:10951000933051F42FEF09C020E031E007C021E083
:1095200004C020E03FEF02C020E030E0F7FE07C0BB
:10953000B601C8012A833983ABDA39812A81F60161
:109540008081830F80838181820F8183FF0C71F77B
:1095500037C0B901C8019CDA33C01192E817F90786
:10956000E1F7C801C0DA2CC0C801A7DA882349F1A5
:10957000F80125810680F781E02DCF01820F911D32
:10958000820F911D1192E817F907E1F719C0D9016F
:109590001C92F801828111968C93119785818150DC
:1095A00012968C931297838113968C9309C0D801DD
:1095B00015968C9103C0D80111968C91F601808389
:1095C00081E00F900F90DF91CF911F910F91FF904D
:1095D000DF90CF90089588E290E00197F1F7089529
:1095E0002EE93FE0009729F0F9013197F1F7019753
:1095F000F9CF08950F93FC010150040F84A996A997
:10960000941718F0081728F402C0081750F0041730
:1096100040F42150260F83A995A9961720F4281706
:1096200020F480E007C0281720F481E0261710F00E
:10963000F8CF81E00F910895DB01ED91FC91199431
:109640002F923F925F926F927F928F929F92AF92F2
:10965000BF92CF92DF92EF92FF920F931F93CF931F
:10966000DF931F92CDB7DEB71C01C62E142FD22E6A
:10967000DC011496ED90FC901597C701BFD9082F17
:10968000F10184819581BDD9982E013019F48FE0C4
:10969000A82E02C0AA24AA94D10114968D919C915F
:1096A0001597A8D9082FF101848195819FD9B82EEB
:1096B000D10114968D919C911597B8D9B0E6BD153E
:1096C00030F4009721F0E80EF91E01E610C0F10118
:1096D00084819581ADD9F0E4FD1530F4009721F037
:1096E000E80EF91E01E403C021E1E20EF11CBD14F5
:1096F00080F4D10150961C92509753961C92539728
:1097000054961C92549751961C92519752961C92C3
:10971000C3C0B01670F3892D90E0F70124912F3F5C
:1097200021F4FFEFEF1AFF0A59C00D114EC0D1010D
:1097300014968D919C91159761D997012F5F3F4F9A
:10974000F701882311F08230E1F48491D10153961E
:109750008C935397F901249154962C935497F701C5
:109760003396E4915096EC935097F7013496E49138
:109770005196EC935197F7013596E4915296EC93FC
:1097800020C08491982F9F709250D10152969C9343
:10979000529782958F7051968C935197F90124912D
:1097A000822F8F7054968C93549722952F705396D6
:1097B0002C935397F7013296E491E295EF7050960F
:1097C000EC93E114F10479F467C0F7013296E49167
:1097D000EA219C012E0F311DE20EF31E0B1509F438
:1097E00088CF0F5F9ACFF101848195810AD9B82E75
:1097F000D10153969C9053975496DC905497519670
:109800008C915197C80E52969C919D0D512E591ACC
:109810000D2D292D452D6C2DC101ECDE8823C9F1BC
:10982000C7018B0D911D5C0187E0890DF82EF69420
:10983000F694F694D50C41019CE1890E911C6F2C95
:10984000712C5D1431F15C2D8501802F8A198F15E3
:10985000E0F4F8018491D10112966D917C911397F7
:109860005C965C935C975D965C925D975F961C92AC
:109870005F975E968C9394014BE3C1015983DCDEC4
:109880000F5F1F4F5981585FE0CFA60CB71C539450
:10989000D8CFF101808901C080E00F90DF91CF9196
:1098A0001F910F91FF90EF90DF90CF90BF90AF90FE
:1098B0009F908F907F906F905F903F902F90089532
:1098C0008F929F92BF92CF92DF92EF92FF920F936F
:1098D0001F93CF93DF931F92CDB7DEB74C01062FB6
:1098E000F42E122F522FE62EE20EBB24BA946C01F6
:1098F0008CE1C80ED11C8E2D851B583078F0F401F8
:1099000062817381848FF58E178EB68E96014BE33C
:10991000C401598391DE59815850EDCF812F887F42
:10992000080F212F277019F187E02827F4016281A1
:109930007381048FF58E178E2F5F27708FEF90E065
:1099400001C0880F2A95EAF7868F9401245E3F4F65
:109950004BE3C4010F90DF91CF911F910F91FF90C6
:10996000EF90DF90CF90BF909F908F9065CE0F903B
:10997000DF91CF911F910F91FF90EF90DF90CF90EB
:10998000BF909F908F900895EF92FF920F931F9337
:10999000CF93DF937C01D62F122FC42F040F212FDA
:1099A0004C2F6D2FC7018CDFCF5F0C13F8CFDF91E9
:1099B000CF911F910F91FF90EF900895DF92EF925A
:1099C000FF920F931F93CF93DF93EC01162FF42E8A
:1099D000E22E10DE882329F02E2D4F2D612FCE018F
:1099E000D3DFDF91CF911F910F91FF90EF90DF9028
:1099F0000895EF92FF920F931F93CF93DF931F92DF
:109A0000CDB7DEB78C01DC011296ED90FC90139778
:109A1000D196ED91FC91D29782E0199520E030E04B
:109A20004AE0B701C80108DEF82ED801D196ED91C1
:109A3000FC91D29783E01995D801D196ED91FC91D4
:109A4000D29780E01995FF2081F1F801628173813E
:109A50009E012F5F3F4F46E4C801EEDD8981D801AA
:109A60008C9312966D917C9113979E012F5F3F4FBF
:109A700047E4C801E1DD8981F80181836281738156
:109A800020E030E048E4C801D7DDD8011B968C9374
:109A90001B9798012D5C3F4F12966D917C91139707
:109AA00047E1C801C9DD81E001C080E00F90DF918E
:109AB000CF911F910F91FF90EF9008951F920F92F9
:109AC0000FB60F9211240BB60F922F933F934F9323
:109AD0005F936F937F938F939F93AF93BF93EF9316
:109AE000FF93E0910E02F0910F021995FF91EF9113
:109AF000BF91AF919F918F917F916F915F914F91A6
:109B00003F912F910F900BBE0F900FBE0F901F90A3
:109B100018951F920F920FB60F9211240BB60F9249
:109B20002F933F934F935F936F937F938F939F9365
:109B3000AF93BF93EF93FF93E0910C02F0910D026E
:109B40001995FF91EF91BF91AF919F918F917F9167
:109B50006F915F914F913F912F910F900BBE0F909E
:109B60000FBE0F901F9018951F920F920FB60F9275
:109B700011240BB60F922F933F934F935F936F93E4
:109B80007F938F939F93AF93BF93EF93FF93E09156
:109B90000202F09103021995FF91EF91BF91AF91ED
:109BA0009F918F917F916F915F914F913F912F91F5
:109BB0000F900BBE0F900FBE0F901F9018951F9225
:109BC0000F920FB60F9211240BB60F922F933F9363
:109BD0004F935F936F937F938F939F93AF93BF93B5
:109BE000EF93FF93E0910002F09101021995FF912C
:109BF000EF91BF91AF919F918F917F916F915F9105
:109C00004F913F912F910F900BBE0F900FBE0F9071
:109C10001F9018951F920F920FB60F9211240BB63A
:109C20000F922F933F934F935F936F937F938F93F5
:109C30009F93AF93BF93EF93FF93E0910A02F0914C
:109C40000B021995FF91EF91BF91AF919F918F9169
:109C50007F916F915F914F913F912F910F900BBE2C
:109C60000F900FBE0F901F9018951F920F920FB676
:109C70000F9211240BB60F922F933F934F935F9344
:109C80006F937F938F939F93AF93BF93EF93FF93C4
:109C9000E0910802F09109021995FF91EF91BF91AF
:109CA000AF919F918F917F916F915F914F913F9174
:109CB0002F910F900BBE0F900FBE0F901F90189515
:109CC0001F920F920FB60F9211240BB60F922F9383
:109CD0003F934F935F936F937F938F939F93AF9334
:109CE000BF93EF93FF93E0910602F091070219955D
:109CF000FF91EF91BF91AF919F918F917F916F9164
:109D00005F914F913F912F910F900BBE0F900FBE1F
:109D10000F901F9018951F920F920FB60F9211245B
:109D20000BB60F922F933F934F935F936F937F9355
:109D30008F939F93AF93BF93EF93FF93E0910402B0
:109D4000F09105021995FF91EF91BF91AF919F910D
:109D50008F917F916F915F914F913F912F910F90D4
:109D60000BBE0F900FBE0F901F901895CF93DF93EF
:109D7000282F30E0F901E05CFA4E8491F901E254B9
:109D8000FC4DD491F901E858FC4DC491CC2391F0DD
:109D900081110E947D45EC2FF0E0EE0FFF1FE8548B
:109DA000F94FA591B491EC91ED2381E090E021F47D
:109DB00080E002C080E090E0DF91CF9108951F9392
:109DC000CF93DF93282F30E0F901E05CFA4E8491C5
:109DD000F901E254FC4DD491F901E858FC4DC491CD
:109DE000CC23C9F0162F81110E947D45EC2FF0E0A5
:109DF000EE0FFF1FEC5BFC4DA591B4918FB7F8946B
:109E0000111105C09C91ED2FE095E92302C0EC9162
:109E1000ED2BEC938FBFDF91CF911F9108951F938E
:109E2000CF93DF93182FEB010E9484BB209711F48E
:109E300060E004C0CF3FD10531F461E0812FDF91B4
:109E4000CF911F91BCCFE12FF0E0E05CFA4EE4919E
:109E50004E2F50E0FA013197E231F10508F09DC034
:109E60008827EC57FF4F8F4F0D942D0884B58068DD
:109E700084BDC7BD97C084B5806284BDC8BD92C093
:109E800080918000806880938000D0938900C09387
:109E9000880088C080918000806280938000D09389
:109EA0008B00C0938A007EC0809180008860809380
:109EB0008000D0938D00C0938C0074C08091B0005E
:109EC00080688093B000C093B3006CC08091B000F4
:109ED00080628093B000C093B40064C08091900011
:109EE000806880939000D0939900C09398005AC0E6
:109EF00080919000806280939000D0939B00C093EB
:109F00009A0050C080919000886080939000D09318
:109F10009D00C0939C0046C08091A0008068809303
:109F2000A0008091A0008F7B8093A000D093A90017
:109F3000C093A80037C08091A00080628093A000E9
:109F4000D093AB00C093AA002DC08091A000886080
:109F50008093A000D093AD00C093AC0023C080914B
:109F60002001806880932001D0932901C0932801AB
:109F700019C080912001806280932001D0932B0131
:109F8000C0932A010FC08091200188608093200136
:109F9000D0932D01C0932C0105C0C038D1050CF021
:109FA0004CCF46CFDF91CF911F9108958F929F9212
:109FB000AF92BF92CF92DF92EF92FF926B017C0142
:109FC0000E94D3454B015C01C114D104E104F104AA
:109FD000F1F00E94D345DC01CB0188199909AA0947
:109FE000BB09883E9340A105B10570F321E0C21A78
:109FF000D108E108F10888EE880E83E0981EA11CC4
:10A00000B11CC114D104E104F10419F7DDCFFF90B4
:10A01000EF90DF90CF90BF90AF909F908F9008957A
:10A020002FB7F894609144047091450480914604E0
:10A03000909147042FBF08950F931F93CF93DF9301
:10A04000EC01EEDF0E811F81288539850115110590
:10A050002105310559F52C852223A9F13A85215096
:10A060002C8721E0230F2A874D85241301C01A86EF
:10A07000FE0124E0329FE00DF11D112406851785B5
:10A08000208931890A831B832C833D83DC01CB012A
:10A09000800F911FA11DB11D8E839F83A887B98753
:10A0A0008C819D81892B79F0769A0DC0DC01CB01E2
:10A0B000801B910BA20BB30BB7FD05C076981E82D7
:10A0C0001F8218861986DF91CF911F910F910895F5
:10A0D000A7DF6093E2137093E3138093E4139093EC
:10A0E000E51308951F920F920FB60F9211242F932C
:10A0F0003F938F939F93AF93BF938091440490912C
:10A100004504A0914604B09147043091430423E0F4
:10A11000230F2D3720F40196A11DB11D05C026E89F
:10A12000230F0296A11DB11D209343048093440484
:10A1300090934504A0934604B0934704809148044B
:10A1400090914904A0914A04B0914B040196A11D3D
:10A15000B11D8093480490934904A0934A04B0939E
:10A160004B04BF91AF919F918F913F912F910F9091
:10A170000FBE0F901F9018958091DB048630D8F4A5
:10A1800096E0899FF0011124E954FB4F20911002C1
:10A1900030911102318320834091FC045091FD04E1
:10A1A0006091FE047091FF0442835383648375833E
:10A1B0008F5F8093DB04089520911002309111028B
:10A1C00028173907D9F09093110280931002409319
:10A1D000FC045093FD046093FE047093FF048F5FB2
:10A1E000904521F41092DE0D1092DB0482E0809302
:10A1F000120281E08093ED091092EA0D08954F92CA
:10A200005F926F927F928F929F92AF92BF92CF9206
:10A21000DF92EF92FF920F931F93CF93DF93CDB70F
:10A22000DEB72A970FB6F894DEBF0FBECDBF1092EF
:10A23000E90D8091F00D882349F00E9487EE40E0FF
:10A2400050E0BA018FE498EFB7DFDAC4209124021E
:10A25000309125024091FC045091FD046091FE0470
:10A260007091FF04C901840F951F2436310524F431
:10A27000853691053CF416C02436310531F084361C
:10A28000910584F484E690E00DC04B3051056105E2
:10A29000710514F00A9706C0463F5F4F6F4F7F4F1E
:10A2A0006CF40A9690932502809324021092FC0489
:10A2B0001092FD041092FE041092FF04809124027B
:10A2C000909125028A3091053CF0883E43E0940746
:10A2D0002CF087EE93E002C08AE090E09093250294
:10A2E000809324020E94E9C8F82E0E9464C58091E0
:10A2F000C60A853198F4FF2049F08091110A9091A7
:10A30000120A892B19F003E214E102C006E013E1FE
:10A3100023E14FE061E089E00E94DDBB8091C60A45
:10A320008D3108F098C1A7E18A2EAAE09A2EBAE8EA
:10A33000CB2EBAE0DB2E1CEDA12E14E0B12E1DE0D9
:10A3400002E1602E712C87E0E82E9CE1592E442416
:10A35000439408EF010F8091C60A8830D8F5F601C2
:10A360008081F11002C0811135C0F40160817181DA
:10A37000072E000C880B990B0F940F0120E030E0A2
:10A3800040E05FE30F9442050F9486066436710542
:10A390002CF46A30710524F426E003C022E101C0E8
:10A3A0002CE0A301421B51099A0157FF02C02F5F05
:10A3B0003F4F35952795502F521B5093C90AE09275
:10A3C000CA0ACB010E9412C40E94FBEE83E093E113
:10A3D0000E94EEEE8091C60A8D3198F58091C80AF0
:10A3E000853178F120E030E040E05FE3F501608105
:10A3F0007181828193810F9442050F9486069B019F
:10A40000643671050CF0F7C22A3031050CF0F1C248
:10A4100026E0F301E21BF1099F01F7FF02C02F5F65
:10A420003F4F35952795021B0093C90A5092CA0ADF
:10A43000CB010E9412C40E94FBEE83E093E10E94D4
:10A44000EEEE8091C60A853110F58091C80A8131FF
:10A45000F0F0F40160817181072E000C880B990BDC
:10A460000F940F01F50120813181428153810F94B6
:10A47000680718160CF0C1C21092B20A02E022E07E
:10A4800041E1612F82E99AE099DA4092B20A175EBF
:10A49000F2E08F0E911C2FEFC21AD20A44E0A40EF4
:10A4A000B11C1F3309F055CF8091C60A883008F0DF
:10A4B0003FC080917D0AF11002C0811139C06091C6
:10A4C000150A7091160A072E000C880B990B0F9431
:10A4D0000F0120E030E040E05FE30F9442050F946D
:10A4E0008606643671052CF46A30710524F446E062
:10A4F00003C042E101C04CE022E130E0241B3109FD
:10A5000037FF02C02F5F3F4F359527953195219535
:10A5100031092F5A2093C90A27E02093CA0ACB0198
:10A520000E9412C40E94FBEE83E093E10E94EEEED3
:10A530008091C60A8D31D0F58091C80A8531B0F17D
:10A5400020E030E040E05FE36091E4047091E504D6
:10A550008091E6049091E7040F9442050F948606DB
:10A560009B01643671050CF053C22A3031050CF0A2
:10A570004DC246E022E130E0241B310937FF02C022
:10A580002F5F3F4F359527953195219531092F5AEA
:10A590002093C90A2CE12093CA0ACB010E9412C45D
:10A5A0000E94FBEE83E093E10E94EEEE8091C60AEA
:10A5B000853138F58091C80A813118F16091150A0A
:10A5C0007091160A072E000C880B990B0F940F013F
:10A5D0002091E4043091E5044091E6045091E704B1
:10A5E0000F94680718160CF015C21092B20A02E018
:10A5F00022E042E168E582E99AE0E0D981E08093D7
:10A60000B20A8091C60A8C3130F58091C80A843133
:10A6100010F18091110A9091120A019644E6489F28
:10A620009001499F300D112437FF02C021503F4F48
:10A63000832F932F990F990B009769F028E62093A9
:10A64000C90A2BE12093CA0A0E9412C40E94FBEEA1
:10A6500085E20E94DFBC8091C60A843328F4809191
:10A66000C80A8A3208F0DFC18091C60A853328F40F
:10A670008091C80A813308F0FCC180911F0B8823A8
:10A6800009F44AC08091C60A843308F045C080911D
:10A69000C80A823308F440C02091140D222319F116
:10A6A0008091BE0D9091BF0DA091C00DB091C10DD4
:10A6B0000097A105B10509F4E1C1BC01CD016D59B7
:10A6C0007F4F8F4F9F4F24E630E040E050E00F94E3
:10A6D000E4046091C20D7091C30D8091C40D9091FE
:10A6E000C50D0F94E40458E4259FB0011124072EF2
:10A6F000000C880B990B0F940F012AE037ED43E211
:10A700005CE30F946E010F948B06262F02E042E368
:10A7100067E382E99AE052D98091C60A813308F052
:10A7200060C08091C80A893208F45BC00E94F4BE00
:10A730002B013C018CE3882E912CA12CB12CC30160
:10A74000B201A50194010F94E404CA01B901A50165
:10A7500094010F94E404CA01E62ED72E59018E010C
:10A760000F5F1F4FF1E84F16F1E55F06F1E06F064E
:10A77000710408F485C1B90128E130E040E050E0FF
:10A780000F94E40429013A01DF92EF92C50168E1D8
:10A7900070E00F9406089F938F935F924F9283E42B
:10A7A00098E09F938F931F930F930F94A2000FB67F
:10A7B000F894DEBF0FBECDBF9AE049165104610484
:10A7C000710408F08CC197E0892F880F980F91953C
:10A7D000955A9093C90A80E38093CA0AC8010E94DF
:10A7E000FBEEE0918C0AF0918D0A84818111CEC03C
:10A7F0006091210570912205809123059091240597
:10A800000F948606CB010E94ABC3BC0187EF94E096
:10A810000F947C086091250570912605809127058D
:10A82000909128050F948606CB010E94ABC3BC0112
:10A8300082EF94E00F947C082CEA35EC47E257E372
:10A840006091290570912A0580912B0590912C0526
:10A850000F94420520E030E048EC52E40F946E0182
:10A860000F9486064B015C0197FD19C090E1891693
:10A8700097E29906A104B104E4F0C501B40120E116
:10A8800037E240E050E00F940605CA01B9012AE022
:10A8900030E040E050E00F940605605D0BC0B094DE
:10A8A000A09490948094811C911CA11CB11C6DE219
:10A8B00001C060E26093010EE8EE8E16E3E09E06B2
:10A8C000A104B10494F0C501B40128EE33E040E0E6
:10A8D00050E00F940605CA01B9012AE030E040E0DB
:10A8E00050E00F940605605D01C060E26093020EC7
:10A8F000C501B40124E630E040E050E00F940605C5
:10A900009AE0492E512C612C712CCA01B901A30186
:10A9100092010F940605605D6093030EC501B401BA
:10A92000A30192010F9406054B015C01672B682B74
:10A93000692B79F08EE28093040ECA01B901A3015C
:10A9400092010F940605605D6093050E80E3880D0B
:10A9500015C0CA01B901A30192010F94060566232F
:10A9600039F08EE28093040E605D6093050E05C0A1
:10A9700080E28093050E8093040E80E28093060EA1
:10A9800061E07EE08BEE94E00F947C088091C60A33
:10A990008632A0F48091C80A8E3180F008E020E869
:10A9A0004EE160E082E99AE009D88091C60A8632D9
:10A9B00028F48091C80A8F3108F093C08091C60AAC
:10A9C000823328F48091C80A8C3208F0FAC0809152
:10A9D000C60A8F3308F014C18091C80A883308F47E
:10A9E0000FC11092C90A8EE38093CA0A0E949CBDCF
:10A9F00007C12CE00ECD22E10CCD02E022E041E1C6
:10AA0000612F82E99AE00E94DE4C41CD4CE0B2CD4C
:10AA100042E1B0CD02E022E042E168E582E99AE05D
:10AA20000E94DE4CEECD07E028E04AE26AE282E9CD
:10AA30009AE00E94DE4C05E022E04CE262E382E90B
:10AA40009AE00E94DE4C6AE08AE20E9433BC609188
:10AA5000940A7091950A82E38093AE0A8BE2809308
:10AA6000AF0A2EEA3AE042E382E99AE00E941C4BE8
:10AA7000FBCD6AE486E30E9433BCFFCD20E033CEF9
:10AA8000E4E6AE16B104C0F4DF92EF92C50168E1CE
:10AA900070E00F9406089F938F9389E398E09F934B
:10AAA0008F931F930F930F94A2000FB6F894DEBFFD
:10AAB0000FBECDBF95E088CEDF92EF923F932F93EC
:10AAC00081E398E09F938F931F930F930F94A200BD
:10AAD0000FB6F894DEBF0FBECDBF96E075CE98E0FE
:10AAE00073CE1092B20A83E08093C90A85E2809304
:10AAF000CA0AFF2029F081E093E10E94EEEE0DC02A
:10AB00008091E804811102C08FE305C08091470560
:10AB10008111F1CF80E20E94DFBC8BE08093C90AF3
:10AB200015E21093CA0A87EF94E00E94FBEE8BE2D5
:10AB30008093C90A1093CA0AFF2029F08FEF92E18F
:10AB40000E94EEEE0DC08091E904811102C08FE3F6
:10AB500005C0809148058111F1CF80E20E94DFBCE1
:10AB600083E38093C90A15E21093CA0A82EF94E046
:10AB70000E94FBEE83E58093C90A1093CA0AFF2066
:10AB800029F08DEF92E10E94EEEE0DC08091EA0473
:10AB9000811102C08FE305C0809149058111F1CF79
:10ABA00080E20E94DFBC8BE58093C90A85E2809336
:10ABB000CA0A8BEE94E00E94FBEE81E08093B20A19
:10ABC000FDCE84E00E94A9EE83E08093C90A12E3DF
:10ABD0001093CA0A86E00E94DAEE0E9464C58CE0F7
:10ABE0008093C90A1093CA0A809124029091250289
:10ABF0000E9412C40E94FBEE85E20E94DFBCE7CEF9
:10AC00002A960FB6F894DEBF0FBECDBFDF91CF916D
:10AC10001F910F91FF90EF90DF90CF90BF90AF907A
:10AC20009F908F907F906F905F904F90089540E03D
:10AC300050E0BA018FEF90E5BFCAE091DB04EE234C
:10AC400081F0E150E093DB0486E0E89FF0011124FD
:10AC5000E954FB4F428153816481758180819181E8
:10AC6000ABCAE5CFAF92BF92CF92DF92EF92FF9245
:10AC70000F931F93CF93DF935C017B0120E030E0C3
:10AC8000F501E20FF31FE491EE2319F02F5F3F4F20
:10AC9000F7CFF701CF018E199F0941914111FACFEA
:10ACA00004E110E0081B11093327021713071CF0F9
:10ACB000DD24D39402C082E0D82E8091930A90E0E4
:10ACC0006D2D70E06F5F7F4F0F941A08C62EC6E09F
:10ACD000C60F8091C60AC81750F08091C80A90E04C
:10ACE0002C2F30E02B503109821793079CF5D0E0D0
:10ACF000E114F104C1F18AE30E94DFBC82E0D812C2
:10AD00000FC0CC0D8091C60AC81768F12091C80AFF
:10AD100030E08C2F90E00B97281739071CF423C0E4
:10AD2000DD2309F1802F880F080F000F0093C90A57
:10AD3000C093CA0A80E20E94DFBCC701DF91CF91B5
:10AD40001F910F91FF90EF90DF90CF90BF90AF9049
:10AD50000C94FBEE1092C90AC093CA0AC5010E9466
:10AD6000EEEED1E0C5CFDF91CF911F910F91FF9013
:10AD7000EF90DF90CF90BF90AF9008950F934CE08D
:10AD8000849F402D112421E0240F20930F058CE097
:10AD9000840F80931005E091C60AF0E090E00296DF
:10ADA0008E179F070CF1822F90E02091C80A30E0A7
:10ADB00082179307CCF4662371F081E08093B20A86
:10ADC0004D5F0BE020E860E082E99AE00E94DE4CF3
:10ADD0001092B20A03C081E08093B20A80911005FC
:10ADE0001092C90A8093CA0A0F910895CF92DF92F8
:10ADF000EF92FF920F93CF93DF93982F862F6A01E4
:10AE00007901692FBBDF9091C60A809110058917DF
:10AE100008F453C09091C80A80910F05981708F460
:10AE20004CC0002359F060E070E0F701E60FF71F17
:10AE3000E491EE2351F06F5F7F4FF7CFD701BD0153
:10AE40006E197F098D918111FACFC62FD4E1D61BDF
:10AE5000F6018491882339F00E94C3EED81BFFEFDE
:10AE6000CF1ADF0AF5CF8AE30E94DFBCDD2329F089
:10AE700080E20E94DFBCD150F9CF809110056AEFCB
:10AE8000C69F602D112460586093C90A8093CA0A36
:10AE9000C701002349F0DF91CF910F91FF90EF9010
:10AEA000DF90CF900C94EEEEDF91CF910F91FF9059
:10AEB000EF90DF90CF900C94FBEEDF91CF910F914C
:10AEC000FF90EF90DF90CF9008950F93CF93DF9393
:10AED000CDB7DEB7ED85FE8560817181828193817A
:10AEE0000F948606CB010E9412C400E09C014985A4
:10AEF0005A8568858F817ADFDF91CF910F91089510
:10AF00009CE0899F802D112421E0280F20930F05BC
:10AF1000845F809310056091C60A70E0482F50E06E
:10AF20004E5F5F4F461757070CF445C030E0409125
:10AF3000C80A50E024173507F4F59EE39093C90A38
:10AF40008093CA0A85E40E94DAEE809146058F5C00
:10AF50000E94DAEE80E20E94DAEEE091460584E09B
:10AF6000E89FF0011124E452FB4F608171818281DE
:10AF700093810F948606CB010E9412C40E94FBEEBF
:10AF80008FE20E94DAEE0E94E9C8E0914605811145
:10AF900007C0AE2FB0E0A657B54F8C9181110BC002
:10AFA000F0E0EE0FFF1FE95EF54F808191810E9476
:10AFB00012C40C94FBEE08954F925F926F927F92B1
:10AFC0008F929F92AF92BF92FF920F931F93CF9356
:10AFD000DF93182F8AEE9CE09093550780935407D7
:10AFE0001092060D82E090E0A0E0B0E08093EF0CBC
:10AFF0009093F00CA093F10CB093F20C10925307C5
:10B0000010924F071092500710925107109252075A
:10B010008FEF9FEFDC0180934B0790934C07A09339
:10B020004D07B0934E07112379F1153008F0F9C0A0
:10B0300040E060E070E0CB010E944FB0882309F44B
:10B04000F0C020E1129FC0011124855C9A4FFC01E1
:10B05000E254FE4F20812F7709F0E3C03C964081F7
:10B06000518162817381443651056105710508F48F
:10B07000D8C0349780809180A280B38081149104DD
:10B08000A104B10421F4CDC0812C912C540140E0E5
:10B09000C501B4010E944FB0F82E882309F4C1C045
:10B0A00080915605909157058115924009F0B9C0DD
:10B0B000A0915B05AA2309F4B4C060915905709171
:10B0C0005A056115710509F4ACC020915805222379
:10B0D00009F4A7C0A093010D2093F30C80E030E0A9
:10B0E000E1E0F0E0C82FAF01082E02C0440F551F69
:10B0F0000A94E2F72417350741F0982F8F5F9830B4
:10B1000089F789E08093FC0C8CC08093FC0C209123
:10B110006105309162052115310519F040E050E0DC
:10B1200008C020916F0530917005409171055091D4
:10B1300072052093F40C3093F50C4093F60C509369
:10B14000F70C24013501460E571E611C711C4092FC
:10B15000020D5092030D6092040D7092050DE09166
:10B160005C05F0915D05F093080DE093070DB0E0EC
:10B170000F942205460E571E681E791E4092090D37
:10B1800050920A0D60920B0D70920C0D85E0EE0F3F
:10B19000FF1F8A95E1F7E150FE4FEF2FFF27E6955D
:10B1A0004E0E5F1E611C711C4092FD0C5092FE0CF5
:10B1B0006092FF0C7092000D20915E0530915F054A
:10B1C0002115310521F0890120E030E008C000910F
:10B1D0006B0510916C0520916D0530916E05B501E0
:10B1E000A4014419550966097709400F511F621FD0
:10B1F000731F04C07695679557954795CA95D2F702
:10B200004093F80C5093F90C6093FA0C7093FB0C7C
:10B21000453F2FE052076105710528F48CE08093CB
:10B22000060DF12C1AC0453F5F4F6105710510F402
:10B2300080E111C08091770590917805A091790502
:10B24000B0917A058093090D90930A0DA0930B0D90
:10B25000B0930C0D80E28093060D8F2DDF91CF917E
:10B260001F910F91FF90BF90AF909F908F907F9014
:10B270006F905F904F900895EF92FF920F931F93FE
:10B28000CF93DF93CDB7DEB76F970FB6F894DEBFDD
:10B290000FBECDBF7B0102E91BE024E93BE0F801D2
:10B2A0003183208322E02093CB0D9093CD0D8093AA
:10B2B000CC0D40E050E0BA0188E99BE00E94BA88DA
:10B2C000F801808191812BE1FC013496DE01159615
:10B2D00001900D922A95E1F7FC01828193819C8374
:10B2E0008B8384E993E09A838983A701BE016F5F12
:10B2F0007F4F89EC93E00E9428BFCE0101960E9407
:10B300005CE86F960FB6F894DEBF0FBECDBFDF913D
:10B31000CF911F910F91FF90EF9008956F927F92C0
:10B320008F929F92AF92BF92DF92EF92FF920F9314
:10B330001F93CF93DF93CDB7DEB7AD970FB6F894D9
:10B34000DEBF0FBECDBF2091200B222309F4F0C138
:10B35000D62E7C018091140D882309F49FC04423CC
:10B3600009F4BBC180912C0D882329F1E5EFF6E1AA
:10B3700084918F010F5F1F4F882321F00E944B7231
:10B38000F801F6CFE2EBF6E184918F010F5F1F4FDA
:10B39000882321F00E944B72F801F6CF61E070E043
:10B3A00080E090E00E940A738AE00E944B7289EA72
:10B3B00096E10E9470E88FE28093310DB12C21E07C
:10B3C00002E31DE09FE1A92E8091E90CB816B8F4C4
:10B3D000AB9CC0011124B8018954944F2DA70E9441
:10B3E000F989C8012DA58C010196F801308133231C
:10B3F00021F02D3811F02F5FF6CFB394E5CF27FD64
:10B4000008C0B80181E19DE00E94F989E4EFF2E211
:10B4100003C0F8011082FACF84918F010F5F1F4F94
:10B42000882321F00E944B72F801F6CFB70180E922
:10B4300096E10E9463C160912C0DFDE86F9FB00101
:10B4400011246F5C724F85E896E10E9463C14091C0
:10B45000C20D5091C30D6091C40D7091C50D8FE761
:10B4600096E10E94F2658AE00E944B7280912C0D59
:10B4700094E0899FF0011124E35DF24F4091C20DE9
:10B480005091C30D6091C40D7091C50D40835183DF
:10B49000628373838F5F80932C0D0DC010922C0DEF
:10B4A00082E0B82E1CC1B70182E796E10E9463C119
:10B4B0008AE00E944B720E947CBD1D8218861C820D
:10B4C0001B8284E993E09A83898383E79BE09093CE
:10B4D000930B8093920BF70180818F3209F067C044
:10B4E00087010F5F1F4FCE0101963C010115110529
:10B4F00009F463C06FE270E0C8010F9471085C0149
:10B50000009709F45BC00817190708F057C04C01F1
:10B51000801A910AA401B801CE0180960F94910877
:10B52000E0E2F0E0EC0FFD1FE80DF91D1082FE01D6
:10B53000B0964F018F01F80181918F01882319F096
:10B540000E944B72F8CF8AE00E944B726091920B7E
:10B550007091930B6115710511F06C5F7F4F21E0C5
:10B56000AE01405E5F4FCE0105960E94F58F8111BE
:10B5700016C0EEE5F6E184918F010F5F1F4F88231F
:10B5800021F00E944B72F801F6CFF40181914F0136
:10B59000882319F00E944B72F8CF8EE287C0709218
:10B5A000930B6092920B85010F5F1F4F9FCF84E931
:10B5B0009BE09093930B8093920B87019091920B59
:10B5C0008091930B692F782FDD2009F459C0611504
:10B5D000710511F06C5F7F4F21E0A80181E19DE0D2
:10B5E0000E94F58F882309F447C08091220D909125
:10B5F000230DA091240DB091250D8093BE0D909345
:10B60000BF0DA093C00DB093C10DB80180E596E1C8
:10B610000E9463C14091BE0D5091BF0D6091C00D5D
:10B620007091C10D88E496E10E94F2658AE00E9463
:10B630004B721092C20D1092C30D1092C40D109255
:10B64000C50DE9E3F6E184917F019FEFE91AF90A5C
:10B65000882321F00E944B72F701F5CFB80180E0FA
:10B6600090E00ADE80912F0B882319F08FE29BE097
:10B6700001C0C80160E02AC0B80185E296E110C0AF
:10B680006115710511F06C5F7F4F26E5A80181E11E
:10B690009DE00E94F58F81110CC0B80181E196E117
:10B6A0000E9463C18EE20E944B728AE00E944B723C
:10B6B0000FC081E080931D0BB7018FEF95E10E94D1
:10B6C00063C18AE00E944B7260E0C8010E94FFC51E
:10B6D000CE0101960E945CE82BC0BB24B394E4EF3A
:10B6E000F2E284918F010F5F1F4F882321F00E94A7
:10B6F0004B72F801F6CFEAE7F6E184918F010F5F14
:10B700001F4F882321F00E944B72F801F6CFE1E031
:10B71000BE1619F002E513E002C008E513E0F801D7
:10B7200081918F01882309F4BECE0E944B72F7CF1E
:10B73000AD960FB6F894DEBF0FBECDBFDF91CF91AF
:10B740001F910F91FF90EF90DF90BF90AF909F906F
:10B750008F907F906F900895CF92DF92EF92FF923B
:10B760000F931F93CF93DF93CDB7DEB7EDB6FEB641
:10B77000DC010D900020E9F79D01281B390B2C5F9F
:10B780003F4F4DB75EB7421B530B0FB6F8945EBFE9
:10B790000FBE4DBF0DB71EB70F5F1F4F9F938F9307
:10B7A00088EF95E19F938F931F930F930F94A200BF
:10B7B000680154E0C50ED11C0F900F900F900F90B0
:10B7C0000F900F90F6018081882339F090E00F945C
:10B7D0003508F60181936F01F5CF60E0C8010E9442
:10B7E0003B46882319F0C8010E941EE884EF95E1CA
:10B7F00090935707809356070E9457460FB6F894C8
:10B80000FEBE0FBEEDBEDF91CF911F910F91FF9055
:10B81000EF90DF90CF900895AF92BF92CF92DF92DA
:10B82000EF92FF920F931F93CF93DF93CDB7DEB7C5
:10B83000AA970FB6F894DEBF0FBECDBF8091720BF2
:10B840008F938091710B8F938BEE95E19F938F93E4
:10B850007E0181E2E80EF11CFF92EF920F94A200AC
:10B860000F900F900F900F900F900F9010E0F70136
:10B8700001900020E9F73197EE19FF091E1774F4C3
:10B880006701C10ED11C17FDDA94F601808190E0AA
:10B890000F943508F60180831F5FE9CF40E050E048
:10B8A000BA0187E79BE00E94BA8800E0CE010196CA
:10B8B0006C0180917A0B823028F4011114C08FEF53
:10B8C0009FEF16C080917F0B9091800BA091810B10
:10B8D000B091820B8F719927AA27BB27892B8A2BBE
:10B8E0008B2B59F71AC08091710B9091720B0196B6
:10B8F0009093720B8093710BAA960FB6F894DEBFEB
:10B900000FBECDBFDF91CF911F910F91FF90EF90B0
:10B91000DF90CF90BF90AF90089540E050E0B60127
:10B9200087E79BE00E94FFB118163CF6F6010190F4
:10B930000020E9F731971E2F1C19115068F05601AD
:10B94000A10EB11C17FDBA94F501808190E00F940F
:10B950003508F5018083F1CF8A858E3709F4A9CFA8
:10B9600045E050E0B701C6010F948308892B09F028
:10B97000A0CFC701F1DE01E09CCFCF92DF92EF9222
:10B98000FF921F93CF93DF931092200B80917A0B3D
:10B99000882321F087E79BE00E94F1891092EE0C4A
:10B9A0001092EB0C85E38093EA0C0E941050EB019F
:10B9B000A8958091EA0C0E9484BB8AEE9CE00E94CC
:10B9C0002C8A2398229A219A209A289A85E080939B
:10B9D000EC0C82E58CBD1DBC1AE08FEF0E94318A11
:10B9E0001150D9F720E030E0A90160E08AEE9CE038
:10B9F0000E94368A182F8093ED0C813049F00E9406
:10BA000010506C1B7D0B613D774060F381E054C0AA
:10BA10002AEA31E040E050E068E08AEE9CE00E94D3
:10BA2000368A82FF03C01093EE0C0EC014E00E9411
:10BA300044728093ED0C1150D1F78A3A11F082E0F4
:10BA40003BC082E08093EE0C8091EE0C823021F0BE
:10BA5000C12CD12C760105C0C12CD12CE12C80E465
:10BA6000F82E20E030E0A90167E38AEE9CE00E9416
:10BA7000368AA701960169E28AEE9CE00E94368A26
:10BA80008093ED0C882349F00E9410506C1B7D0BB5
:10BA9000613D774030F38AE00FC08091EE0C823038
:10BAA00011F520E030E0A9016AE38AEE9CE00E94F3
:10BAB000368A882351F088E08093EB0C8AEE9CE074
:10BAC0000E942C8AE4EFF2E219C00E944472807C4A
:10BAD000803C19F483E08093EE0C0E9444720E9433
:10BAE00044720E9444728AEE9CE00E942C8A10925A
:10BAF000EC0C81E061DA811131C015C08491EF0155
:10BB00002196882321F00E944B72FE01F7CFEDEDC4
:10BB1000F5E18491EF012196882309F456C00E9433
:10BB20004B72FE01F6CF80E047DA811117C0E5EFD6
:10BB3000F6E18491EF012196882321F00E944B7257
:10BB4000FE01F7CFE9ECF5E18491EF01219688231E
:10BB500009F43BC00E944B72FE01F6CF6FEE7CE011
:10BB600087E79BE00E945089811116C0E5EFF6E15E
:10BB70008491EF012196882321F00E944B72FE01EF
:10BB8000F7CFE8EBF5E18491EF0121968823E9F006
:10BB90000E944B72FE01F7CF81E08093200BE4EF0F
:10BBA000F2E28491EF012196882321F00E944B72EA
:10BBB000FE01F7CFECEAF5E18491EF0121968823AD
:10BBC00021F00E944B72FE01F7CF8BE1E7E7FBE02B
:10BBD000A8E9BBE001900D928A95E1F78091750B81
:10BBE0009091760B9093970B8093960B83E79BE055
:10BBF0009093930B8093920BDF91CF911F91FF90C5
:10BC0000EF90DF90CF9008950F931F93CF93DF9322
:10BC10008C01EB019091FE0A2091FF0A921307C05C
:10BC200082EF9AE00E941C500E94F7D1F3CFF801F6
:10BC3000A081B181488159818091FD0A34E0839FC0
:10BC4000F0011124EA50F54FB387A2875587448746
:10BC50009F5F9093FE0A8F5F821719F08093FD0A11
:10BC600002C01092FD0ADF91CF911F910F910895AC
:10BC7000CF93DF93CDB7DEB780914A05811110C015
:10BC80009E01275F3F4F4F81588562E470E083E358
:10BC900092E00F94D1000E94C3C583E0809312020A
:10BCA000DF91CF9108958091100B8130A1F1823006
:10BCB00059F40E94F4BE6093110B7093120B8093A1
:10BCC000130B9093140B18C01092150B1092160BB7
:10BCD0001092170B1092180B1092190B10921A0B4E
:10BCE00010921B0B10921C0B1092110B1092120B46
:10BCF0001092130B1092140B81E08093100B0E9492
:10BD000010506093150B7093160B8093170B909344
:10BD1000180B81E0089580E00895EF92FF921F9341
:10BD2000CF93DF93D091470581E0D8271091480544
:10BD30001827C0914905C827D11102C0112319F055
:10BD4000E4EFF2E203C0C111FBCF7DC084917F011B
:10BD50009FEFE91AF90A882321F00E944B72F7013C
:10BD6000F5CFE6EAF5E184917F019FEFE91AF90A40
:10BD7000882321F00E944B72F701F5CFDD2369F093
:10BD8000E4EAF5E184917F019FEFE91AF90A88233B
:10BD900021F00E944B72F701F5CF112369F0E2EA1E
:10BDA000F5E184917F019FEFE91AF90A882321F0D8
:10BDB0000E944B72F701F5CFC11103C0E8E9F5E12C
:10BDC0000DC0E0EAF5E184917F019FEFE91AF90ADD
:10BDD0008823A1F30E944B72F701F5CF84917F0174
:10BDE0009FEFE91AF90A882321F00E944B72F701AC
:10BDF000F5CFC11103C049EC53E002C04EE553E05A
:10BE0000111103C029EC33E002C020E633E0D11168
:10BE100003C089EC93E002C082E693E05F934F9306
:10BE20003F932F939F938F9386E895E19F938F93F2
:10BE30001F921EDF8DB79EB709960FB6F8949EBF6E
:10BE40000FBE8DBFC1E08C2FDF91CF911F91FF906E
:10BE5000EF900895CF92DF92EF92FF92E091460526
:10BE6000E0934505C0902D05D0902E05E0902F055C
:10BE7000F0903005ED5F84E0E89FF0011124EF5C65
:10BE8000FA4F2081318142815381C701B6010F945D
:10BE90006E010F9473076093EC0A7093ED0A809320
:10BEA000EE0A9093EF0AC701B6010F9486062FB7EA
:10BEB000F89460931D0570931E0580931F05909361
:10BEC00020052FBF1092DC0A1092DD0A1092DE0AC4
:10BED0001092DF0AFF90EF90DF90CF90089580914D
:10BEE000100B813079F482E08093100B0E94105087
:10BEF0006093190B70931A0B80931B0B90931C0B80
:10BF000081E0089580E00895E82FF0E0E05CFA4ECB
:10BF1000E4918E2F90E0FC013797EC30F10508F5A5
:10BF20008827EA56FF4F8F4F0D942D088091B1005E
:10BF3000887F84608093B100089580919100887F0C
:10BF400084608093910008958091A100887F84602F
:10BF50008093A100089580912101887F846080935F
:10BF600021010895FC01DB018C912081318138276A
:10BF700098E0A901440F551F37FD06C09A01915062
:10BF8000C1F73183208308959A01B1E22B27B0E1F4
:10BF90003B27F5CFBC0180E090E04AE00E94A4720C
:10BFA0008DE00E944B728AE00C944B72EF92FF92EC
:10BFB0000F931F93CF93DF931F92CDB7DEB78B0103
:10BFC000622F49830E94BE569091C60A8091100547
:10BFD0004981891708F43FC09091C80A80910F05E4
:10BFE000981708F438C0442399F120E030E0F801B4
:10BFF000E20FF31FE491EE2319F02F5F3F4FF7CFCD
:10C0000086E190E0821B930B97FD019695958795AD
:10C0100036E1F32E49EEE42EE80E8E2D8F0D87FDCE
:10C020000EC080E20E94DFBCFA94F7CFF801849141
:10C03000882339F00E94C3EEF81A0F5F1F4F1F14B8
:10C04000ACF31F1444F480E20E94DFBCFA94F9CFF1
:10C0500086E1F82EF4CF0F90DF91CF911F910F91D1
:10C06000FF90EF900895CF92DF92EF92FF920F939F
:10C070001F93CF93DF937C018B016A01E9010E943A
:10C08000BC5083E080931202F0920B05E0920A0507
:10C0900010930905009308051092040510920505F8
:10C0A0001092060510920705A601DD0C660B770BB2
:10C0B00040930005509301056093020570930305BA
:10C0C000F80180819181092E000CAA0BBB0B809393
:10C0D000FC049093FD04A093FE04B093FF0484E657
:10C0E0009BE79093110280931002D0930E05C093AA
:10C0F0000D0510920C05DF91CF911F910F91FF90CC
:10C10000EF90DF90CF900895CF93DF931F92CDB73C
:10C11000DEB7789484B5826084BD84B5816084BDC7
:10C1200085B5826085BD85B5816085BD80916E00D5
:10C13000816080936E001092810080918100826006
:10C140008093810080918100816080938100809143
:10C1500080008160809380008091B1008460809332
:10C16000B1008091B00081608093B0008091910017
:10C170008260809391008091910081608093910012
:10C18000809190008160809390008091A1008260F6
:10C190008093A1008091A10081608093A100809193
:10C1A000A00081608093A000809121018260809333
:10C1B00021018091210181608093210180912001E2
:10C1C00081608093200180917A00846080937A005E
:10C1D00080917A00826080937A0080917A008160F9
:10C1E00080937A0080917A00806880937A00109220
:10C1F000C1006F98779A82E08093C0001092C500CA
:10C2000087E08093C4008091C10080618093C10069
:10C210008091C10088608093C1008091C1008068D6
:10C220008093C1008091C1008F7D8093C1001092E6
:10C230005807E7E7F8E184918F010F5F1F4F8823CC
:10C2400021F00E944B72F801F6CFE4EFF2E2849104
:10C250008F010F5F1F4F882321F00E944B72F8015E
:10C26000F6CF14B710FF0DC0EEE6F8E184917F0120
:10C270009FEFE91AF90A882321F00E944B72F70117
:10C28000F5CF11FF0DC0EDE5F8E184917F019FEF3F
:10C29000E91AF90A882321F00E944B72F701F5CFC1
:10C2A00012FF0DC0EBE4F8E184917F019FEFE91AE2
:10C2B000F90A882321F00E944B72F701F5CF13FF92
:10C2C0000DC0EAE3F8E184917F019FEFE91AF90AD2
:10C2D000882321F00E944B72F701F5CF15FF0CC0A7
:10C2E000E9E2F8E184918F010F5F1F4F882321F06D
:10C2F0000E944B72F801F6CF14BEE2E2F8E184919D
:10C300008F010F5F1F4F882321F00E944B72F801AD
:10C31000F6CF80E20E944B72EBE1F8E184918F014D
:10C320000F5F1F4F882321F00E944B72F801F6CF58
:10C330008AE00E944B72E4EFF2E284918F010F5F7A
:10C340001F4F882321F00E944B72F801F6CFEBE0DB
:10C35000F8E184918F010F5F1F4F882321F00E9425
:10C360004B72F801F6CFE7EFF7E184918F010F5F91
:10C370001F4F882321F00E944B72F801F6CFEEEB9D
:10C38000F7E184918F010F5F1F4F882321F00E94F6
:10C390004B72F801F6CFE4EFF2E284918F010F5F68
:10C3A0001F4F882321F00E944B72F801F6CFE7EA75
:10C3B000F7E184918F010F5F1F4F882321F00E94C6
:10C3C0004B72F801F6CFE4EFF2E284918F010F5F38
:10C3D0001F4F882321F00E944B72F801F6CF809105
:10C3E0005B1590915C15BE016F5F7F4F009719F050
:10C3F000681B790B02C06156754188E997E10E947C
:10C400004AC160EF74E081E897E10E944AC18AE086
:10C410000E944B7281E08093720780937307809330
:10C420007407809375070E94DDD38CE0E6E6F7E0A1
:10C43000A1E2B5E001900D928A95E1F70E943A4998
:10C440008091190290911A0290931C0280931B0212
:10C4500080910101806480930101809101018061DC
:10C4600080930101809101018860809301016D9AA0
:10C470008091010188608093010186E045DD809113
:10C48000010180628093010188E03EDD6C9A82E0C8
:10C490003BDD87ED80937A0010927E0010927D0044
:10C4A00080917E00816080937E0080917E0082601A
:10C4B00080937E0080917E00846080937E0080E87F
:10C4C00088BD80916E00846080936E006AEF70E09A
:10C4D00080E090E00E94D64F85E090E09093600766
:10C4E00080935F0760E080911502909116020E9490
:10C4F000D3CC20E030E040EA50E40F94090187FFFC
:10C500000AC08091150290911602409790931602EE
:10C5100080931502E7CF81E391E090931A02809314
:10C52000190260E080915B0790915C070E94D3CC78
:10C5300020E030E848E953E40F946807181654F4F3
:10C5400080915B0790915C07409690935C07809385
:10C550005B07E7CF85E090E09093620780936107E7
:10C5600061E080911702909118020E94D3CC20E0E4
:10C5700030E040EA50E40F94090187FF0AC080913F
:10C580001702909118024097909318028093170217
:10C59000E7CF81E391E090931C0280931B0261E05E
:10C5A00080915D0790915E070E94D3CC20E030E837
:10C5B00048E953E40F946807181654F480915D0716
:10C5C00090915E07409690935E0780935D07E7CF5A
:10C5D00080911302909114020E94B5CE20E030E0C9
:10C5E00040EA50E40F94090187FF0AC080911302CA
:10C5F0009091140240979093140280931302E8CF15
:10C600008091590790915A070E94B5CE20E030E002
:10C6100046E153E40F946807181654F480915907C3
:10C6200090915A07409690935A0780935907E8CF04
:10C6300098E288E10FB6F894A895809360000FBE49
:10C64000909360001FB7F89480916307811124C014
:10C65000EDEAF3E28491E3EFF3E29491E82FF0E066
:10C66000EE0FFF1FE25AFC4DA591B491EC91E92326
:10C6700021F461E085E30E94DF4E85E30E9484BBE4
:10C680008CB580618CBD8CB580648CBD84E30E94C8
:10C6900084BB83E30E9484BB809163078F5F809398
:10C6A00063071FBF579A1EE7E12E13E0F12E10E03B
:10C6B000F70161917F0170E0812F0E94E4F71F5F15
:10C6C0001530B1F7999A989A809107018068809304
:10C6D00007019A9A809107018064809307018091F5
:10C6E0000701806280930701809107018860809331
:10C6F0000701809107018061809307018091070104
:10C700008260809307018091070184608093070114
:10C71000B3E8EB2EB3E0FB2E10E0F70161917F014F
:10C72000812F0E94BEF71F5F1530B9F780910A0173
:10C73000826080930A0180910A01816080930A01DE
:10C7400080910A01846080930A0180910A018064CB
:10C7500080930A0180910A01806880930A010F9AF0
:10C76000179A0E9A169A0D9A159A0C9A149A0B9A71
:10C77000139A26982E9A25982D9A24982C9A389AAE
:10C780004098179A10924705399A4198169A109234
:10C7900048053A9A4298159A109249053B9A43984F
:10C7A000149A3C9A4498139A809180008C7F8093CD
:10C7B000800080918100877E8860809381008091D5
:10C7C00080008F738093800080918100887F8260D9
:10C7D0008093810080E090E49093890080938800AA
:10C7E000109285001092840080916F008260809387
:10C7F0006F0081E08093650778940E947FDD6C9ADA
:10C800000E9421C964EC79E080E090E00E9448C475
:10C8100080911D02811118C064EC79E080E090E005
:10C820000E9448C481E0809365078093640770E6A6
:10C83000572EEDE04E2EF5E9CF2EF8E1DF2EA0E0E9
:10C84000AA2EA0E0BA2E8FC010921D022091920A4B
:10C8500030E07901F8E3EF1AF108F7FE04C079013E
:10C8600087E3E81AF108F594E7942E5131093695DB
:10C870002795F22E0E94ABBD0CEF16E123E147E0B5
:10C880006CE08E2D0E94DDBB84E00E94A9EE009139
:10C89000920A10E002571109169507956091930AC4
:10C8A000625144E653E08F2D0E945DBC6091930A73
:10C8B00066504AE653E0802F0E945DBC0E94A3BBF5
:10C8C0008111DACFA9CF8091970780FD36C1809181
:10C8D000970784FD32C190E2F92E8091970781FD80
:10C8E00049C18091970785FD45C100E28091970776
:10C8F00082FD5CC18091970786FD58C110E28AE0F5
:10C900000E944B721F926F921F921F931F920F9360
:10C910001F92FF92DF92CF921F92AAD9109297078F
:10C920000FB6F894DEBF0FBECDBF80917607882387
:10C9300091F010921F0B81E19DE00E94BF8981E17F
:10C940009DE00E94F18910921E0B10921D0B0E9417
:10C9500034840E946ECE80E00E94D5E8A114B10418
:10C9600031F00E9400002AE0722E30E2632E8091A6
:10C970001909843010F40E94B6468091CA0D8823AC
:10C98000F1F00E9410500091C60D1091C70D20913A
:10C99000C80D3091C90DDC01CB01801B910BA20B9E
:10C9A000B30BB7FD0CC01092CA0D8091200B811102
:10C9B000C1C00E94BD5C8091200B8111BBC08091E1
:10C9C0001909882309F498C080911D0B882309F464
:10C9D00080C000911809509E800111240856184FFC
:10C9E00068ED78E1C8010F948800892BF9F081E1A6
:10C9F0009DE00E94BF8981E19DE00E94F189109233
:10CA00001E0B10921D0BE5ECF8E184918F010F5F76
:10CA10001F4F882341F00E944B72F801F6CF80919E
:10CA20001E0B811156C00E94B9EB55C0F801019050
:10CA30000020E9F731977F01E01AF10A1092110DF9
:10CA40006EE470E0C8010F9471084C01009729F45E
:10CA5000F7013197E00FF11F0EC060E270E00F9414
:10CA600071088C010F5F1F4F6AE270E0C4010F94E0
:10CA70007108FC013197418272821382F8010190A2
:10CA80000020E9F73197AF01401B510BB80181E15C
:10CA90009DE00E940B8B8091110D882309F4BFCF7C
:10CAA000E5EFF6E184918F010F5F1F4F882321F09E
:10CAB0000E944B72F801F6CFEEE7F8E184918F0106
:10CAC0000F5F1F4F882309F4AACF0E944B72F80111
:10CAD000F5CF0E94472980911909882369F0815078
:10CAE00080931909809118098F5F843018F480931E
:10CAF000180902C01092180980919707882309F439
:10CB00002ACFE4EFF2E284918F010F5F1F4F882359
:10CB100021F00E944B72F801F6CFE6EBF8E1849128
:10CB20008F010F5F1F4F882309F4CDCE0E944B72F7
:10CB3000F801F5CF0E940C5C42CF60918B07709199
:10CB40008C0780918D0790918E070F940F01209193
:10CB50007707309178074091790750917A070F94C1
:10CB60006E01AB01BC0182EB98E10E9406C188E531
:10CB7000F82EB3CE60918F07709190078091910746
:10CB8000909192070F940F0120917B0730917C07C1
:10CB900040917D0750917E070F946E01AB01BC015F
:10CBA0008EEA98E10E9406C109E5A0CE6091930744
:10CBB0007091940780919507909196070F940F01BB
:10CBC00020917F0730918007409181075091820723
:10CBD0000F946E01AB01BC018AEA98E10E9406C184
:10CBE0001AE58DCECF92DF92EF92FF92CF93DF9333
:10CBF0006A017B01FC018491EF012196882321F0D9
:10CC00000E944B72FE01F7CF4AE0C701B601DF91E7
:10CC1000CF91FF90EF90DF90CF900C94A472CF92C1
:10CC2000DF92EF92FF92CF93DF936A017B01FC01C9
:10CC30008491EF012196882321F00E944B72FE011E
:10CC4000F7CF42E0C701B601DF91CF91FF90EF909F
:10CC5000DF90CF900C942473CF92EF92FF920F93BA
:10CC60001F93E0908702F090880200918902109152
:10CC70008A02C09046052DE235E049E255E065E2C2
:10CC800075E081E295E00E943BA31F910F91FF9018
:10CC9000EF90CF900895CF93DF938091200B88235E
:10CCA00049F1EDE7F9E18491EF012196882321F024
:10CCB0000E944B72FE01F7CF6091C20D7091C30DBF
:10CCC0008091C40D9091C50D4AE00E94A4728FE23C
:10CCD0000E944B726091BE0D7091BF0D8091C00D8E
:10CCE0009091C10D4AE00E94A4728AE0DF91CF9139
:10CCF0000C944B72EFE8F9E18491EF0121968823BF
:10CD000021F00E944B72FE01F7CFDF91CF91089581
:10CD10008091200B8823A9F083E50E94E6498823AF
:10CD200081F00E945449AB01BC014093C20D509365
:10CD3000C30D6093C40D7093C50D81E19DE00C940B
:10CD4000BA880895E0912C04F0912D048081882305
:10CD500029F0803209F410823196F8CF40E061E08A
:10CD600080912C0490912D040C948E590F931F9355
:10CD7000CF93DF93CDB7DEB76F970FB6F894DEBFD2
:10CD80000FBECDBFECE6F9E184918F010F5F1F4F1D
:10CD9000882321F00E944B72F801F6CF1092CB0D40
:10CDA00040E050E0BA0187E79BE00E94BA888BE13F
:10CDB000E7E7FBE0DE01159601900D928A95E1F719
:10CDC0008091750B9091760B9C838B8384E993E023
:10CDD0009A83898340E050E0BE016F5F7F4F89EC0A
:10CDE00093E00E9428BFCE0101960E945CE8EDE529
:10CDF000F9E184918F010F5F1F4F882321F00E947A
:10CE00004B72F801F6CF6F960FB6F894DEBF0FBEE7
:10CE1000CDBFDF91CF911F910F910895BF92CF9217
:10CE2000DF92EF92FF920F931F93CF93DF9381E0F6
:10CE300080939A02BB24B39481E090919A02992343
:10CE400009F44FC0882309F44CC080E00E94D5E863
:10CE500007E11AE0CCEDD4E0F801619171918F0106
:10CE600061157105B1F1072E000C880B990B0F9419
:10CE70000F019B01AC01688179818A819B810F94AC
:10CE800041056B017C0120E030E0A9010F946807A7
:10CE900018165CF420E030E040E251E4C701B6012E
:10CEA0000F9468071816ACF40AC020E030E040E2A6
:10CEB00051ECC701B6010F94090187FF0AC0B09277
:10CEC000DE0D40E050E0BA0181E29EE70E94DC50B6
:10CED000B3CF249680E0FAE00B311F0709F4ADCF01
:10CEE000BBCFDF91CF911F910F91FF90EF90DF901B
:10CEF000CF90BF900C941756CF92DF92EF92FF9293
:10CF00000F931F93CF93DF9300D01F92CDB7DEB75F
:10CF1000182F662351F010922409109220091092C4
:10CF2000210910922209109223090E941050C090EA
:10CF30002009D0902109E0902209F09023099B015B
:10CF4000AC012C193D094E095F0957FD3EC017FD84
:10CF500016C040912409212F012E000C330B2C5FA9
:10CF60003F4FE42F042E000CFF0B2E173F076CF1F0
:10CF700041172CF000E911E020E030E004C004EC9F
:10CF800019E020E030E0DC01CB01800F911FA21FEF
:10CF9000B31F8093200990932109A0932209B09395
:10CFA000230980ED97E09C838B838CE291E09A8348
:10CFB0008983BE016D5F7F4FCE0101960E94045EA2
:10CFC000809124098F5F809324090F900F900F9018
:10CFD0000F90DF91CF911F910F91FF90EF90DF9015
:10CFE000CF900895CF92DF92FF920F931F93CF932C
:10CFF000DF9385E40E94E649D82F811102C00E9488
:10D0000044F88EE4C82E83E0D82E01E215E0C0E09B
:10D01000F12CF60181916F010E94E649882359F0B5
:10D020000E948449F8016083718382839383C330B3
:10D0300011F0FF24F394CF5F0C5F1F4FC43049F70A
:10D04000FF2019F00E943A4903C0D1110E942A5FC3
:10D05000DF91CF911F910F91FF90DF90CF900C94B3
:10D060001385BF92CF92DF92EF92FF920F931F939F
:10D07000CF93DF9385E2E82E89E0F82E01E215E0F8
:10D080009BE3C92E94E0D92ECEE4D3E0BC2E84E0FD
:10D09000B80E89910E94B7498823D9F00E9484492B
:10D0A000F6012081211104C020913F04222331F098
:10D0B000F801208131814281538103C020E030E0BA
:10D0C000A9010F944205F7016083718382839383E2
:10D0D0000AC0F80180819181A281B381F701808328
:10D0E0009183A283B383F4E0EF0EF11C0C5F1F4F1A
:10D0F0008FEFC81AD80ABC12CCCF86E40E94E6494A
:10D100008823C9F00E94844920E030E0A9010F94EF
:10D110006807181684F40E94844920E030E040E754
:10D1200052E40F941E0660938702709388028093E6
:10D13000890290938A02DF91CF911F910F91FF9006
:10D14000EF90DF90CF90BF9008959F92AF92BF92E3
:10D15000CF92DF92EF92FF920F931F93CF93DF93C3
:10D1600000D01F92CDB7DEB7902EA12EB22ED32EB7
:10D1700094E089027001112487010F5D1A4FF801B4
:10D18000108211821282138249835A836B837C83BB
:10D190000E943A4949815A816B817C81F801408320
:10D1A000518362837383C090460520E030E0A9017B
:10D1B000692D7A2D8B2D9D2D0F940901811108C0A9
:10D1C000F701E25DF64CE590F5900591149106C0EB
:10D1D000892D9A2DAB2DBD2D7C018D012DE235E0E1
:10D1E00049E255E065E275E081E295E00E943BA3EB
:10D1F0000E9444F8109297070F900F900F900F9095
:10D20000DF91CF911F910F91FF90EF90DF90CF9022
:10D21000BF90AF909F9008954F925F926F927F92D0
:10D220008F929F92AF92BF92CF92DF92EF92FF9236
:10D230000F931F93CF93DF935C014B01EA018901A8
:10D2400040908702509088026090890270908A0214
:10D25000288139814A815B816091290570912A0575
:10D2600080912B0590912C050F94090187FF29C00F
:10D27000F801C080D180E280F38020E030E0A90195
:10D28000C701B6010F940901811106C0E6E3F9E375
:10D29000C590D590E590F490C0928702D092880214
:10D2A000E0928902F0928A0288819981AA81BB81E9
:10D2B0008093290590932A05A0932B05B0932C0504
:10D2C000CBDCF801C080D180E280F38020E030E048
:10D2D000A901C701B6010F940901811106C0C12C33
:10D2E000D12C88ECE82E82E4F82EC0928702D092EE
:10D2F0008802E0928902F0928A02F5018081918190
:10D30000A281B3818093210590932205A0932305E8
:10D31000B0932405F40180819181A281B38180932F
:10D32000250590932605A0932705B093280594DC46
:10D33000288139814A815B816091290570912A0594
:10D3400080912B0590912C050F94680718164CF5C9
:10D35000F801C080D180E280F38020E030E0A901B4
:10D36000C701B6010F940901811106C0E6E3F9E394
:10D37000C590D590E590F490C0928702D092880233
:10D38000E0928902F0928A0288819981AA81BB8108
:10D390008093290590932A05A0932B05B0932C0523
:10D3A0005BDC0E9444F840928702509288026092AF
:10D3B000890270928A02DF91CF911F910F91FF90A5
:10D3C000EF90DF90CF90BF90AF909F908F907F9025
:10D3D0006F905F904F9008959B01AC0165E275E0FE
:10D3E00081E295E019CF80E1E1E2F5E0A5E2B9E064
:10D3F00001900D928A95E1F708952F923F924F92F6
:10D400005F926F927F928F929F92AF92BF92CF92D4
:10D41000DF92EF92FF920F931F93CF93DF93CDB7DD
:10D42000DEB762970FB6F894DEBF0FBECDBF182FE0
:10D430000E9444F820914605298B40E050E0BA0153
:10D4400080E00E9431E68091870290918802A0914D
:10D450008902B0918A0280931C0990931D09A093C0
:10D460001E09B0931F098091240290912502909388
:10D470001B0980931A0984E690E09093250280931B
:10D4800024020E94685081E080936507111119C041
:10D4900088E50E94B749082F89E50E94B749182FEF
:10D4A0008AE50E94B749282E011106C0111113C048
:10D4B000882361F0012F0FC0112369F0012F382E4E
:10D4C0000BC011E001E02224239402C0182F082F82
:10D4D0003324339401C0312C86DF311005C0011193
:10D4E00003C0112309F40EC120E030E040EA50E40B
:10D4F0006091F2137091F3138091F4139091F513EE
:10D500000F94420560932D0970932E0980932F0983
:10D51000909330092091290530912A0540912B05DF
:10D5200050912C050F946807181654F419821A822A
:10D530001B821C82BE016F5F7F4F8DE299E04CDF42
:10D5400031100DC0011103C01111D7C0DBC0111182
:10D5500006C080E00E9436E73320B1F3CEC01092BF
:10D560002505109226051092270510922805109285
:10D5700021051092220510922305109224050E9485
:10D580003A49EBE7F9E384918A8BEFE6F9E3C5903A
:10D59000D590E590F490E3E7F9E385909590A59018
:10D5A000B490A5019401C701B6010F94680718163D
:10D5B0002CF4A7019601C501B40104C0A501940192
:10D5C000C701B6010F941E066D877E878F87988BE3
:10D5D0008EE2682E89E3782EF3016591759185912D
:10D5E000949122E3422E29E3522EF20125913591A6
:10D5F000459154910F94090187FF02C0F30101C0C6
:10D60000F20145905590659074902D853E854F852B
:10D610005889CA01B9010F946E0120E030E040E85A
:10D620005FE30F9442050F94AD079B01AC01C3016A
:10D63000B2010F946E0169877A878B879C87ECE72C
:10D64000F9E394919D8720E030E040EC5FE3C50171
:10D65000B4010F946E012B013C01AD856A2FAA0F16
:10D66000770B880B990B0F940F019B01AC01C30141
:10D67000B2010F946E0169837A838B839C8320E0CF
:10D6800030E040EC5FE3C701B6010F946E016B011F
:10D690007C01BA896B2FBB0F770B880B990B0F940A
:10D6A0000F019B01AC01C701B6010F946E016D83A0
:10D6B0007E838F8398879E01275F3F4F49E255E025
:10D6C000BE016F5F7F4FCE010596A6DD10929707D2
:10D6D0001092250510922605109227051092280514
:10D6E0001092210510922205109223051092240514
:10D6F00031102FCF01112DCF27CF81E00E9436E7C7
:10D70000311003C0222009F4B7C080914705882357
:10D7100021F08091480581111CC060E08FE499E1FF
:10D720000E94E1C5E4EFF2E284918F010F5F1F4F89
:10D73000882319F0B0D6F801F7CFE0E4F9E184913D
:10D740008F010F5F1F4F882309F496C0A4D6F801FC
:10D75000F6CF0E943A494090EA135090EB13609044
:10D76000EC137090ED1320E030E040E251E4C3018F
:10D77000B2010F9442054B015C016093250970933F
:10D78000260980932709909328098091EE139091A0
:10D79000EF13A091F013B091F1138D879E87AF879F
:10D7A000B88B20E030E040E251E4BC01CD010F94A1
:10D7B00042056B017C016093290970932A098093CB
:10D7C0002B0990932C098091290590912A05A0910D
:10D7D0002B05B0912C0580932D0990932E09A093D1
:10D7E0002F09B0933009A3019201C501B4010F9430
:10D7F00041054B015C0122E630E140E050EC0F9422
:10D80000680787FD7EC021E230E04FE853E4C501A0
:10D81000B4010F94090118160CF473C02D853E85D0
:10D820004F855889C701B6010F9441056B017C01F2
:10D830002FE632E143E85AEB0F94680787FD61C099
:10D8400021E230E04AE853E4C701B6010F94090130
:10D8500018160CF456C019821A821B821C829E0173
:10D860002F5F3F4F49E255E069E279E085E299E0B8
:10D87000D3DC82E00E9436E70E943A498091640737
:10D880008093650780911C0990911D09A0911E0944
:10D89000B0911F098093870290938802A093890218
:10D8A000B0938A0280911A0990911B0990932502E6
:10D8B000809324020E94685021E040E050E0BA01C9
:10D8C00089890E949F8183E0809312020E941385C0
:10D8D00062960FB6F894DEBF0FBECDBFDF91CF9139
:10D8E0001F910F91FF90EF90DF90CF90BF90AF907E
:10D8F0009F908F907F906F905F904F903F902F9070
:10D90000089560E08FE299E10E94E1C5E4EFF2E260
:10D9100084918F010F5F1F4F882319F0BCD5F80148
:10D92000F7CFEDE1F9E184918F010F5F1F4F88235D
:10D9300009F4A2CFB0D5F801F6CF80E1E5E2F9E035
:10D94000A1E2B5E001900D928A95E1F708952F923A
:10D950003F924F925F926F927F928F929F92AF927F
:10D96000BF92CF92DF92EF92FF920F931F93CF93CC
:10D97000DF93CDB7DEB7C854D1090FB6F894DEBF38
:10D980000FBECDBF90917802992309F4B5C4382E0B
:10D9900068DB82E50E94E649882309F42AC10E94D7
:10D9A00084496B017C0140902105509022056090D4
:10D9B000230570902405209125053091260540917E
:10D9C000270550912805298B3A8B4B8B5C8B8091D6
:10D9D000250990912609A0912709B09128098D8BDE
:10D9E0009E8BAF8BB88F2091290930912A094091E5
:10D9F0002B0950912C0929A33AA34BA35CA320E047
:10DA000030E0A901C701B6010F940901882309F488
:10DA10005BC4A30192016D897E898F89988D0F94D3
:10DA2000090181110DC029893A894B895C8969A155
:10DA30007AA18BA19CA10F940901882309F444C405
:10DA400020E030E0A901C701B6010F940901881F49
:10DA50008827881F381209C080E090E0A0E8BFE363
:10DA600089A79AA7ABA7BCA708C020E030E040E890
:10DA70005FEB29A73AA74BA75CA7A30192016D8989
:10DA80007E898F89988D0F9441056D8F7E8F8F8F42
:10DA900098A329893A894B895C8969A17AA18BA1CC
:10DAA0009CA10F9441056DA37EA38FA398A72D8DF4
:10DAB0003E8D4F8D58A1CA01B9010F946E014B01E3
:10DAC0005C012DA13EA14FA158A5CA01B9010F9437
:10DAD0006E019B01AC01C501B4010F9442050F9486
:10DAE000AD07698F7A8F8B8F9C8F20E030E040E00C
:10DAF0005FE30F946E014B015C01A7019601C70122
:10DB0000B6010F946E016B017C01A5019401C50162
:10DB1000B4010F946E019B01AC01C701B6010F94D3
:10DB200041050F94AD079B01AC0169A57AA58BA5B2
:10DB30009CA50F946E014B015C012D893E894F8994
:10DB4000588DC301B2010F94420520E030E040E05F
:10DB50005FE30F946E016B017C016DA17EA18FA12B
:10DB600098A59058298D3A8D4B8D5C8D0F941E068B
:10DB70009B01AC01C501B4010F946E019B01AC0186
:10DB8000C701B6010F944205A30192010F9441050C
:10DB90006B017C0129A13AA14BA15CA169897A8919
:10DBA0008B899C890F94420520E030E040E05FE3E0
:10DBB0000F946E012B013C01298D3A8D4B8D5C8DAC
:10DBC0006D8D7E8D8F8D98A10F941E069B01AC01EB
:10DBD000C501B4010F946E019B01AC01C301B201F8
:10DBE0000F94420529893A894B895C890F94410534
:10DBF00014C089E40E94E649882329F00E948449E0
:10DC00006B017C0103C0C12CD12C76018AE40E94F7
:10DC1000E6498823D9F00E94844969A37AA38BA39B
:10DC20009CA320E030E0A901C701B6010F940901CF
:10DC300081111AC020E030E0A90169A17AA18BA16D
:10DC40009CA10F94090181110FC03EC320E030E078
:10DC5000A901C701B6010F940901882309F434C34F
:10DC600019A21AA21BA21CA2D701C601B058898B07
:10DC70009A8BAB8BBC8B29A13AA14BA15CA15058CC
:10DC80002D8B3E8B4F8B588F9C01AD01BC01CD017C
:10DC90000F946E014B015C012D893E894F89588D8F
:10DCA000CA01B9010F946E019B01AC01C501B40119
:10DCB0000F9442050F94AD0769AF7AAF8BAF9CAF5D
:10DCC0008091210590912205A0912305B091240512
:10DCD000898F9A8FAB8FBC8FA7019601BC01CD01B4
:10DCE0000F94420569A77AA78BA79CA720912505C9
:10DCF0003091260540912705509128052DA33EA37C
:10DD00004FA358A729A13AA14BA15CA16DA17EA167
:10DD10008FA198A50F94420525966CAF7DAF8EAF6D
:10DD20009FAF25978091250990912609A0912709F9
:10DD3000B09128098DA79EA7AFA7B8AB29A53AA592
:10DD40004BA55CA5BC01CD010F9441056B017C0185
:10DD50002091290930912A0940912B0950912C09D1
:10DD600029AB3AAB4BAB5CAB25962CAD3DAD4EAD84
:10DD70005FAD259769A97AA98BA99CA90F94410544
:10DD80004B015C018091290590912A05A0912B05FA
:10DD9000B0912C058DAB9EABAFABB8AF9C01AD0184
:10DDA00060912D0970912E0980912F099091300971
:10DDB0000F9441056D8F7E8F8F8F98A3209131092D
:10DDC00030913209409133095091340921962CAF9A
:10DDD0003DAF4EAF5FAF219780912D0590912E05FD
:10DDE000A0912F05B091300529968CAF9DAFAEAFB5
:10DDF000BFAF2997A701960169897A898B899C8988
:10DE00000F946E012B013C01A50194016D897E895F
:10DE10008F89988D0F946E019B01AC01C301B201F3
:10DE20000F9442052B013C01A501940169897A896F
:10DE30008B899C890F946E014B015C01A7019601AF
:10DE40006D897E898F89988D0F946E019B01AC013D
:10DE5000C501B4010F944105A30192010F94B505CA
:10DE60006B017C0120E030E0A9010F94090187FFDC
:10DE70000AC02BED3FE049EC50E4C701B6010F9416
:10DE800042056B017C01332051F02BED3FE049EC62
:10DE900050E4C701B6010F9441056B017C0120E0FD
:10DEA00030E0A901C701B6010F940901811120C01A
:10DEB0002DA53EA54FA558A9698D7A8D8B8D9C8D7A
:10DEC0000F940901811114C029A93AA94BA95CA991
:10DED0006DA17EA18FA198A50F940901811108C0A1
:10DEE0009BEDC92E9FE0D92E99ECE92E90E4F92EF6
:10DEF00029AD3AAD4BAD5CADC701B6010F946E01D3
:10DF00009B01AC010F946E014B015C012D8D3E8D88
:10DF10004F8D58A1CA01B9010F946E019B01AC014C
:10DF2000C501B4010F9442050F94AD074B015C018C
:10DF30002FE632E143E85AE30F94090187FDC1C19E
:10DF4000C501B4010F94B7060F948B061B01672B14
:10DF500019F422242394312CB10180E090E00F9435
:10DF60000D014B015C019B01AC01C701B6010F948F
:10DF70001E06698F7A8F8B8F9C8FA50194016D8D02
:10DF80007E8D8F8D98A10F941E0669AF7AAF8BAFEF
:10DF90009CAF29962CAD3DAD4EAD5FAD2997219636
:10DFA0006CAD7DAD8EAD9FAD21970F944105A50160
:10DFB00094010F941E0621966CAF7DAF8EAF9FAF7C
:10DFC0002197298D3A8D4B8D5C8DCA01B9010F9433
:10DFD0006E0120E030E040E05FE30F946E019B01B2
:10DFE000AC0160E070E080E89FE30F9441056DA70D
:10DFF0007EA78FA798AB2DA93EA94FA958AD298719
:10E000003A874B875C8729968CAD9DADAEADBFAD91
:10E0100029978D879E87AF87B88B60912402709176
:10E020002502072E000C880B990B0F940F012091ED
:10E030008702309188024091890250918A020F94A0
:10E040006E012AE037ED43E25CE30F946E0169ABA9
:10E050007AAB8BAB9CAB0E9410509B01AC01285358
:10E060003F4F4F4F5F4F2DAB3EAB4FAB58AF498843
:10E070005A886B887C8841E050E05EA34DA359E14B
:10E080005D8FADA1BEA1A215B30509F409C10E941F
:10E09000F7D10E941050DC01CB012DA93EA94FA958
:10E0A00058AD821B930BA40BB50BB7FD0FC00E949C
:10E0B00010509B01AC0128533F4F4F4F5F4F2DAB8A
:10E0C0003EAB4FAB58AF80E00E94D5E83D8D31505C
:10E0D0003D8F3323E9F12DA53EA54FA558A96D89A4
:10E0E0007E898F89988D0F946E016B017C01298D3B
:10E0F0003A8D4B8D5C8DB201C3010F946E01A70167
:10E1000096010F9442056B017C012DA53EA54FA5FC
:10E1100058A9B201C3010F946E014B015C01298D16
:10E120003A8D4B8D5C8D6D897E898F89988D0F948A
:10E130006E019B01AC01C501B4010F9441052B0197
:10E140003C01C601D7018D8B9E8BAF8BB88F51C020
:10E150004DA15EA1BA0180E090E00F940D01298DE0
:10E160003A8D4B8D5C8D0F946E014B015C010F94C9
:10E170001B066B017C01C501B4010F94A3074B0181
:10E180005C01A701960169897A898B899C890F9422
:10E190006E012B013C01A501940169A17AA18BA11B
:10E1A0009CA10F946E019B01AC01C301B2010F94BD
:10E1B00042052B013C01A501940169897A898B896B
:10E1C0009C890F946E014B015C01A701960169A126
:10E1D0007AA18BA19CA10F946E019B01AC01C5019A
:10E1E000B4010F9441056D8B7E8B8F8B988F59E115
:10E1F0005D8F9201A30169A57AA58BA59CA50F94BB
:10E20000420569837A838B839C832D893E894F895C
:10E21000588D25966CAD7DAD8EAD9FAD25970F9435
:10E2200042056D837E838F83988729AD3AAD4BADD0
:10E230005CAD69857A858B859C850F9442056987DD
:10E240007A878B879C8721962CAD3DAD4EAD5FAD17
:10E2500021976D857E858F8598890F9442056D87FE
:10E260007E878F87988BCE0101960E9464EBC090C9
:10E270004605E9A8FAA80BA91CA99E01235F3F4FF8
:10E28000AE01475F5F4FBE016B5F7F4FCE010196CE
:10E290000E943BA38DA19EA101969EA38DA3F1CECA
:10E2A000C0904605E9A8FAA80BA91CA921E339E00A
:10E2B0004DE259E069E279E085E299E00E943BA3F2
:10E2C0003CDB0E94685018C0E5EFF6E184917F01C5
:10E2D000BFEFEB1AFB0A882319F0DDD0F701F6CF68
:10E2E000E7E0F9E184917F012FEFE21AF20A882337
:10E2F00019F0D1D0F701F6CFC85BDF4F0FB6F89415
:10E30000DEBF0FBECDBFDF91CF911F910F91FF9068
:10E31000EF90DF90CF90BF90AF909F908F907F90C5
:10E320006F905F904F903F902F900895CF92EF9213
:10E33000FF920F931F93C09046057B018C0121E350
:10E3400039E04DE259E069E279E085E299E00E9426
:10E350003BA31F910F91FF90EF90CF900895CF9224
:10E36000DF92EF92FF920F931F93CF93DF9394E08E
:10E370008902E0011124FE01EA59F84F20E030E063
:10E38000A90160817181828193810F944205FE0110
:10E39000EA50FC4E20813181428153810F94420525
:10E3A0006B017C01FE01E651FC4E60837183828328
:10E3B0009383FE01E151F74E65917591859194919A
:10E3C0008E01015D1B4FA70196010F944205F801D4
:10E3D0006083718382839383FE01E550F74E6591DC
:10E3E000759185919491CA5DDD4FA70196010F94B7
:10E3F0004205688379838A839B83DF91CF911F9144
:10E400000F91FF90EF90DF90CF900895EF92FF92E1
:10E410000F931F93CF93DF937C0184E50E94E6491D
:10E42000D82F882329F10E946449C82F8230E4F054
:10E43000E4EFF2E284918F010F5F1F4F882319F000
:10E440002AD0F801F7CF8DE426D0B70180E090E024
:10E450004AE07AD06C2FCC0F770B8CED98E10E94BC
:10E460004AC18AE018D008C080932E04D0E004C0CE
:10E470008091460580932E048D2FDF91CF911F91BF
:10E480000F91FF90EF9008958FEF8EBD0DB407FEB2
:10E49000FDCF8EB5089591E0909358073FB7F8945B
:10E4A0002091EA099091EB093FBF291304C0909194
:10E4B000C00095FD3EC09091EA099F5F9F71209139
:10E4C000EB09921325C00FB607FCF9CF2091C000CD
:10E4D00025FFF5CF2091EB09E22FF0E0E653F64F50
:10E4E00030812F5F2F712093EB093093C60020916C
:10E4F000C00020642093C0003091EA092091EB090C
:10E500003213DDCF2091C1002F7D2093C100D7CFE2
:10E51000E091EA09F0E0E653F64F80832FB7F894D4
:10E520009093EA098091C10080628093C1002FBF5F
:10E5300008959FB7F8948093C6008091C0008064CE
:10E540008093C0009FBF08958F929F92AF92BF9219
:10E55000EF92FF921F93CF93DF93CDB7DEB7A097D3
:10E560000FB6F894DEBF0FBECDBF611571058105F2
:10E57000910579F110E0842E912CA12CB12CEE2480
:10E58000E394F12CEC0EFD1EE10EF11C17FDFA9444
:10E59000A50194010F94E404F7016083B901CA0155
:10E5A0001F5F611571058105910549F7115010F143
:10E5B000E1E0F0E0EC0FFD1FE10FF11D17FDFA9512
:10E5C00080818A3010F097E301C090E3890F63DF08
:10E5D000EDCF80E3A0960FB6F894DEBF0FBECDBF9F
:10E5E000DF91CF911F91FF90EF90BF90AF909F90E0
:10E5F0008F9051CFA0960FB6F894DEBF0FBECDBF5F
:10E60000DF91CF911F91FF90EF90BF90AF909F90BF
:10E610008F900895CF92DF92EF92FF926B017C0171
:10E6200097FF0AC08DE237DFF094E094D094C09455
:10E63000C11CD11CE11CF11C4AE0C701B601FF90CE
:10E64000EF90DF90CF9080CF8F929F92AF92BF924A
:10E65000CF92DF92EF92FF92CF936B017C01B42EA9
:10E6600020E030E0A9010F94090187FF06C08DE288
:10E6700012DFF7FAF094F7F8F094C0E060E070E091
:10E6800080E09FE3CB1541F02DEC3CEC4CEC5DE3DE
:10E690000F946E01CF5FF6CF9B01AC01C701B601AD
:10E6A0000F9442056B017C010F948B064B015C01BA
:10E6B0004AE04ADFCC2379F1C501B4010F940D0182
:10E6C0009B01AC01C701B6010F9441056B017C01B0
:10E6D0008EE2E1DE20E030E040E251E4C701B60125
:10E6E0000F946E014B015C010F9486066B01770F4E
:10E6F000EE08FF08C701B6018DDFC701B6010F9410
:10E700000F019B01AC01C501B4010F9441056B01E0
:10E710007C01C150F9F6CF91FF90EF90DF90CF9040
:10E72000BF90AF909F908F9008958FB7F89490917D
:10E73000C9092091C809291759F0E92FF0E0E85BD1
:10E74000F64F208130E09F5F9F779093C90902C008
:10E750002FEF3FEF8FBFC90108951F920F920FB6A1
:10E760000F9211240BB60F922F933F934F935F9309
:10E770006F937F938F939F93AF93BF93EF93FF9389
:10E780009091C6002FB7F894E091C80981E08E0FF0
:10E790008F773091C909831731F0F0E0E85BF64FCD
:10E7A00090838093C8092FBF20914709422F50E0E2
:10E7B0004C30510508F046C0FA018827EE55FF4F4E
:10E7C0008F4F0D942D089D3441F09E34B9F481E0B3
:10E7D00005C09A3330F09D3471F582E0809347098B
:10E7E00046C0903308F043C0903209F440C09D32D7
:10E7F00011F53DC0913329F0943329F09032D9F4CA
:10E8000036C083E0EBCF88E0E9CF903321F091333D
:10E8100091F486E0E3CF84E0E1CF983361F485E0C2
:10E82000DDCF923341F487E0D9CF913321F489E0F1
:10E83000D5CF903311F08BE0D1CF8AE0CFCF9A3093
:10E84000B1F413C09A3099F4273049F02A3059F0C6
:10E85000253059F410929A021092F10D06C089ECFD
:10E8600099E10E9470E80E94348410924709FF9158
:10E87000EF91BF91AF919F918F917F916F915F9138
:10E880004F913F912F910F900BBE0F900FBE0F90A5
:10E890001F9018951F920F920FB60F9211240BB66E
:10E8A0000F928F939F93EF93FF938091EB09E82F43
:10E8B000F0E0E653F64F90818F5F8F718093EB0904
:10E8C0009093C6008091C00080648093C0009091B6
:10E8D000EA098091EB09981305C08091C1008F7DF2
:10E8E0008093C100FF91EF919F918F910F900BBE8C
:10E8F0000F900FBE0F901F9018954F925F926F92DE
:10E900007F928F929F92AF92BF92CF92EF92FF929F
:10E910000F931F93CF93DF93CDB7DEB728970FB632
:10E92000F894DEBF0FBECDBF5C014B013A01290157
:10E930008091070A83FD45C020E030E0A901F8017D
:10E9400060817181828193810F94090181110CC0D2
:10E9500020E030E0A901F50160817181828193811D
:10E960000F940901882369F1F090060AF11027C07D
:10E97000E0914605F0E0EE0FFF1FE95EF54F2081C4
:10E98000318180911E0290911F0228173907BCF433
:10E99000E5EFF6E184918F010F5F1F4F882319F097
:10E9A0007ADDF801F7CFE0EAF9E184918F010F5F9A
:10E9B0001F4F882309F40FC16EDDF801F6CF0E94C6
:10E9C0000E6781E08093460990911F0B992321F0F7
:10E9D00010921F0B809345090E946F5FCC2051F06D
:10E9E00081E08093DE0D40E050E0BA0183E49FE7D0
:10E9F0000E94DC500E9444F880E1E1E2F5E0A5E3EA
:10EA0000B9E001900D928A95E1F720E030E0A9018C
:10EA1000F50160817181828193810F9409018823BE
:10EA200001F10E94F369F501208131814281538116
:10EA300060913109709132098091330990913409C4
:10EA40000F94420560933109709332098093330922
:10EA50009093340960E070E080E792E467DC0E9404
:10EA600044F8F40180809180A280B38020E030E0FF
:10EA7000A901C501B4010F9468071816FCF480E0E1
:10EA800090E0A0EAB0E489839A83AB83BC83A501BC
:10EA900094016091290570912A0580912B05909130
:10EAA0002C050F9442056D837E838F839887BE016A
:10EAB0006F5F7F4FCE0105960E94EC6980E090E089
:10EAC000A8ECB2E489839A83AB83BC839E012F5F59
:10EAD0003F4F49E255E0B201C3010E940C6920E0BA
:10EAE00030E0A901F80160817181828193810F94E6
:10EAF0000901882379F1CC2069F081E08093DE0D53
:10EB000040E050E0BA0182EB9EE70E94DC5080E0DA
:10EB10000E94D5E80E94F369F80120813181428189
:10EB2000538160913109709132098091330990913C
:10EB300034090F9442056093310970933209809330
:10EB400033099093340960E070E080E291E4EEDBF9
:10EB50000E9444F8CC2051F081E08093DE0D40E02B
:10EB600050E0BA018FEF9CE70E94DC5061E08E2DEF
:10EB70000E947C6780E00E94D5E80E9464E864E619
:10EB800070E080E090E00E9448C40E941050DC01D8
:10EB9000CB0188539045AF4FBF4F8093620E909347
:10EBA000630EA093640EB093650E10928A0A0E94C1
:10EBB0001050DC01CB0188539045AF4FBF4F80937D
:10EBC000660E9093670EA093680EB093690E109234
:10EBD0008B0AFF24F3948F2D28960FB6F894DEBF8E
:10EBE0000FBECDBFDF91CF911F910F91FF90EF909E
:10EBF000CF90BF90AF909F908F907F906F905F90DD
:10EC00004F900895AF92BF92CF92DF92EF92FF9212
:10EC10001F93CF93DF9300D01F92CDB7DEB77C0157
:10EC20005B01D42E10918A0A1092620E1092630E2C
:10EC30001092640E1092650E10928A0A80E00E9473
:10EC400016CE90918B0A192B1092660E1092670EB9
:10EC50001092680E1092690E10928B0A81E00E9449
:10EC600016CE11110E940E6761E08D2D0E947C6707
:10EC70000E94F36920E030E0A901F7016081718111
:10EC8000828193810F940901882309F445C01123DF
:10EC900051F081E08093DE0D40E050E0BA018FEF4B
:10ECA0009CE70E94DC5081E08093F10D8091F10D92
:10ECB000882351F0112341F060E08D2D0E947C6784
:10ECC00081E00E94D5E8F2CF81E08093DE0D40E044
:10ECD00050E0BA018EE69CE70E94DC50F7012081EB
:10ECE0003181428153816091310970913209809163
:10ECF0003309909134090F94420560933109709360
:10ED00003209809333099093340960E070E080EC1D
:10ED100090E40CDB0E9444F8F501C080D180E280D1
:10ED2000F38011E020E030E0A901C701B6010F94A3
:10ED30006807181624F51093DE0D40E050E0BA0184
:10ED40008DED9BE70E94DC50A7019601609131098F
:10ED50007091320980913309909134090F944205E2
:10ED60006093310970933209809333099093340989
:10ED700060E070E080E490E4D9DA0E9444F81092F8
:10ED8000F10D1093DE0D1092EC0940E050E0BA0155
:10ED900084ED9FE70E94DC508091EC09811104C052
:10EDA00081E00E94D5E8F8CFC12CD12C98E4E92E5F
:10EDB00092E4F92E813009F4B5CF11E01093DE0D05
:10EDC00040E050E0BA018DE69BE70E94DC50809164
:10EDD000410990914209A0914309B091440980935F
:10EDE0002D0590932E05A0932F05B09330058093A9
:10EDF000310990933209A0933309B09334090E94EA
:10EE00002A5F80E090E0A8ECB2E489839A83AB8328
:10EE1000BC839E012F5F3F4F49E255E069E379E0F3
:10EE200085E399E00E940C6980E090E0A0EAB0E4FC
:10EE300089839A83AB83BC83BE016F5F7F4F8DE371
:10EE400099E00E94EC690E94175680914509882339
:10EE500039F08091200B811110931F0B10924509FE
:10EE6000109246090F900F900F900F90DF91CF9165
:10EE70001F91FF90EF90DF90CF90BF90AF900895DB
:10EE8000CF92DF92EF92FF920F931F93CF93DF9376
:10EE900000D01F92CDB7DEB78091FC049091FD04A5
:10EEA000A091FE04B091FF04B7FF08C01092FC04CB
:10EEB0001092FD041092FE041092FF048091000550
:10EEC00090910105A0910205B09103054091FC04C9
:10EED0005091FD046091FE047091FF048417950722
:10EEE000A607B70744F48093FC049093FD04A09315
:10EEF000FE04B093FF0480911202882379F14091BF
:10EF0000FC045091FD046091FE047091FF04809117
:10EF1000040590910505A0910605B09107056A01C9
:10EF20007B01C80ED91EEA1EFB1EC701B6010F9455
:10EF30000D0120E030E048EC52E40F946E0169834B
:10EF40007A838B839C83CE0101960E94C1C2BC014F
:10EF500080910A0590910B050E9432568091F00D28
:10EF600010910C05811106C01123E1F1809112026C
:10EF70008823C1F14091FC045091FD046091FE048E
:10EF80007091FF048091040590910505A0910605FC
:10EF9000B09107056A017B01C80ED91EEA1EFB1E4F
:10EFA000C701B6010F940D0120E030E048EC52E4B7
:10EFB0000F946E010F948B06E0910805F0910905FE
:10EFC000309721F06083718382839383112329F02A
:10EFD000E0910D05F0910E0519958091F00D8111CC
:10EFE0000E941D568091F00D882329F0E0910D05B7
:10EFF000F0910E0519950F900F900F900F90DF91E3
:10F00000CF911F910F91FF90EF90DF90CF900895D7
:10F01000CF92DF92EF92FF920F931F93CF93DF93E4
:10F0200000D01F92CDB7DEB78091FC049091FD0413
:10F03000A091FE04B091FF04B7FF08C01092FC0439
:10F040001092FD041092FE041092FF0480910005BE
:10F0500090910105A0910205B09103054091FC0437
:10F060005091FD046091FE047091FF048417950790
:10F07000A607B70744F48093FC049093FD04A09383
:10F08000FE04B093FF0480911202882379F140912D
:10F09000FC045091FD046091FE047091FF04809186
:10F0A000040590910505A0910605B09107056A0138
:10F0B0007B01C80ED91EEA1EFB1EC701B6010F94C4
:10F0C0000F0120E030E048EC52E40F946E016983B8
:10F0D0007A838B839C83CE0101960E94C1C2BC01BE
:10F0E00080910A0590910B050E9432568091F00D97
:10F0F00010910C05811106C01123D1F180911202EB
:10F100008823B1F14091FC045091FD046091FE040C
:10F110007091FF048091040590910505A09106056A
:10F12000B09107056A017B01C80ED91EEA1EFB1EBD
:10F13000C701B6010F940F0120E030E048EC52E423
:10F140000F946E01E0910805F0910905309721F0C8
:10F150006083718382839383112329F0E0910D05ED
:10F16000F0910E0519958091F00D81110E941D56A8
:10F170000F900F900F900F90DF91CF911F910F91F3
:10F18000FF90EF90DF90CF900895CF92DF92EF92B3
:10F19000FF920F931F93CF93DF9300D01F92CDB7B1
:10F1A000DEB78091FC049091FD04A091FE04B09123
:10F1B000FF04B7FF08C01092FC041092FD041092E7
:10F1C000FE041092FF048091000590910105A0912A
:10F1D0000205B09103054091FC045091FD0460913B
:10F1E000FE047091FF0484179507A607B70744F43F
:10F1F0008093FC049093FD04A093FE04B093FF045D
:10F2000080911202882379F14091FC045091FD0411
:10F210006091FE047091FF048091040590910505B2
:10F22000A0910605B09107056A017B01C80ED91EA1
:10F23000EA1EFB1EC701B6010F940F012AE037ED4D
:10F2400043E25CE30F946E0169837A838B839C8332
:10F25000CE0101960E948BC1BC0180910A0590915C
:10F260000B050E9432568091F00D10910C05811112
:10F2700006C01123D1F1809112028823B1F140918F
:10F28000FC045091FD046091FE047091FF04809194
:10F29000040590910505A0910605B09107056A0146
:10F2A0007B01C80ED91EEA1EFB1EC701B6010F94D2
:10F2B0000F012AE037ED43E25CE30F946E01E09129
:10F2C0000805F0910905309721F0608371838283EE
:10F2D0009383112329F0E0910D05F0910E05199506
:10F2E0008091F00D81110E941D568091F00D8823B0
:10F2F00029F0E0910D05F0910E0519950F900F90F2
:10F300000F900F90DF91CF911F910F91FF90EF9091
:10F31000DF90CF900895CF92DF92EF92FF920F93FC
:10F320001F93CF93DF9300D01F92CDB7DEB78091AC
:10F33000FC049091FD04A091FE04B091FF04B7FF7E
:10F3400008C01092FC041092FD041092FE0410926A
:10F35000FF048091000590910105A0910205B091F4
:10F3600003054091FC045091FD046091FE047091EE
:10F37000FF0484179507A607B70744F48093FC049D
:10F380009093FD04A093FE04B093FF0480911202B9
:10F39000882379F14091FC045091FD046091FE04B2
:10F3A0007091FF048091040590910505A0910605D8
:10F3B000B09107056A017B01C80ED91EEA1EFB1E2B
:10F3C000C701B6010F940F012AE037ED43E25CE379
:10F3D0000F946E0169837A838B839C83CE0101969F
:10F3E0000E9440C2BC0180910A0590910B050E94C9
:10F3F00032568091F00D10910C05811106C0112339
:10F40000D1F1809112028823B1F14091FC04509116
:10F41000FD046091FE047091FF04809104059091B9
:10F420000505A0910605B09107056A017B01C80E8C
:10F43000D91EEA1EFB1EC701B6010F940F012AE078
:10F4400037ED43E25CE30F946E01E0910805F09123
:10F450000905309721F060837183828393831123A0
:10F4600029F0E0910D05F0910E0519958091F00DB0
:10F4700081110E941D560F900F900F900F90DF91F9
:10F48000CF911F910F91FF90EF90DF90CF90089553
:10F490000F931F93CF938091FC049091FD04A09152
:10F4A000FE04B091FF04B7FF08C01092FC04109254
:10F4B000FD041092FE041092FF04809100059091CB
:10F4C0000105A0910205B09103054091FC04509103
:10F4D000FD046091FE047091FF0484179507A60750
:10F4E000B70744F48093FC049093FD04A093FE04BA
:10F4F000B093FF0480911202882331F14091FC0403
:10F500005091FD046091FE047091FF048091040508
:10F5100090910505A0910605B09107058A019B0110
:10F52000080F191F2A1F3B1FC901B8010F940F01B3
:10F530000F948606CB010E9412C4BC0180910A057B
:10F5400090910B050E9432568091F00DC0910C05F0
:10F55000811106C0CC23A1F180911202882381F190
:10F560004091FC045091FD046091FE047091FF04F1
:10F570008091040590910505A0910605B0910705BD
:10F580008A019B01080F191F2A1F3B1FC901B801DF
:10F590000F940F01E0910805F0910905309721F0D3
:10F5A0006083718382839383CC2329F0E0910D05DE
:10F5B000F0910E0519958091F00D81110E941D5654
:10F5C0008091F00DCF911F910F91089561CF60DF71
:10F5D000882329F0E0910D05F0910E051994089506
:10F5E0008091FC049091FD04A091FE04B091FF0471
:10F5F000B7FF08C01092FC041092FD041092FE04A4
:10F600001092FF048091000590910105A0910205E0
:10F61000B09103054091FC045091FD046091FE04FB
:10F620007091FF0484179507A607B70744F48093E9
:10F63000FC049093FD04A093FE04B093FF0480911A
:10F640001202882399F020910405309105058091DC
:10F65000FC049091FD04820F931F0E9412C4BC0110
:10F6600080910A0590910B050E9432568091F00D11
:10F6700020910C05811106C0222311F18091120204
:10F680008823F1F040910405509105058091FC0418
:10F690009091FD04840F951FE0910805F0910905F4
:10F6A000309711F091838083222329F0E0910D059A
:10F6B000F0910E0519958091F00D81110E941D5653
:10F6C0008091F00D08958CCF8BDF882329F0E09195
:10F6D0000D05F0910E0519940895CF93DF931092C4
:10F6E000E90D8091FC049091FD04A091FE04B0917D
:10F6F000FF0481309048A105B10540F01092FC0450
:10F700001092FD041092FE041092FF04C091FC04BC
:10F710008091F70918160CF5282F082E000C330BD2
:10F72000255031094C2F0C2E000C550B4217530756
:10F73000A4F085301CF0CBEFC80F01C0C0E08C2FC7
:10F740000C2E000C990BAA0BBB0B8093FC0490931E
:10F75000FD04A093FE04B093FF04C093F609D0E02B
:10F76000C11109C0809112028823E9F021E041E033
:10F7700062EA7BE115C0C13049F48091120288230E
:10F7800091F020E041E063E97BE10AC0C23059F426
:10F7900080911202882339F020E041E069E87BE1A2
:10F7A0008D2F0E94D65FDF5FCF5FD530C9F683E033
:10F7B0008093F709DF91CF9108951F93CF93DF9343
:10F7C0001092E90D8091FC049091FD04A091FE043B
:10F7D000B091FF0481309048A105B10540F010922E
:10F7E000FC041092FD041092FE041092FF04C091DC
:10F7F000FC048091F50918160CF5282F082E000C32
:10F80000330B255031094C2F0C2E000C550B421791
:10F810005307A4F085301CF0CBEFC80F01C0C0E047
:10F820008C2F0C2E000C990BAA0BBB0B8093FC04A5
:10F830009093FD04A093FE04B093FF04C093F609D7
:10F84000D0E012E0C11109C0809112028823D9F1E1
:10F8500021E041E06CE77BE115C0C13049F48091C3
:10F860001202882381F120E041E063E77BE10AC0D6
:10F87000C23061F480911202882329F120E041E036
:10F8800062E67BE18D2F0E94D65F1DC0C33049F434
:10F89000809112028823B9F020E041E060E67BE12C
:10F8A000F1CFC43081F480911202882351F021E01D
:10F8B00040E065E57BE18D2F0E94D65F8D2F0E9491
:10F8C000805710931202DF5FCF5FD53009F0BACFB7
:10F8D000D093F509DF91CF911F9108951F93CF9396
:10F8E000DF931092E90D8091FC049091FD04A091AA
:10F8F000FE04B091FF0481309048A105B10540F0AD
:10F900001092FC041092FD041092FE041092FF0469
:10F91000C091FC048091F40918160CF5282F082ECC
:10F92000000C330B255031094C2F0C2E000C550BBD
:10F9300042175307A4F085301CF0CBEFC80F01C06D
:10F94000C0E08C2F0C2E000C990BAA0BBB0B8093E4
:10F95000FC049093FD04A093FE04B093FF04C093B5
:10F96000F609D0E012E0C11109C08091120288238B
:10F97000D9F121E041E068E47BE115C0C13049F4F0
:10F9800080911202882381F120E041E06FE37BE166
:10F990000AC0C23061F480911202882329F120E06C
:10F9A00041E061E37BE18D2F0E94D65F1DC0C33033
:10F9B00049F4809112028823B9F020E041E06FE21F
:10F9C0007BE1F1CFC43081F480911202882351F0A1
:10F9D00021E040E064E27BE18D2F0E94D65F8D2F15
:10F9E0000E94805710931202DF5FCF5FD53009F07D
:10F9F000BACFD093F409DF91CF911F9108951F934F
:10FA0000CF93DF931092E90D8091FC049091FD0457
:10FA1000A091FE04B091FF0481309048A105B1058A
:10FA200040F01092FC041092FD041092FE0410921B
:10FA3000FF04C091FC048091F30918160CF5282FDF
:10FA4000082E000C330B255031094C2F0C2E000CC6
:10FA5000550B42175307A4F085301CF0CBEFC80FAD
:10FA600001C0C0E08C2F0C2E000C990BAA0BBB0B15
:10FA70008093FC049093FD04A093FE04B093FF04D4
:10FA8000C093F609D0E012E0C11109C080911202C2
:10FA90008823D9F121E041E067E17BE115C0C13065
:10FAA00049F480911202882381F120E041E067E06F
:10FAB0007BE10AC0C23061F480911202882329F1EF
:10FAC00020E041E066EF7AE18D2F0E94D65F1DC0F5
:10FAD000C33049F4809112028823B9F020E041E05C
:10FAE00067EE7AE1F1CFC43081F48091120288236D
:10FAF00051F021E040E06CED7AE18D2F0E94D65F5D
:10FB00008D2F0E94805710931202DF5FCF5FD53098
:10FB100009F0BACFD093F309DF91CF911F910895E7
:10FB20001F93CF93DF931092E90D8091FC04909185
:10FB3000FD04A091FE04B091FF0481309048A1051E
:10FB4000B10540F01092FC041092FD041092FE04E6
:10FB50001092FF04C091FC048091F20918160CF574
:10FB6000282F082E000C330B255031094C2F0C2E5A
:10FB7000000C550B42175307A4F085301CF0CBEF57
:10FB8000C80F01C0C0E08C2F0C2E000C990BAA0BE3
:10FB9000BB0B8093FC049093FD04A093FE04B093F0
:10FBA000FF04C093F609D0E012E0C11109C08091B2
:10FBB00012028823D9F121E041E06FEC7AE115C00F
:10FBC000C13049F480911202882381F120E041E0A4
:10FBD0006FEB7AE10AC0C23061F48091120288238F
:10FBE00029F120E041E062EB7AE18D2F0E94D65F9F
:10FBF0001DC0C33049F4809112028823B9F020E07F
:10FC000041E060EB7AE1F1CFC43081F480911202DF
:10FC1000882351F021E040E065EA7AE18D2F0E94CF
:10FC2000D65F8D2F0E94805710931202DF5FCF5F47
:10FC3000D53009F0BACFD093F209DF91CF911F915F
:10FC400008951F93CF93DF931092E90D8091FC04E8
:10FC50009091FD04A091FE04B091FF048130904882
:10FC6000A105B10540F01092FC041092FD04109221
:10FC7000FE041092FF04C091FC048091F109181653
:10FC80000CF5282F082E000C330B255031094C2F72
:10FC90000C2E000C550B42175307A4F085301CF0B6
:10FCA000CBEFC80F01C0C0E08C2F0C2E000C990BBD
:10FCB000AA0BBB0B8093FC049093FD04A093FE045D
:10FCC000B093FF04C093F609D0E012E0C11109C05F
:10FCD000809112028823D9F121E041E068E97AE1BC
:10FCE00015C0C13049F480911202882381F120E0CF
:10FCF00041E069E87AE10AC0C23061F48091120201
:10FD0000882329F120E041E06AE77AE18D2F0E9403
:10FD1000D65F1DC0C33049F4809112028823B9F028
:10FD200020E041E068E77AE1F1CFC43081F48091CE
:10FD30001202882351F021E040E06DE67AE18D2F38
:10FD40000E94D65F8D2F0E94805710931202DF5FB2
:10FD5000CF5FD53009F0BACFD093F109DF91CF91C1
:10FD60001F9108951F93CF93DF931092E90D809117
:10FD7000FC049091FD04A091FE04B091FF04813039
:10FD80009048A105B10540F01092FC041092FD04CA
:10FD90001092FE041092FF04C091FC048091F009BF
:10FDA00018160CF5282F082E000C330B255031099E
:10FDB0004C2F0C2E000C550B42175307A4F0853026
:10FDC0001CF0CBEFC80F01C0C0E08C2F0C2E000C34
:10FDD000990BAA0BBB0B8093FC049093FD04A0939A
:10FDE000FE04B093FF04C093F609D0E012E0C11105
:10FDF00009C0809112028823D9F121E041E060E638
:10FE00007AE115C0C13049F480911202882381F152
:10FE100020E041E067E57AE10AC0C23061F48091F8
:10FE20001202882329F120E041E067E47AE18D2F76
:10FE30000E94D65F1DC0C33049F48091120288230E
:10FE4000B9F020E041E065E47AE1F1CFC43081F41B
:10FE500080911202882351F021E040E06AE37AE1C8
:10FE60008D2F0E94D65F8D2F0E9480571093120213
:10FE7000DF5FCF5FD53009F0BACFD093F009DF91C3
:10FE8000CF911F9108951F93CF93DF931092E90DA7
:10FE90008091FC049091FD04A091FE04B091FF04B8
:10FEA00081309048A105B10540F01092FC041092F9
:10FEB000FD041092FE041092FF04C091FC04809196
:10FEC000EF0918160CF5282F082E000C330B2550BF
:10FED00031094C2F0C2E000C550B42175307A4F080
:10FEE00085301CF0CBEFC80F01C0C0E08C2F0C2E6A
:10FEF000000C990BAA0BBB0B8093FC049093FD04A0
:10FF0000A093FE04B093FF04C093F609D0E012E082
:10FF1000C11109C0809112028823D9F121E041E08A
:10FF20006DE27AE115C0C13049F480911202882354
:10FF300081F120E041E06EE17AE10AC0C23061F473
:10FF400080911202882329F120E041E06EE07AE1FD
:10FF50008D2F0E94D65F1DC0C33049F480911202DC
:10FF60008823B9F020E041E067E07AE1F1CFC430C6
:10FF700081F480911202882351F021E040E06CEF7F
:10FF800079E18D2F0E94D65F8D2F0E9480571093AC
:10FF90001202DF5FCF5FD53009F0BACFD093EF09FF
:10FFA000DF91CF911F910895FF920F931F93CF93ED
:10FFB000DF931092E90D8091FC049091FD04A091D3
:10FFC000FE04B091FF0481309048A105B10540F0D6
:10FFD0001092FC041092FD041092FE041092FF0493
:10FFE000C091FC048091EE091816DCF4282F082E2D
:10FFF000000C330B215031094C2F0C2E000C550BEB
:020000021000EC
:100000004217530774F0CFEFC80F8C2F90E0A0E099
:10001000B0E08093FC049093FD04A093FE04B093A1
:10002000FF041092ED098091F609C81714F4C093EB
:10003000F6098091F609082E000C990B04962C2FD6
:100040000C2E000C330B8217930724F48CEF8C0FCB
:100050008093F6091091F609D0E081E001E092E08A
:10006000F92E111125C08823B1F01C16A4F080913F
:10007000FC049091FD04A091FE04B091FF04019650
:10008000A11DB11D8093FC049093FD04A093FE0478
:10009000B093FF04CF5F80911202882309F442C01D
:1000A00020E041E06CEE79E18D2F0E94D65F3AC0EE
:1000B0001130D1F48091F00D811105C080911202B0
:1000C000882381F109C0C130C9F7F092EC09809111
:1000D000ED09882399F32FC081E0C13009F080E059
:1000E00020E24FED59E11BC01230E1F48091F00D98
:1000F000811105C0809112028823A1F009C0C2308D
:10010000C9F70093EC098091ED09882399F313C096
:1001100081E0C23009F080E020E242ED59E16D2F2C
:100120000E9425C5DF5F1F5F80E0D53009F099CFC1
:1001300083E08093EE09DF91CF911F910F91FF90A3
:1001400008956F927F928F929F92AF92BF92CF92BB
:10015000DF92EF92FF920F931F93CF93DF9300D024
:100160001F92CDB7DEB76C013B01470158012983CF
:100170003A834B835C830E94BC5083E080931202DD
:10018000D0920B05C0920A0570920905609208058D
:1001900029813A814B815C81CA01B9010F9486069D
:1001A00060930405709305058093060590930705F9
:1001B0000F940F016B017C019B01AC01C501B401DF
:1001C0000F9441050F948606609300057093010516
:1001D0008093020590930305A7019601F3016081C6
:1001E0007181828193810F9441050F948B066093F6
:1001F000FC047093FD048093FE049093FF0486EE4C
:100200009AE790931102809310020F900F900F9035
:100210000F90DF91CF911F910F91FF90EF90DF90A2
:10022000CF90BF90AF909F908F907F906F900895E8
:10023000CF92DF92EF92FF920F931F93CF93DF93B2
:100240008C01EB016A0179010E94BC5023E02093EC
:10025000120210930B0500930A05D0930905C09371
:100260000805A601DD0C660B770B4093040550933F
:1002700005056093060570930705C701FF0CAA0BDF
:10028000BB0B841B950BA60BB70B809300059093BB
:100290000105A0930205B093030588819981092E79
:1002A000000CAA0BBB0B841B950BA60BB70B809302
:1002B000FC049093FD04A093FE04B093FF0483E636
:1002C0009BE79093110280931002DF91CF911F91D1
:1002D0000F91FF90EF90DF90CF900895EF92FF92F3
:1002E0000F931F93CF937C018B01C42F80E20E9458
:1002F0004B72CF3F11F084E501C082E40E944B7243
:10030000C7FD04C080E38C0F0E944B728AE30E94F9
:100310004B72F701608171818281938142E00E947A
:100320002473F801408151816281738183ED9BE1E7
:10033000CF911F910F91FF90EF900C9406C10F93F6
:100340001F93CF93DF93823048F1C82FE4EFF2E29E
:1003500084918F010F5F1F4F882321F00E944B7201
:10036000F801F6CF84E50E944B726C2F70E080E0BC
:1003700090E04AE00E94A47280E20E944B72C1E0C9
:10038000D3E08991882319F00E944B72FACF8AE05A
:10039000DF91CF911F910F910C944B72DF91CF9110
:1003A0001F910F910C9431E681E0809378021092B6
:1003B0004A0583E50E94B749811102C00C9423ECE1
:1003C0000E9475498823D1F30895CF93DF93E5EF19
:1003D000F6E18491EF012196882321F00E944B726F
:1003E000FE01F7CFE8EFFDE18491EF01219688232C
:1003F00021F00E944B72FE01F7CFDF91CF9108955B
:100400000F931F93CF9383E50E94E649882309F455
:1004100047C00E946449813039F0823009F040C001
:100420000EE413E0C0E021C00EE413E0C0E0F801E8
:1004300081918F010E94E649882339F00E94644926
:100440004FEF682F8C2F0E9414F7CF5FC43079F7DD
:1004500082E40E94E649882319F10E9464494FEF23
:10046000682F1BC0CF5FC43079F0F80181918F01F4
:100470000E94E6498823B1F30E946449482F6FEF38
:100480008C2F0E9414F7EECF82E40E94E649882365
:1004900039F00E946449482F6FEF84E00E9414F7FE
:1004A000CF911F910F910C945CF60F931F93CF93F4
:1004B00083E50E94B749811104C00EE413E0C0E057
:1004C0000EC0C0E00E946449682F8C2F0E94BEF7C6
:1004D000CF5FC530B9F7F1CFCF5FC43071F0F8010D
:1004E00081918F010E94B7498823B1F30E9464492A
:1004F000682F8C2F0E94BEF7EFCF82E40E94B7498D
:10050000882331F00E946449682F84E00E94BEF77E
:10051000CF911F910F910C945CF6CF93DF9383E5FD
:100520000E94E649882321F00E945449EB0102C051
:10053000C0E0D0E080E50E94E649882321F00E94D7
:100540005449CB0102C080E090E0BE01DF91CF9121
:100550000C94D5F70F931F93CF930EE413E0C0E0F4
:10056000F80181918F010E94B749882329F00E94E8
:1005700054498C2F0E94E4F7CF5FC43089F782E49E
:100580000E94B749882329F00E94544984E00E94C0
:10059000E4F783E50E94B749882349F0C0E00E9450
:1005A00054498C2F0E94E4F7CF5FC530C1F7CF913B
:1005B0001F910F910895BF92CF92DF92EF92FF9219
:1005C0000F931F93CF93DF93CDB7DEB76C970FB622
:1005D000F894DEBF0FBECDBF0E948D5E882319F058
:1005E00081E00E94FD6984E50E94B749811103C042
:1005F000DD24DA940BC00E946449D0904605D816D9
:10060000B9F321E040E050E0BA0199DE85E40E94B0
:10061000B749882319F00E94844904C060E070E063
:1006200080E090EC6D8B7E8B8F8B988F8AE50E949B
:10063000E649882319F00E94844904C060E070E014
:1006400080E291E4698B7A8B8B8B9C8B88E50E948E
:10065000E649882319F00E94844904C060E070E0F4
:1006600080E291E46D877E878F87988B89E50E9471
:10067000E649882319F00E94844904C060E070E0D4
:1006800085E893E469877A878B879C8785E50E9454
:10069000B749882319F00E94844904C060E070E0E3
:1006A00088EC92EC6D837E838F8398878CE40E9424
:1006B000B749882319F00E94844903C060E070E0C4
:1006C000CB0169837A838B839C8382E40E94E64911
:1006D000882321F00E945449F62E02C085E0F82EAE
:1006E000B090100B809146098111A3C0CC24C39413
:1006F000EF2C8E010B5F1F4F9E01275F3F4FAE0116
:10070000435F5F4FBE016F5E7F4FCE0145960E94F3
:100710007D74882309F48DC081E08093F10D11E090
:100720008091F10D882309F470C060E08F2D0E9444
:100730007C6780918A0A90918B0A911103C088236B
:1007400009F45FC01093DE0D40E050E0BA0180E98B
:100750009DE70E94DC508091F10D882321F081E01B
:100760000E94D5E8F8CF1092620E1092630E10929C
:10077000640E1092650E10928A0A0E9416CE109294
:10078000660E1092670E1092680E1092690E10920B
:100790008B0A81E00E9416CE0E940E671093DE0D38
:1007A00040E050E0BA018FEF9CE70E94DC500E94CD
:1007B0001050DC01CB0188539045AF4FBF4F809361
:1007C000620E9093630EA093640EB093650E109228
:1007D0008A0A0E941050DC01CB0188539045AF4F2C
:1007E000BF4F8093660E9093670EA093680EB093F0
:1007F000690E10928B0A1093F10D61E08F2D0E940B
:100800007C6781E00E94D5E88BCF80E090E0A8E48F
:10081000B2E4898F9A8FAB8FBC8F80914609882371
:1008200041F04F2DBE01675E7F4FCE0101960E94C1
:10083000027621E040E050E0BA018D2D80DD81E0BC
:10084000B81202C00E94535E6C960FB6F894DEBFD9
:100850000FBECDBFDF91CF911F910F91FF90EF9011
:10086000DF90CF90BF90089588E893E19093C013F4
:100870008093BF1380916F008D7F80936F00909164
:10088000F00A8091F10A981719F00E94F5DDF7CF70
:100890001092FF0D1092FE0D80916F008260809388
:1008A0006F008FB7F8941092DA0D1092DB0D109252
:1008B000DC0D1092DD0D8FBF0E9444F880E00E9495
:1008C00027F86093F8097093F9098093FA099093D7
:1008D000FB0981E00E9427F86093FC097093FD09F1
:1008E0008093FE099093FF0982E00E9427F86093AD
:1008F000000A7093010A8093020A9093030A8CE025
:10090000E8EFF9E0A1E2B5E001900D928A95E1F7F8
:100910000C943A49CF93DF93E0E0FDE18491EF013D
:100920002196882321F00E944B72FE01F7CFE2EF5F
:10093000FCE18491EF012196882321F00E944B7203
:10094000FE01F7CFEBEDFCE18491EF0121968823C6
:1009500021F00E944B72FE01F7CFEBECFCE1849199
:10096000EF012196882321F00E944B72FE01F7CF00
:10097000EAEBFCE18491EF012196882321F00E94AB
:100980004B72FE01F7CFE9EAFCE18491EF01219679
:10099000882321F00E944B72FE01F7CFEAE9FCE1C7
:1009A0008491EF012196882321F00E944B72FE0171
:1009B000F7CFE5E8FCE18491EF012196882321F04F
:1009C0000E944B72FE01F7CFEFE6FCE18491EF014C
:1009D0002196882321F00E944B72FE01F7CFEAE5B1
:1009E000FCE18491EF012196882321F00E944B7253
:1009F000FE01F7CFEDE3FCE18491EF01219688231E
:100A000021F00E944B72FE01F7CFE5E2FCE18491F8
:100A1000EF012196882321F00E944B72FE01F7CF4F
:100A2000DF91CF9108954F925F926F927F928F9254
:100A30009F92AF92BF92CF92DF92EF92FF92CF93AD
:100A4000DF93E2E2FCE18491EF012196882321F01B
:100A50000E944B72FE01F7CF609121057091220533
:100A6000809123059091240542E00E942473EEE1D9
:100A7000FCE18491EF012196882321F00E944B72C2
:100A8000FE01F7CF6091250570912605809127051D
:100A90009091280542E00E942473EAE1FCE18491F0
:100AA000EF012196882321F00E944B72FE01F7CFBF
:100AB0006091290570912A0580912B0590912C0554
:100AC00042E00E942473E6E1FCE18491EF0121966B
:100AD000882321F00E944B72FE01F7CF60912D0513
:100AE00070912E0580912F059091300542E00E9473
:100AF00024738FB7F89440901105509012056090C0
:100B00001305709014058090150590901605A0901F
:100B10001705B0901805C0901905D0901A05E090FF
:100B20001B05F0901C058FBFECE0FCE18491EF0108
:100B30002196882321F00E944B72FE01F7CFC3015A
:100B4000B2010E940A73E8E0FCE18491EF01219672
:100B5000882321F00E944B72FE01F7CFC501B4013A
:100B60000E940A73E4E0FCE18491EF01219688235E
:100B700021F00E944B72FE01F7CFC701B6010E941F
:100B80000A738AE0DF91CF91FF90EF90DF90CF90D2
:100B9000BF90AF909F908F907F906F905F904F909D
:100BA0000C944B72CF93DF9383E50E94E649882330
:100BB00021F00E945449EB0102C0C0E0D0E0DD27E3
:100BC000C230D105BCF0E5EFF6E18491EF0121964A
:100BD000882321F00E944B72FE01F7CFE2EEFBE189
:100BE0008491EF012196882309F450C00E944B7232
:100BF000FE01F6CF88E40E94E6498823A9F00E940E
:100C00005449683771053CF0633281E078072CF075
:100C100062E271E002C068E770E0FE01EE0FFF1FC4
:100C2000E75DFA4E7183608386E40E94E64988237B
:100C3000A9F00E945449FE01EE0FFF1FEF5DFA4E2E
:100C4000718360836F3F710519F014F06FEF70E0EE
:100C500077FF02C060E070E07183608382E40E94ED
:100C6000E649882399F00E9454496530710534F0B3
:100C7000683871052CF067E870E002C065E070E04C
:100C8000CC0FDD1FCB5DDA4E79836883DF91CF9186
:100C900008950F931F93CF93DF93CDB7DEB72897B7
:100CA0000FB6F894DEBF0FBECDBF00912E0410E04A
:100CB000F801EE0FFF1FE95EF54F60817181072E8D
:100CC000000C880B990B0F940F016D837E838F832B
:100CD0009887000F111F000F111FF801E452FB4FFE
:100CE00080819181A281B38189839A83AB83BC8304
:100CF0004EEFBE016B5F7F4FCE010196EFDA609140
:100D0000150A7091160A072E000C880B990B0F9488
:100D10000F016D837E838F8398878091E404909187
:100D2000E504A091E604B091E70489839A83AB833C
:100D3000BC834FEFBE016B5F7F4FCE010196CEDAD1
:100D40006091170A7091180A072E000C880B990BF6
:100D50000F940F016D837E838F8398878091DC04CD
:100D60009091DD04A091DE04B091DF0489839A8321
:100D7000AB83BC8340E0BE016B5F7F4FCE01019629
:100D8000ADDA6091190A70911A0A072E000C880BCF
:100D9000990B0F940F016D837E838F8398878091C9
:100DA000E0049091E104A091E204B091E30489830E
:100DB0009A83AB83BC8341E0BE016B5F7F4FCE0162
:100DC00001968CDAEEEDFBE184918F010F5F1F4FEE
:100DD000882321F00E944B72F801F6CFE0912E0497
:100DE000F0E0EB56F14F608170E080E090E00E940F
:100DF0000A73E9EDFBE184918F010F5F1F4F882398
:100E000021F00E944B72F801F6CF6091920E70E0D3
:100E100080E090E00E940A7360E070E086ED9BE164
:100E20000E944AC18AE30E944B726091950E70E065
:100E300080E090E00E940A7361E070E086ED9BE143
:100E40000E944AC18AE30E944B726091960E70E044
:100E500080E090E00E940A7328960FB6F894DEBFF7
:100E60000FBECDBFDF91CF911F910F9108951F93BA
:100E7000CF93DF9388E690E00E940672811156C0FE
:100E80008091070A83FD52C083E50E94E6498823CA
:100E900009F44CC00E94844910912E04C12FD0E067
:100EA000CC0FDD1FC95ED54F0F948606798368830A
:100EB000812F0E9416CE0E94844920E030E040E756
:100EC00052E40F94090118163CF00E9487BD60E0BF
:100ED0008EEB9BE10E94E1C50E948449C0912E04E3
:100EE000D0E0FE01EE0FFF1FEE0FFF1FE452FB4F9D
:100EF00020813181428153810F9468071816B4F420
:100F000084ED92E09F938F932196DF93CF938FEAA6
:100F10009BE19F938F931F920E94385E8DB79EB77F
:100F200007960FB6F8949EBF0FBE8DBFDF91CF918D
:100F30001F9108953F924F925F926F927F928F928E
:100F40009F92AF92BF92CF92DF92EF92FF920F9358
:100F50001F93CF93DF93CDB7DEB72C970FB6F894DE
:100F6000DEBF0FBECDBF5C01DC0159968D909C9019
:100F70005A97F40181859285A385B4859C01AD01C2
:100F80002F5F3F4F4F4F5F4F29873A874B875C87D3
:100F9000D5011496CD90DD90ED90FC901797C1147B
:100FA000D104E104F10439F0BFEFCB1ADB0AEB0AFC
:100FB000FB0A312C07C0F401C080D180E280F380AD
:100FC00033243394260137011D821E821F82188626
:100FD000F40181859285A385B4852D813E814F8161
:100FE0005885281739074A075B0708F064C08985C8
:100FF0009A85AB85BC858C159D05AE05BF0550F463
:1010000082E0C82ED12CE12CF12C92E0492E512CFB
:10101000612C712C9E012F5F3F4FB701A601C401C7
:101020000E9418B1882309F446C089819A81AB8156
:10103000BC81892B8A2B8B2B41F0260137019FEF36
:10104000491A590A690A790A05C0C414D504E60484
:10105000F70491F02D813E814F8158852F5F3F4FDE
:101060004F4F5F4F2D833E834F8358873FEFC31A07
:10107000D30AE30AF30AACCF0FEF1FEF2FEF3FE0E5
:10108000B301A201C4010E9487B0F82E882399F011
:10109000D50114964D915D916D917C9117974115F5
:1010A00051056105710549F093018201C4010E9457
:1010B00087B0811102C0F12C29C0D50114964D9240
:1010C0005D926D927C921797332051F0D301C2014B
:1010D0000196A11DB11DF40180839183A283B38386
:1010E000F50185899689A789B08D892B8A2B8B2B51
:1010F00069F4D50155964D925D926D927C92589708
:1011000011968C911197806811968C938F2D2C9647
:101110000FB6F894DEBF0FBECDBFDF91CF911F9108
:101120000F91FF90EF90DF90CF90BF90AF909F9086
:101130008F907F906F905F904F903F9008950F93A6
:101140001F93CF93DF938B010E941050EB010E94FD
:1011500044728F3F49F00E9410506C1B7D0B60174A
:101160007107A8F380E001C081E0DF91CF911F916A
:101170000F9108958F929F92AF92BF92CF92DF927C
:10118000EF92FF920F931F93CF93DF93EC018B812C
:10119000811102C080E077C009891A892B893C89B6
:1011A0000417150726073707A8F36A017B01823069
:1011B00029F4C886D986EA86FB860DC0C114D104FD
:1011C000E104F10451F41C821D821E821F821886E4
:1011D00019861A861B8681E056C088849984AA8461
:1011E000BB84E98DFA8D258530E0275F3F4FB5013F
:1011F000A4014150510961097109022E04C076957C
:101200006795579547950A94D2F7D701C60101977C
:10121000A109B10904C0B695A795979587952A9518
:10122000D2F784179507A607B70720F089288A28E0
:101230008B2849F44D895E896F89788D4C835D8355
:101240006E837F8304C0841B950BA60BB70B4C01E8
:101250005D018E010C5F1F4F81149104A104B10444
:1012600009F4A7CF4C815D816E817F819801898DC2
:101270009A8D0E9418B191E0891A9108A108B108CD
:101280008111EACF87CFDF91CF911F910F91FF900E
:10129000EF90DF90CF90BF90AF909F908F90089588
:1012A0000F931F93CF93DF93FC012381222311F02F
:1012B00080E044C08B01EC01FB018789803139F16A
:1012C0008032B1F783E08B83F801428D538D648DBA
:1012D000758D4D8B5E8B6F8B788F9E012F5E3F4F90
:1012E000C8010E9499B1882319F31A8F098F81E0F0
:1012F00089831C821D821E821F82188619861A8687
:101300001B861C861D861E861F86188A17C082E0D3
:101310008B831D8A1E8A1F8A188EFB01808D918DFA
:10132000A0E0B0E025E0880F991FAA1FBB1F2A95F7
:10133000D1F7898B9A8BAB8BBC8BD7CFDF91CF91B9
:101340001F910F910895CF93DF93EC0141E061115C
:1013500001C040E06C857D858E859F850E944FB0E1
:10136000882341F0888920E2829FC0011124855B97
:101370009A4F02C080E090E0DF91CF910895CF9323
:10138000DF93EC018B81882331F1898187FF1FC0B6
:1013900061E0CE01D8DFFC01892BE9F08081853E38
:1013A000D1F08B81823040F489899A89AB89BC89DC
:1013B000848F958FA68FB78F8D899E89AF89B88DC1
:1013C000938F828FB58BA48B89818F778983DF91EF
:1013D000CF910C940FB081E0888380E0DF91CF91B2
:1013E0000895CF93DF93EC01CADF1B82DF91CF9189
:1013F0000895CF93DF93EB01FC012381211102C0FB
:1014000080E027C02250223020F48FE288831982A6
:101410001FC060E098DF009799F3FC0190E080E046
:101420002EE23081303269F0883029F4DE01A90FD4
:10143000B11D2C939F5F3081DE01A90FB11D3C933C
:101440009F5F8F5F31968B3061F7C90FD11D188276
:1014500081E0DF91CF91089561E0FC0180810C94DF
:10146000DF4E8EBD0DB407FEFDCF0895CF92DF9203
:10147000EF92FF921F93CF93DF9300D01F92CDB7CF
:10148000DEB76C01162FFC019281892F806A869548
:101490008CBD90FD03C081E0963009F480E08DBDE5
:1014A00060E0F601808129833A834B835C830E944C
:1014B000DF4E6CE271E0C60142DE812F8064D1DF35
:1014C00088E1E82EF12C5C814B813A812981DA0197
:1014D000C9010E2C04C0B695A795979587950A94D7
:1014E000D2F729833A834B835C83BBDFF8E0EF1AA2
:1014F000F10829813A814B815C8188EFE8168FEFF2
:10150000F80629F7112321F0183021F08FEF03C0DE
:1015100085E901C087E8A5DF1C3011F40E94447200
:1015200010E00E944472F601838387FF04C01F3FCE
:1015300011F01F5FF6CF0F900F900F900F90DF917B
:10154000CF911F91FF90EF90DF90CF9008950F9370
:101550001F93CF93DF93EC0189018C81833039F0A5
:1015600089E0440F551F661F771F8A95D1F79A01AE
:10157000AB0168E1CE017ADF882311F086E030C04C
:101580008EEF8EBD80E090E00DB407FEFDCFF80138
:10159000E80FF91F20812EBD0DB407FEFDCF21817C
:1015A0002EBD0296811522E0920771F70DB407FE59
:1015B000FDCF8FEF56DF8FEF54DF0E9444728B8395
:1015C0008F71853029F083E18983CE0145DF09C021
:1015D00068E572E0CE01B3DD182F811106C087E106
:1015E0008983CE0139DF10E010C020E030E0A9018E
:1015F0006DE0CE013BDF811104C00E94447288235C
:1016000011F086E1EDCFCE0127DF812FDF91CF9161
:101610001F910F9108952F923F924F925F926F9278
:101620007F928F929F92AF92BF92CF92DF92EF9272
:10163000FF920F931F93CF93DF9300D01F92CDB7EC
:10164000DEB78C014B011A01DC0113968C911397C4
:101650008130C1F411968C9181FF14C082FF18C0B3
:10166000F801418952896389748980859185A285B1
:10167000B38584179507A607B70751F0C8017ADD2F
:10168000811106C081E0F80180838FEF9FEF2DC1AB
:10169000610184C0D80159968D919C915A97FC01A3
:1016A000248121502A013B0139E0769467945794B4
:1016B00047943A95D1F7722E74207A01F1E0FF2217
:1016C000772009F477C080E092E08E199F095601D7
:1016D0008C159D0508F45C01D80159962D913C911B
:1016E0005A9714968D919D910D90BC91A02D0297C3
:1016F000A109B109F901058404C0880F991FAA1F27
:10170000BB1F0A94D2F74685578560897189840F7B
:10171000951FA61FB71F9C01AD01270D311D411D4F
:10172000511D29013A01A11432E0B30609F088C025
:1017300080914B0790914C07A0914D07B0914E07B7
:1017400084159505A605B70569F4109253078FEF28
:101750009FEFDC0180934B0790934C07A0934D07BC
:10176000B0934E079401B301A20180915407909168
:101770005507EDDE882309F485CFF8018085918532
:10178000A285B3858A0D9B1DA11DB11D8087918700
:10179000A287B3878A0C9B1CCA18DB08D80118964D
:1017A0004D915D916D917C911B97C114D10409F00D
:1017B00071CF7CC0E114F10409F085CF14964D91EE
:1017C0005D916D917C9117974115510561057105EA
:1017D00059F455968D919D910D90BC91A02D009737
:1017E000A105B10539F521C09E012F5F3F4F0E9431
:1017F00018B1882309F446CF89819A81AB81BC81D5
:10180000F801218D328DF9012789203139F4883F83
:10181000FFEF9F07A105B10540F40CC0883F2FEFF3
:101820009207A2072FE0B20728F0C80183DB8111DD
:101830004ACF28CFF80184839583A683B78343CF0B
:10184000E114F10419F5D80118964D915D916D914F
:101850007C911B9751968D919D910D90BC91A02DDF
:10186000481759076A077B0788F00E940FB0882342
:1018700009F408CF81E08093530740924B075092C0
:101880004C0760924D0770924E0708C041E0C301BB
:10189000B2010E944FB0882309F4F4CEA501B4012F
:1018A000C701855B9A4F0F944A0867CF51968D9177
:1018B0009D910D90BC91A02D84179507A607B707A1
:1018C00040F4F801418B528B638B748B818180686B
:1018D0008183D80111968C9183FD02C0C10105C09E
:1018E000C8014DDD8111FACFCDCE0F900F900F9032
:1018F0000F90DF91CF911F910F91FF90EF90DF90AC
:10190000CF90BF90AF909F908F907F906F905F909F
:101910004F903F902F900895EF92FF920F931F9357
:10192000CF93DF93EC0179018C81833039F089E02A
:10193000440F551F661F771F8A95D1F79A01AB0197
:1019400061E1CE0193DD882329F084E08983CE0113
:1019500083DD38C00E9410508B010E9444728B833B
:101960008F3F49F40E941050601B710B6D32714023
:10197000A0F381E103C08E3F39F08FE08983CE016F
:101980006BDD8FEF6EDD1EC08FEF8EBDF701D701CF
:10199000A150BE4F0DB407FEFDCF9EB591938EBDF5
:1019A000EA17FB07B9F70DB407FEFDCF8EB58C9390
:1019B0000E9444720E944472CE014EDD8FEF51DDD1
:1019C00081E001C080E0DF91CF911F910F91FF90E6
:1019D000EF9008952F923F924F925F926F927F9275
:1019E0008F929F92AF92BF92CF92DF92EF92FF922F
:1019F0000F931F93CF93DF9300D01F92CDB7DEB725
:101A00009C838B834B015A01DC0113968C918111CD
:101A100003C08FEF9FEFEAC0EB81FC81818180FFE3
:101A2000F8CFAB81BC8151960D911D912D913C91C8
:101A3000549718964D915D916D917C911B97C501BE
:101A4000A0E0B0E068017901C41AD50AE60AF70AF5
:101A5000C816D906EA06FB0618F45801A41AB50AF6
:101A600075018B819C8104969A838983612C92E015
:101A7000792EE114F10409F48BC0AB81BC81189676
:101A80004D915D916D917C911B976A01B1E0DB22D4
:101A9000EB81FC8123811A012B0189E05694479444
:101AA000379427948A95D1F7818D928D223061F4F5
:101AB000FC01828D938DA48DB58DBC01CD01620D8D
:101AC000731D841D951D4AC0DC0114961C91115094
:101AD0001221C114D10401F511111EC0452B462B52
:101AE000472B59F4EB81FC8185899689A789B08DB4
:101AF00084839583A683B7830FC0AB81BC81149682
:101B00004D915D916D917C91179729813A810E9449
:101B100018B1882309F47DCFEB81FC81218D328DB2
:101B200084819581A681B7810297A109B109F90144
:101B3000058404C0880F991FAA1FBB1F0A94D2F7FF
:101B40004685578560897189840F951FA61FB71F29
:101B5000BC01CD01610F711D811D911D93012C19D7
:101B60003D0987012E153F0508F489010115F2E0B2
:101B70001F0771F520914B0730914C0740914D079D
:101B800050914E07621773078407950719F420C018
:101B9000C5012CC09401AB01BC0180915407909108
:101BA0005507BADE882309F434CF800E911EEB81ED
:101BB000FC8180859185A285B385800F911FA11D31
:101BC000B11D80879187A287B387E01AF10A51CFB0
:101BD00040E00E944FB0882309F41BCFB601655B3B
:101BE0007A4FA801C4010F944A08DFCF0F900F90DD
:101BF0000F900F90DF91CF911F910F91FF90EF9079
:101C0000DF90CF90BF90AF909F908F907F906F901C
